:020000040800F2
:100000000000012029AB0508A9AB05083D750408CF
:10001000C1750408A9AB0508A9AB050800000000DC
:10002000000000000000000000000000A9AB05086F
:10003000A9AB050800000000A9AB05088D2E040837
:10004000A9AB0508A9AB0508A9AB0508A9AB05082C
:10005000A9AB0508A9AB05082D810408598204083D
:100060001D820408E1810408A5810408158E050895
:10007000058E0508F58D0508E58D0508D18D050867
:10008000BD8D0508A98D0508A9AB0508A9AB050814
:10009000A9AB0508A9AB0508A9AB05086981040847
:1000A000955105081D52050885510508455205085A
:1000B0000D520508FD510508ED510508DD940508B0
:1000C000019505082194050845940508A9AB050884
:1000D000A9AB0508653A04081D380408D53504089D
:1000E000F1800408A9AB0508A9AB050875510508FE
:1000F000A5510508A9AB0508CD510508958D050842
:10010000A9AB0508A9AB0508DD510508A9AB050891
:100110008D33040845310408A9AB050835F60008FD
:10012000818D05086D8D0508598D0508458D0508DB
:10013000318D0508000000000000000000000000F4
:100140000000000000000000000000009509010808
:100150001D8D0508098D0508F58C0508FD2E040880
:100160005D93050885930508A9AB0508A9AB0508AB
:10017000A9AB0508A9AB05080000000000000000BD
:10018000A9AB0508A9AB0508A9AB0508A9AB0508EB
:10019000A9AB0508A9AB050800000000A9AB05083C
:1001A000000000000000000000000000A9AB0508EE
:1001B000A9AB0508A9AB050800000000000000007D
:1001C000000000000000000000000000000000002F
:1001D000000000000000000000000000A9AB0508BE
:0801E00080A6050001000000EB
:1001E8002320010010000000A4580120B459012068
:1001F80000000000F92002080D1001007000000046
:1002080028580120C45901200000000091A30308C8
:10021800040008008000000068570120345A0120BB
:100228000000000000000000FD01010024000000A3
:100238000C570120B45A012000000000E709040807
:10024800FB01010001000000C8560120D85A012016
:100258000000000071200508FC01010009000000F1
:1002680094550120DC5A0120000000008120050877
:10027800F70101000600000088550120E85A012016
:100288000000000080090008F901010004000000D6
:1002980084550120F05A012000000000950A040846
:1002A8000A8001002800000020550120F45A01208E
:1002B80000000000E51F0208160215003F000000BC
:1002C800E82901201C5B012000000000012005082E
:1002D80034000100100000004C5401205C5B012038
:1002E8000000000071A702081102010008000000C8
:1002F800245401206C5B01200000000086090008DE
:1003080012120100040000001C540120745B01203B
:10031800000000008E0900081820010032000000CB
:10032800E8530120785B0120000000000D2105083A
:10033800061001001C000000CC290120AC5B012044
:1003480000000000A1200508122001001100000093
:10035800EC520120C85B012000000000920900084F
:10036800000201000B00000028500120DC5B012086
:100378000000000011160508130201000400000027
:10038800C8290120E85B012000000000A40900083A
:10039800FA01010003000000AC4F0120EC5B0120D2
:1003A80000000000F5150508020201000300000026
:1003B80094490120F05B01200000000000000000CB
:1003C8000C0201000400000070490120F45B0120C8
:1003D80000000000DD150508110001000C000000F8
:1003E800E5360120F85B012000000000B59F0308F6
:1003F800FE0101001400000070350120045C01209A
:1004080000000000751605080B3001001A000000F6
:100418009C5F01204864012000000000A809000832
:100428001F30010024000000645F01206464012083
:1004380000000000C40900080502010004000000D3
:10044800F46001208864012000000000E809000829
:10045800030101000A000000005F01208C640120F4
:1004680000000000D91C0108220201001C01000044
:10047800A87001207873012000000000B91F05084A
:100488000C200600CC000000206F0120947401208D
:10049800000000001D9E0308010201000B0000007F
:1004A800886E012060750120000000000116050813
:1004B8001B020100100000005C6E01206C75012019
:1004C80000000000B91505081B1001000C00000011
:1004D800446701207C75012000000000A5AC0108DC
:1004E80021020100F0000000C46501208875012088
:1004F800000000000DAC01082312010010000000EC
:10050800706B01207876012000000000EC090008DB
:10051800371001002E000000D86D012088760120D8
:1005280000000000FC0900080E02010002000000A3
:100538006C6B0120B8760120000000002A0A000830
:100548001610010006000000646B0120BC76012033
:10055800000000002C0A00082F10010022000000F3
:10056800C8720120C476012000000000320A000889
:100578001E00010009000000A46A0120E87601209D
:1005880000000000540A00080510010006000000E1
:10059800F06A0120F4760120000000005E0A0008DD
:1005A800F58101006800000054650120FC760120F7
:1005B80000000000A59D0108FD070100760000006D
:1005C80098640120647701200000000089850108F3
:1005D800261001000E000000EC770120DC770120D6
:1005E80000000000018401082C0004001000000035
:1005F8005887012048870120000000008540020834
:100608002B001200240000008C870120688701203D
:10061800000000005940020829201400780000005A
:10062800B8850120B087012000000000000000000C
:10063800F62101000C000000F08301202888012029
:1006480000000000640A00081C0202001C000000F0
:10065800788401207888012000000000D939050835
:100668000412010002000000008501209488012086
:1006780000000000700A00080F02010001000000DD
:10068800FC8401209888012000000000720A0008FC
:100698001400010004000000B08301209C880120A0
:1006A80000000000740A0008012001000C0000008E
:1006B800D87A0120A088012000000000780A0008EC
:1006C8000EF003009E010000C0780120AC880120D4
:1006D80000000000919C02081300010004000000C3
:1006E800908001204C8A012000000000840A000844
:1006F80001010100040000000C780120508A01204B
:1007080000000000000000000001010004000000DB
:1007180004780120548A012000000000880A00089B
:10072800020101000300000000780120588A01201E
:10073800000000005D9E030819000100050000008C
:100748009490012014910120000000008C0A0008F8
:100758001A0001000E000000008F01201C910120EA
:1007680000000000920A0008203201000A00000080
:10077800F08D01202C910120000000006D9C0208E2
:1007880015001000700000003C8C012038910120F9
:1007980000000000000000002A00080060000000BF
:1007A800488F0120A891012000000000459C020804
:1007B8000300010001000000E4950120CC9A01200B
:1007C8000000000000000000031201003D000000CE
:1007D8007C950120D09A012000000000A00A0008A2
:1007E80025201E002C010000E4920120109B01200E
:1007F80000000000000000001010010002000000CE
:100808006C9201203C9C012000000000DE0A0008D8
:10081800F821010006000000C0920120409C012040
:1008280000000000E00A0008020001000C000000BF
:1008380068A00120FCA001200000000000000000CA
:100848002902010040000000389F012008A1012072
:1008580000000000E60A00080A0201001400000077
:10086800AC9E012068A1012000000000799F0308C8
:100878002802040004000000B8A5012050A70120A8
:1008880000000000D9150508270204000400000034
:10089800B4A5012054A7012000000000CD150508CB
:1008A8001F02080010000000F8A2012058A701202C
:1008B80000000000711505081A0201003C00000044
:1008C800BCA2012068A70120000000007D210508C6
:1008D80038100100010000009CA10120A4A70120FC
:1008E80000000000260B000827000100040000009B
:1008F8002CA8012030A8012000000000280B0008C7
:10090800070201000200000010B2012028B20120F5
:10091800000000002C0B00081D0202000600000069
:1009280074B101202CB2012000000000000000007A
:10093800060204001000000090B1012034B201202A
:10094800000000007D1E05080812040014000000C5
:100958007CB1012044B201200000000019160508EE
:10096800100201000100000090D101208CD101206B
:08097800000000002E0B000836
:100980002001000000002B00000001010101FFFF19
:10099000FFFF000000010000054C41494F0000002E
:1009A0000002000000000100AE014A015E012C01BE
:1009B00064010100000001000A019A01001E0A0002
:1009C000000200000000000000010000000500001F
:1009D0000102030000000000000000000000000011
:1009E0000000000000800700000000000000000080
:1009F00000000000000000000000000020003200A5
:100A0000C800D00796001400320028004C044006AD
:100A10000005500014000F000800640001000000F1
:100A200005000A000000F40196000000C40900005F
:100A3000190000000000000000000000000000009D
:100A400000000000000000000000000000000000A6
:100A50000000000000050100000000000000200070
:100A6000010100000000000001000000020200007F
:100A70000000000003000023E8036400040A0001F2
:100A800014001E0008004530A300000000002801EB
:100A900000007E05EA05B4053200E803D007000037
:100AA0000000000000000000000000000000000046
:100AB0000000000000000000000000000000000036
:100AC0000000000000000000000000000000000026
:100AD0000000000000000000000000000100000510
:100AE0000101F401140000000000000000000000FB
:100AF00000000000000000000000000000000000F6
:100B000000000000000000000000000000000000E5
:100B100000000000000000000000000000000000D5
:0F0B2000000000000000000020030000013C0066
:100B2F0000C20100000008000A0600020000004099
:100B3F000100000009026400030100C03209040033
:100B4F0000010300000009211101000122360007F6
:100B5F0005830308000A080B0102020201000904C1
:100B6F00010001020201000524001001052401000B
:100B7F00020424020205240601020705820308006D
:100B8F00FF09040200020A000000070501024000ED
:100B9F00000705810240000071080108699A0008EA
:100BAF008907010800000000418C0008F19200083D
:100BBF006D8C000800000000000000000000000025
:100BCF00218C0008318C0008118C0008018C000862
:100BDF001A030000000000000000000000000000E9
:100BEF0000000000000000000000000004030904E2
:100BFF000A06000200000040010000000907200063
:100C0F00010104C03209040000020806500507055F
:100C1F008102400000070501024000000902200088
:100C2F00010104C03209040000020806500507053F
:100C3F008102400000070501024000000902200068
:100C4F00010104C03209040000020806500507051F
:100C5F008102000200070501020002000A060002DD
:100C6F00000000400100000009022200010100E025
:100C7F0032090400000103010200092111010001E2
:100C8F002236000705830308000A0000090222002C
:100C9F00010100E0320904000001030102000921F3
:100CAF001101000122360007058303080007000029
:100CBF0009022200010100E03209040000010301D2
:100CCF0002000921110100012236000705830308E4
:100CDF00000A00000A0600020000004001000000A8
:100CEF0009074300020104C0320904000001020297
:100CFF000100052400100105240100010424020253
:100D0F0005240600010705820308001009040100ED
:100D1F00020A0000000705010240000007058102DA
:100D2F004000000009024300020100C03209040024
:100D3F000001020201000524001001052401000139
:100D4F00042402020524060001070582030800108F
:100D5F0009040100020A0000000705010200020059
:100D6F00070581020002000009024300020100C0D2
:100D7F0032090400000102020100052400100105E0
:100D8F002401000104240202052406000107058244
:100D9F000308001009040100020A00000007050102
:100DAF00024000000705810240000000120100020E
:100DBF000000004083042A570002010203010000D3
:100DCF00120100020200004083044057000201029A
:100DDF000301000012010002EF02014083045632AA
:100DEF00000201020301000005010905A101A10094
:100DFF00050109300931093209330935093409363A
:100E0F0009371581257F7508950881020509190194
:100E1F00290815002501950875018102C0C0000041
:100E2F00092111010001223600000000000000001E
:100E3F000401000000070000000000000000000097
:100E4F000002000010000000000000000000000081
:100E5F0007000000100000007D00000001000000EE
:100E6F000000803F00FF0000000000000000AA55B6
:100E7F000701000001AA5505010000082CEF050825
:100E8F00FF1FFF1F2D202D2D202D2D2D2D202D2D22
:100E9F002D2D0000000000000000000000000000E9
:100EAF00000000AA550B010000AA5505010000AA79
:100EBF00550902000000AA5503009F000100000021
:100ECF00C0120000406401200000000018640120DF
:100EDF0000000000947106089C71060800000000D5
:100EEF00D19E0308A086010004000000000000004E
:100EFF0000000000000000000000000000000000E3
:100F0F0000000000000000000000000000000000D2
:100F1F000000000094710608A4710608000000008C
:100F2F001D070408E8030000040000000000000093
:100F3F0000000000000000000000000000000000A2
:100F4F000000000000000000000000000000000092
:100F5F0000000000AC710608000000000000000057
:100F6F00B90F00007D000000FF000000000000002E
:100F7F000000000000000000000000000000000062
:100F8F000000000000000000000000000000000052
:100F9F0000000000ACF00608000000000000000098
:100FAF00ED0500007D000000FF00000000000000C4
:100FBF000000000000000000000000000000000022
:100FCF000000000000000000000000000000000012
:100FDF00000000008C8706080000000000000000E1
:100FEF00351100007D000000FF0000000000000030
:100FFF0000000000000000000000000000000000E2
:10100F0000000000000000000000000000000000D1
:10101F0000000000B471060800000000000000008E
:10102F0081120408E8030000030000000000000024
:10103F0000000000000000000000000000000000A1
:10104F000000000000000000000000000000000091
:10105F0000000000B871060800000000000000004A
:10106F00C50B03081027000003000000000000005C
:10107F000000000000000000000000000000000061
:10108F000000000000000000000000000000000051
:10109F0000000000C0EC060800000000753C0208CC
:1010AF002D7604085F7600000500000000000000A8
:1010BF000000000000000000000000000000000021
:1010CF000000000000000000000000000000000011
:1010DF000000000050F006080000000000000000B3
:1010EF00E990040810270000010000000000000034
:1010FF0000000000000000000000000000000000E1
:10110F0000000000000000000000000000000000D0
:10111F0000000000C471060800000000000000007D
:10112F0021070408E803000005000000000000008C
:10113F0000000000000000000000000000000000A0
:10114F000000000000000000000000000000000090
:10115F0000000000D0710608000000000000000031
:10116F00F1A10308204E0000030000000000000062
:10117F000000000000000000000000000000000060
:10118F000000000000000000000000000000000050
:10119F0000000000E07106080000000000000000E1
:1011AF00D99F0308204E000003000000000000003C
:1011BF000000000000000000000000000000000020
:1011CF000000000000000000000000000000000010
:1011DF0000000000F0710608000000000000000091
:1011EF00C1170408400D03000300000000000000B9
:1011FF0000000000000000000000000000000000E0
:10120F0000000000000000000000000000000000CF
:10121F00000000000072060800000000000000003F
:10122F00D5CF0308102700000100000000000000C8
:10123F00000000000000000000000000000000009F
:10124F00000000000000000000000000000000008F
:10125F0000000000087206080000000000000000F7
:10126F00C5B80108102700000300000000000000AF
:10127F00000000000000000000000000000000005F
:10128F00000000000000000000000000000000004F
:10129F00000000000C7206080000000000000000B3
:1012AF000111040850C300000100000000000000FD
:1012BF00000000000000000000000000000000001F
:1012CF00000000000000000000000000000000000F
:1012DF00000000001472060800000000000000006B
:1012EF00CD0E0408A08601000000000000000000E1
:1012FF0000000000000000000000000000000000DF
:10130F0000000000000000000000000000000000CE
:10131F00000000002072060800000000000000001E
:10132F00B90A0408A86100000100000000000000D5
:10133F00000000000000000000000000000000009E
:10134F00000000000000000000000000000000008E
:10135F00000000002C7206080000000000000000D2
:10136F002D0C0208A0860100010000000000000003
:10137F00000000000000000000000000000000005E
:10138F00000000000000000000000000000000004E
:10139F000000000038720608000000000000000086
:1013AF00B9400408A00F0000010000000000000079
:1013BF00000000000000000000000000000000001E
:1013CF00000000000000000000000000000000000E
:1013DF00000000004472060800000000000000003A
:1013EF004D1302081027000001000000000000004C
:1013FF0000000000000000000000000000000000DE
:10140F0000000000000000000000000000000000CD
:10141F0000000000507206080000000000000000ED
:10142F0019A60308A00F0000010000000000000033
:10143F00000000000000000000000000000000009D
:10144F00000000000000000000000000000000008D
:10145F00000000005C7206080000000000000000A1
:10146F0055EA01081A4100000100000000000000C9
:10147F00000000000000000000000000000000005D
:10148F00000000000000000000000000000000004D
:10149F00000000006072060800000000000000005D
:1014AF00111D0108102700000100000000000000BE
:1014BF00000000000000000000000000000000001D
:1014CF00000000000000000000000000000000000D
:1014DF00000000006C720608000000000000000011
:1014EF00F955020850C30000010000000000000081
:1014FF0000000000000000000000000000000000DD
:10150F0000000000000000000000000000000000CC
:10151F0000000000707206080000000000000000CC
:10152F0075230108400D03000000000000000000BB
:10153F00000000000000000000000000000000009C
:10154F00000000000000000000000000000000008C
:10155F000000000078720608000000000000000084
:10156F000D9F0308400D0300000000000000000065
:10157F00000000000000000000000000000000005C
:10158F00000000000000000000000000000000004C
:10159F00000000008072060800000000000000003C
:1015AF00B1F8010850C30000030000000000000064
:1015BF00000000000000000000000000000000001C
:1015CF00000000000000000000000000000000000C
:1015DF00000000008C7206080000000000000000F0
:1015EF00BDAF030840420F000000000000000000E4
:1015FF0000000000000000000000000000000000DC
:10160F0000000000000000000000000000000000CB
:10161F0000000000987206080000000000000000A3
:10162F00D9A6030850C3000000000000000000000E
:10163F00000000000000000000000000000000009B
:10164F00000000000000000000000000000000008B
:10165F00000000000100000000000100E001000098
:10166F00FFFFFFFF01000000D98E010800000000FE
:10167F000000000058F105087EFF0000FFFFFFFF8C
:10168F000800000042570200000001064257020006
:10169F00000001060101FF0101FF0000FFFFFFFF36
:1016AF00B507020800000000000000001CFB050841
:1016BF00DD0A02080000000000000000D4FA05084F
:1016CF002D202D2D202D2D2D2D202D2D2D000000E9
:1016DF0000000000000000000000000000000000FB
:1016EF0000000000000000000000000090FA050854
:1016FF00A06001209CFF2C01000000005872012007
:10170F00E0150C1700000000EC6F01200200000034
:10171F00C8FA0508986A012088136F1701000000A6
:10172F009A6A012088136F17000000003E590120AC
:10173F0000000000000000003C59012000000000E4
:10174F00000000003A5901200000000000000000D6
:10175F003859012000000000000000003659012018
:10176F0000000000000000003459012000000000BC
:10177F0000000000A0030120000000000000000096
:10178F00FC69012003000000B8FB0508906A0120E6
:10179F0088136F1701000000EA60012088136F178C
:1017AF0000000000A18F01080000000000000000F1
:1017BF00C8FB0508ED6F0120010000001CFC0508A7
:1017CF00EC6001200100000028FC0508E260012008
:1017DF000200000030FC05080000000000000000BF
:1017EF00000000003CFC0508898F01080000000084
:1017FF0000000000D8FC05080000000000000000F9
:10180F00000000002CFD0508000000000000000093
:10181F00000000009CFD05089C6A012002000000EA
:10182F00D4FD0508E6600120E0150C17000000004C
:10183F00807C0120D47C0120D60101000000000033
:10184F000000000000000000D81306080000000090
:10185F0000000000000000009014060800000000C7
:10186F0000000000000000003C140608000000000B
:10187F0000000000B54402083D800120FF00000079
:10188F00FFFFFFFF79430208000000000000000087
:10189F006813060801000000FA00000001000000B4
:1018AF000100000001000000000101010000000024
:1018BF00D27A01200000F40101000000D07A01204B
:1018CF000000F40101000000CE7A01200000F401B5
:1018DF0001000000CC7A01200000F401010000009B
:1018EF00CA7A01200000F40101000000C87A01202B
:1018FF000000F40101000000C67A01200000F4018D
:10190F00010000004D1E0208111E02080000000019
:10191F00E8FF0508B67A012005320100C47A0120DC
:10192F006400F40101000000C27A01206400C409C0
:10193F0001000000B47A0120E803D0070100000085
:10194F00B27A0120E803D00701000000B07A01202D
:10195F00E803D00701000000AE7A01201E00B80B8B
:10196F0001000000BC7A012005000F0001000000FB
:10197F00BE7A012003000A0001000000AC7A0120AA
:10198F001E00F40101000000C07A012002000000D7
:10199F0074000608AA7A01201400640001000000F8
:1019AF00B87A01203200E80301000000A87A012074
:1019BF000000C80001000000817A012000C801006A
:1019CF00807A0120005001007F7A0120005A010027
:1019DF007D7A01200200000080000608E07E0608E4
:1019EF00E87E0608FA5801200100C4090000000033
:1019FF00F85801200100C40900000000F65801202A
:101A0F000100C40900000000F45801200100C409BE
:101A1F0000000000F05801200100C4090000000080
:101A2F00F25801200100C40900000000EE58012007
:101A3F000100C40900000000EC5801200100C40996
:101A4F00000000002B78012000C801002A78012037
:101A5F0000C80100287801200000FFFF0A000000E5
:101A6F00267801200100C800010000002478012021
:101A7F003200307532000000227801207EFF140002
:101A8F00050000002078012005002C010500000052
:101A9F001E780120055A05001B78012000FF010068
:101AAF001D78012002000000BC0E012019780120D2
:101ABF0003000000B4F205081A78012000FF0100AE
:101ACF001C78012002000000BC0E012018780120B4
:101ADF0003000000B4F20508A11D0208311D020821
:101AEF00000000008C000608E87A0120EE02CA0808
:101AFF0001000000E67A012000C801006400000028
:101B0F00E57A012000C8010064000000E47A01209A
:101B1F000200000098010608127801200000803EA4
:101B2F00050000001078012080C1803E05000000F4
:101B3F000A7801200083007D05000000087801204D
:101B4F0080C1803E050000000378012000FF0100E6
:101B5F00FE7701206400F40101000000FD770120F1
:101B6F0004000000A4010608FC7701200200000019
:101B7F00B8010608B17801200D000000C401060865
:101B8F00AE78012000640100AC78012032001027EC
:101B9F000A000000AA7801200D000000C401060809
:101BAF00A97801200D000000C4010608A8780120C3
:101BBF0002000000FC010608000000000000000009
:101BCF000000000008020608EE7A01203E00000027
:101BDF0040020608EC7A01200100FF7F010000009F
:101BEF00EB7A0120020000003C030608B3780120C5
:101BFF00030000004C030608B27801200300000028
:101C0F004C0306086E7A0120000A01006C7A01204D
:101C1F000000E803010000006A7A01200000E803D9
:101C2F0001000000687A01200000E80301000000B5
:101C3F00667A01200000E803010000005E7A0120AF
:101C4F000000E80301000000647A01200000E803AF
:101C5F0001000000627A01200000E803010000008B
:101C6F00607A0120001401007C7A0120020000003C
:101C7F005C0306087A7A01200000F40101000000DD
:101C8F00787A01200000F40101000000767A01202B
:101C9F000000F40101000000747A01200000F4013B
:101CAF0001000000727A01200000A00F0100000067
:101CBF00707A01200000A00F01000000957A01202A
:101CCF0019640100947A01200200000068030608DD
:101CDF00927A0120E803D0070A000000907A0120D1
:101CEF00006401000A000000857A012000640100F1
:101CFF00847A0120006401008C7A012000640100C5
:101D0F000A0000008B7A0120006401000A00000025
:101D1F008A7A0120006401000A0000008F7A0120F6
:101D2F0000FF01000A0000008E7A012000FF010071
:101D3F000A0000008D7A012000FF01000A00000058
:101D4F00897A012001FF01000A000000887A012032
:101D5F0001FF01000A000000877A012001FF010046
:101D6F000A000000BC7801200000F401010000000F
:101D7F00BA7801200000A00F01000000B878012000
:101D8F000000A00F01000000B67801200000A00F96
:101D9F0001000000B47801200000A00F0100000036
:101DAF00A580012000C80100A4800120006401006B
:101DBF00A380012000640100A280012000640100C3
:101DCF00A180012000640100A0800120FF08010014
:101DDF009F80012001640100991C02085D1C02080C
:101DEF000000000074030608A880012001320100E2
:101DFF00A780012001000000E4030608A68001204F
:101E0F0004000000EC0306089E800120006401001E
:101E1F009C8001201400E803010000009A8001203B
:101E2F00E80330750A0000009880012000C8010007
:101E3F009780012000C801009680012000C8010092
:101E4F009580012000320100AA800120004B010083
:101E5F00A9800120040000000004060894800120DE
:101E6F00006401000A000000B88001200000D007C4
:101E7F0001000000B380012000C80100B2800120E2
:101E8F0000C80100B180012000C80100B680012008
:101E9F000000D00701000000B080012000C8010041
:101EAF00AF80012000C80100AE80012000C80100F2
:101EBF00B48001200000D00701000000AD80012098
:101ECF0000C80100AC80012000C80100AB800120D8
:101EDF0000C80100511A0208391A02080000000058
:101EEF0014040608A5780120005A0100A4780120E7
:101EFF0000C80100A2780120E803D007010000000C
:101F0F000000000000000000F5440208B0040608BD
:101F1F004C555841494F000017780120000301002C
:101F2F0016780120000301007D19020839190208F3
:101F3F00000000000405060801190208C118020874
:101F4F0000000000A0050608C11902085D43020841
:101F5F00000000002006060814780120010301008C
:101F6F00291F0208FD1E020800000000780906085C
:101F7F00691802083918020800000000E80906086D
:101F8F00611A0208C145020800000000840A060811
:101F9F00F5480208551F0208000000002C0B060828
:101FAF00B11A02080000000000000000B80B06087C
:101FBF008D1B0208351B0208000000001C0C0608D0
:101FCF00211C0208E51B020800000000C40C0608D3
:101FDF006D940208D51C020800000000500D060881
:101FEF00A77A012001060100F91A0208C51A020892
:101FFF00000000004C0E0608A39302088D4602084D
:10200F0000000000BC0E0608B594020855470208F0
:10201F00000000000C100608A67A01200103010041
:10202F00091A0208D919020800000000E01006087A
:10203F00119502080000000000000000441106087E
:10204F00991802084543020800000000C411060851
:10205F000000000000000000000000005012060801
:10206F00091D0208CD47020800000000C012060833
:10207F00FFFFFFFF0000803F000000000000000096
:10208F000000000000000000000000000000000041
:10209F000000000000000000000000000000803F72
:1020AF000000000000000000000000000000803F62
:1020BF000000000000000000000000000000803F52
:1020CF000000000000000000000000000100000000
:1020DF000000FA430000FA430000803FE5D10308F7
:1020EF00000000000000000000000000FFFFFFFFE5
:1020FF00FF0000000000000058A1012008000000B0
:10210F000000000048A1012008000000818900089C
:10211F006589000821890008000000001589000862
:10212F0001890008ED880008000000000000000091
:10213F000000000000000000DD8800080000000023
:10214F00CD8800087D8F0008698B0008318B00084F
:10215F00458B0008E98A0008D58A0008C18A000863
:10216F00459B0008C988000845880008DDFB00086A
:10217F00685E0C00FFFFFFFF0200000000600240DE
:10218F00106002400000000000000000000B000083
:10219F00000000000000000000000000006002408E
:1021AF00286002400100000000000000060C000043
:1021BF00000000000000000000000000006002406E
:1021CF00406002400200000000000000100D0000FF
:1021DF00000000000000000000000000006002404E
:1021EF00586002400300000000000000160E0000BF
:1021FF00000000000000000000000000006002402E
:10220F00706002400400000000000000200F00007A
:10221F00000000000000000000000000006002400D
:10222F00886002400500000000000000261000003A
:10223F0000000000000000000000000000600240ED
:10224F00A0600240060000000000000030110000F6
:10225F0000000000000000000000000000600240CD
:10226F00B86002400700000000000000362F000099
:10227F0000000000000000000000000000640240A9
:10228F001064024000000000000000000038000051
:10229F000000000000000000000000000064024089
:1022AF002864024001000000000000000639000011
:1022BF000000000000000000000000000064024069
:1022CF00406402400200000000000000103A0000CD
:1022DF000000000000000000000000000064024049
:1022EF00586402400300000000000000163B00008D
:1022FF000000000000000000000000000064024029
:10230F00706402400400000000000000203C000048
:10231F000000000000000000000000000064024008
:10232F008864024005000000000000002644000001
:10233F0000000000000000000000000000640240E8
:10234F00A0640240060000000000000030450000BD
:10235F0000000000000000000000000000640240C8
:10236F00B86402400700000000000000364600007D
:10237F00000000000000000000000000010000004D
:10238F00A00F0000B80B00000102FFFF01000000CA
:10239F00FFFF0000B4EC060800000802050304006C
:1023AF0000000000BCEC0608010008020504040050
:1023BF0000000000EC9A06080200FE010110030065
:1023CF00000000003C820608030014020003000016
:1023DF0000000000C4EC060804001F020200080001
:1023EF0000000000CCEC060805001F0202010800E7
:1023FF0000000000FFFFFFFF05FC0008159A000812
:10240F00ED0501080000000000000000B5050108FF
:10241F00BD040108000000000000000000000000E3
:10242F00A58B0008958B0008858B0008758B00081D
:10243F0009220508D5160508D1160508CD16050879
:10244F0085240508C9160508C51605084C66060833
:10245F000000000040000000010000000004000028
:10246F001F0000001C0000001F0000001E000000E5
:10247F001F0000001E0000001F0000001F000000D2
:10248F001E0000001F0000001E0000001F000000C3
:10249F000068214CFFFF0100F4010000EC6F0608FB
:1024AF00B001000002000000090000000100000060
:1024BF00941901200000000000000000000000003F
:1024CF0000000000000000000000000000000000FD
:1024DF0000000000000000000000000000000000ED
:1024EF0000000000000000000000000000000000DD
:1024FF0000000000000000000000000000000000CD
:10250F0000000000000000000000000000000000BC
:04251F0000000000B8
:10252300010000000100000024230020000000003F
:042533002000000084
:082800000000000000000000D0
:10800000026C03463AB11A6CD20608D50022012050
:1080100083F83C207047426480F83C20F3E71A6CF8
:1080200049494A4811401A6841F00201F0B4196404
:108030004168474D21F44031416041685C6821430B
:1080400041605168186921F48071D3F808C0DF6875
:10805000516054689E6A44EA0024AE4254605468F9
:1080600024F040745460506840EA0C0050609068FE
:1080700020F400609060916841EA0701916054D05B
:108080009068DC6A20F07060906091680E439660A2
:10809000906820F040509060916821439160906812
:1080A0009C6920F002009060916841EA440191606F
:1080B00093F82010002941D05468596A44F40064B0
:1080C000481E5460516821F460415160516841EA92
:1080D00040315160D06A0025DC6920F470005E698F
:1080E000611ED0622846D46A44EA0154D46294687E
:1080F00024F400749460946893F8301044EA4124A6
:108100009460946824F480649460916841EA8621C4
:1081100091605D641A6C22F0030242F001021A645D
:10812000002283F83C20F0BC7047916821F0706118
:108130009160916821F040519160B0E7516821F45D
:1081400000615160C6E700BFFDEEFFFF0023014064
:108150000100000F2DE9F04F022389468A462DEDDC
:10816000108B99B0DFEDCABA14930346169004330E
:10817000159217934FEADA06169DDDF85CC04FEAB8
:10818000CA0305EB46111396F0004FF0000B01EB0C
:10819000061437010390A6EB86020194049706EBC0
:1081A000460E04EBC202041D381D06EB86072C4464
:1081B000C6EBC60802972844029D02EB46174FEA19
:1081C000C808ED0001EBC60602954FEA0E150595AD
:1081D0004FEACE050695139D4FEA451E019D95ED8C
:1081E000007AD34492ED005AD7ED004AD945D1ED3B
:1081F000006A50ED013A35EE241AD6ED002A1CED46
:10820000016A73EE875A54ED017A33EEC73A36EEBF
:10821000264A77EEA21A36EE666A77EEE27A74EEB6
:10822000256A71EE812A77EE633A37EEC57A36EE2B
:10823000A22A77EEE47A76EEE26A0CED012A37EEB6
:10824000247A77EE857AD1ED018AC1ED006A74EE69
:10825000655A96ED015AB0EE460A94ED004AA7EE33
:108260002B6AD2ED010AE7EEAB3A74EE456AD7ED20
:10827000012AA7EE6B0A9CED007AD5ED014A34EE97
:10828000054A37EE689A90ED005A36EEE02A76EE0F
:10829000E26A30EEA28A32EE222A76EEA06AF0EE90
:1082A000492A75EE640A37EE287A75EE249AE2EED2
:1082B0006B2A74EEC54AF0EE608AB0EE40AAE6EE94
:1082C000AB4AE6EEAB8AA6EEEBAAF0EE496AB0EE58
:1082D000629A37EE695AE2EE2B6AB0EE432A74EEE8
:1082E00008AAA7EEEB9AA7EEAB2A77EE297A35EE2D
:1082F000617A75EEC89A35EE415A75EEC45A37EE7A
:10830000AABA77EEEA7A37EE011A8CED00BA36EEA9
:10831000287AC1ED017A39EE844A76EEC27A1944A0
:1083200075EE885A9C4435EE215A00ED014A70EEF4
:108330008A0A70EE244AC5ED005A36EE686A80ED6E
:10834000001A72EEA33A85ED015A33EE093A04EDB4
:10835000017A72EE266A87ED006A1D44C6ED000AB6
:108360001844C2ED004AC4ED007A1C44C7ED016A0E
:108370001F44C6ED013A1E4482ED013A1A443FF60D
:108380002EAF139A072A40F2C681039A0EF1080E07
:10839000169F08F108000832029E059D4FF0000864
:1083A00094463A46083608357244069C0499D346EA
:1083B000109207EB0C0208340C310F92BA190E928E
:1083C0007A190D923A190C923A180B927A1809926E
:1083D00007F10C020A9201220892149ADDF824C0D7
:1083E0009044159A0A9F02EBC8020B9EA8EB880ED8
:1083F0000C9D02EBC80192ED00BA0D9C01EBC80286
:10840000D1ED00AA0E9802EBC80192ED00AA01EB93
:10841000C802D1ED009A02EBC80192ED009A01EB7F
:10842000C802D1ED008A0F9902EB0E1E92ED008A70
:10843000109A0EEBC80ADEED017A1192CDED047AA6
:108440000AEBC802DAED017A02EBC80A1291CDED0F
:10845000057AD2ED017A0AEBC802DDF820E0CDED15
:10846000017ADAED017A02EBC80ACDED067AD2ED97
:10847000017A0AEBC802CDED027ADAED017ACDED90
:10848000077AD2ED017ADDE91121CDED037A01E021
:10849000F304353F17ED017ADE44D2ED007A94ED16
:1084A000005AF145D5ED006A37EE274AD0ED004A73
:1084B00077EE677A1CED016A96ED007A91ED001A6D
:1084C00076EE055A36EE872A97ED00DA71EE24EA49
:1084D00076EE453A74EE252A31EE641A35EE466A98
:1084E0003EEE825A74EE655A31EE664A72EE854A65
:1084F00031EE471AB0EE67CA47ED014A34EE077A0B
:10850000D1ED014A31EE261AD0ED016A72EEC52A8C
:1085100095ED014AA7EE6BCA74EEE60A96ED010AE4
:10852000E7EE2B7A92ED017A94ED015A74EEA64AA9
:108530003DEE473ADCED006A70EEC4CA70EEC00A48
:10854000B0EE43EA7CEE80CA74EE001A70EE840A44
:10855000ACEEEBEA36EEC54A3DEE077AB0EE63DAF2
:1085600036EE850AACEEAB3AF0EE4EDAA1EE2BDA3F
:10857000A1EE2B6AE1EE6BDA75EE666AB0EE441A94
:10858000F0EE4CCA37EE405AA0EEAB1AE0EEEBCA62
:10859000E0EEAB6A37EE007A74EEA10A35EEE1FA4E
:1085A00075EEE45A75EE6EFA37EE600A71EEA55A72
:1085B000DDED061A35EE425A7FEE244A3FEE822A5E
:1085C00022EEE1FA61EE80FADDED051A3EEE855A03
:1085D0003EEE066A73EEAD3A21EE82EA73EE4DDAB4
:1085E0003DEE033A24EEE1DADDED071A34EE2C4AD3
:1085F0007CEE266A61EE85CA25EEE1CADDED041A3D
:1086000077EE81EA77EEC17AE9EEA2FADDED032A90
:10861000A9EE80FA9DED030AAAEEA4EADDED014A77
:10862000AAEE82DA9DED012AE8EEA5CADDED025A36
:10863000A8EE85CA9DED025A21EEAD1A62EE832A9C
:108640006EEEE11A27EEC00A64EEA34A26EEC22AB5
:1086500065EE865A24EE455AABEE2E1AEBEE2D1A35
:10866000E8EE272AA8EE030AEAEE264AAAEE232A13
:10867000E9EE045AA9EE065A37EE207A87ED007A21
:108680001F44C2ED00FA82ED01FA1A440CED01EA32
:108690008CED00DA9C44C4ED00CA84ED01CA1C4490
:1086A00081ED001AC1ED011A1944C6ED002A86EDCC
:1086B000010A1E44C0ED005A80ED015A1844C5ED70
:1086C000004A85ED012A1D443FF6E4AE1099089A50
:1086D0000831013210910F99089208310F910E99CB
:1086E00008310E910D9908310D910C9908310C91BA
:1086F0000B9908310B910A9908310A9109990831AF
:108700000991139991427FF468AE149B8A46DB006D
:108710009BB214932EE519B0BDEC108BBDE8F08F21
:10872000124B30B41D686B6A28B943EA014300203C
:10873000AB6230BC7047AC6A013803EB14440BD019
:10874000002303F14002013305EB8202DBB25268E1
:10875000834204EB1244F4D3403044EA014405EB75
:1087600080004460002030BC704700BFF819012031
:10877000037870B42BB30246C0F10105531912F807
:10878000014FDBB2002CF9D101335B000E4C032208
:108790000B8084F8043484F80524017879B102232D
:1087A00000265A1CE518023354FA82F285F80414A4
:1087B000DBB282F8046410F8011F0029F1D170BC0B
:1087C00070470223E2E700BFF819012030B5EFF34C
:1087D0001181802383F312880A4AD2F80435D2F833
:1087E0000845D2F80405D2F80855CAB282F31188B8
:1087F000013BA84294BF4FF4006000201B1B1844AB
:1088000030BD00BFF8190120012380F851307047B6
:10881000014BD3F80C057047F8190120012070476F
:10882000024BC3F81025C3F814157047F81901203E
:10883000024BC3F81825C3F81C157047F81901201E
:1088400070477047212870B505D0222829D02028EC
:1088500010D0002070BD0029FBD0072AF9D1184B99
:1088600018791C685A799B79087100200C604A714C
:108870008B7170BD0029ECD0072AEAD11148104B4A
:108880000C680E794D79D0F8142589791C601E7119
:108890005D719971002ADCD02146D0F8100590470F
:1088A000D7E70029D5D0022AD3D1064AD2F81C3501
:1088B000002BCED00988D2F818059847C9E700BF29
:1088C00000000120F81901200020704703460A2209
:1088D00001481A80704700BF080001200346642247
:1088E00001481A80704700BF14000120012901D0FF
:1088F00000207047014BD3F890301847000001204A
:10890000012900D05EE1024BD3F88C30184700BF3C
:1089100000000120014BD3F88830184700000120E7
:1089200010B40B780A46044603F00303012B05D06C
:10893000022B0BD000205DF8044B70478B8843B9A5
:10894000204611465DF8044B00F014BD8B88832B44
:10895000F6D0034B5DF8044BD3F88030184700BFC6
:108960000000012038B5054B04460D46DB6F9847E3
:108970002946204601F066F8002038BD000001209D
:1089800038B5054B04460D469B6F9847294620464F
:1089900001F090F8002038BD0000012011F0800F98
:1089A00001F00F01F0B4D0F8A8424FF01C0042D102
:1089B000C1EBC10500FB0140002604EB850500F575
:1089C000FE7085F8FD61457801708360C27005B165
:1089D000C180022A01D10023037194F8BC33012B1A
:1089E0001AD00122236884F8BC234178057891428B
:1089F0002CD003F5006605F00F0103F530638A40C3
:108A0000F16903EB451341EA0242F2611A6812046C
:108A100005D5002384F8BC330020F0BC7047826881
:108A20001D68C2F30A02C07818492A4342EA80420C
:108A300011431960EDE7C1EBC105012600FB0140C0
:108A400004EB85053C3085F83D60BCE705F00F067A
:108A5000D3F81CC803F5106203F50067B14002EBC0
:108A6000451241EA0C01F96113681904D1D48368F5
:108A70001668C3F30A03C0780449334343EA8043CA
:108A800043EA855319431160C3E700BF008000101B
:108A9000F0B4002452004E1C2746030FB0F1204FC3
:108AA0004FEA001003F1300503F1370334BF0D55D1
:108AB0000B5537550234A242EFD1F0BC704700BFCE
:108AC000024808B5FFF754FE014808BD407006088B
:108AD000FC1D0120024808B5FFF74AFE014808BD09
:108AE00050700608FC1D01200B481A220B4B006831
:108AF0001B680A80C01801D109487047094B082239
:108B0000094910B51C68FFF7C3FF04220749204636
:108B1000FFF7BEFF024810BD107AF01F187AF01F51
:108B2000B0000120147AF01FB2000120C200012021
:108B3000024808B5FFF71CFE014808BD5C70060836
:108B4000FC1D012008B520B90448FFF711FE0448B8
:108B500008BD0448FFF70CFE014808BD6870060810
:108B6000FC1D01208C700608042301480B8070470F
:108B7000CC00012003460A2201481A80704700BF3A
:108B8000D00001200346202201481A80704700BF10
:108B9000DC0001200346202201481A80704700BFF4
:108BA000FC0001200346202201481A80704700BFC4
:108BB0001C01012003460A2201481A80704700BFA9
:108BC0003C0101200023D0F8982218461373704707
:108BD0000346222201481A80704700BF4801012045
:108BE0000346222201481A80704700BF6C01012011
:108BF0000346222201481A80704700BF90010120DD
:108C000003460A2201481A80704700BFB4010120C0
:108C10000346432201481A80704700BFC00101206B
:108C20000346432201481A80704700BF0402012016
:108C30000346432201481A80704700BF48020120C2
:108C4000D0F8943283B110B5D0F8904294F8000275
:108C5000FF2807D09B68214694F801229847FF23FC
:108C600084F80032002010BD0020704701F00F0191
:108C7000D0F8A822C1EBC10102EB810238B5D0F8CF
:108C80009032D0F89452D2F8144203F50371EA6896
:108C9000D3F80402C3F80C429047002038BD00BF4F
:108CA00008B5D0F88C325B689847002008BD00BF3B
:108CB00008B5D0F88C321BB11B68984700B908BDC5
:108CC000022008BD0B4B01E0013B10D00269002AD5
:108CD000FADA0369074A43F00103036101E0013A4C
:108CE00005D0036913F00103F9D11846704703203A
:108CF000704700BF400D0300144B10B4046C9C423D
:108D00001AD800F53060002301290361036943F498
:108D100000230361036943F018030361036943F00F
:108D2000C043036104D14261036843F080230360C0
:108D300000205DF8044B7047D0F8003B00F5306030
:108D4000002BE0DA00205DF8044B70470A30544FE6
:108D500038B5D0F8A84201F00F03626893422BD8CF
:108D60000A062BD41C25C1EBC102002005FB0141E2
:108D700004EB820201F5FE7182F8FD0101220B7005
:108D80008A7094F8BC03904216D084F8BC234A78C9
:108D90002068012A09781DD000F5306202EB4112EB
:108DA0001568002D00DBF1B9116841F40011116064
:108DB0001BB3002384F8BC33002038BD1C21C3EB57
:108DC000C302012001FB034104EB82023C3182F823
:108DD0003D00D3E700F5106202EB4112156800294F
:108DE000E2D0002DE0DB116821F0804111601168B4
:108DF00041F400111160002BDBD104F57172217C6C
:108E0000FFF77AFFD5E700BF10B504468021FFF7D2
:108E10009FFF00212046BDE8104099E72DE9F84367
:108E2000884600294FD04718461E284C802507F158
:108E3000FF39EFF3118185F31288D4F80425C9B204
:108E4000D4F80805D4F80435D4F808C581F311889E
:108E5000634594BF4FF400630023121A1344012B9F
:108E60001AD1012039F06EFFEFF3118185F31288DA
:108E7000D4F80425C9B2D4F80805D4F80435D4F8D8
:108E8000087581F31188BB4294BF4FF4006300233F
:108E9000121A1344012BE4D0EFF3118285F31288E8
:108EA000D4F80835D2B216F8011F234483F82015F0
:108EB000D4F808350133C3F30A03C4F8083582F344
:108EC00011884E45B5D14046BDE8F883F819012018
:108ED000F8B5002390F8505080F85030CDB10F4EC7
:108EE00096F8942F032A16D1D6F8CC7F00F13C04D3
:108EF00029462046FFF792FFD6F8CC3F2D1A0444AE
:108F0000DB1B322B01D8002DF2D1B5FA85F04009D8
:108F1000F8BD0120FCE71846FAE700BFF819012068
:108F2000002280F85120D3E790F85020531C0244CF
:108F3000DBB280F8503082F83C1090F851200AB132
:108F4000132B00D9C4E77047F8B50B4E0D461446F5
:108F500096F8943F032B0ED1D6F8CC7F002C0ADD77
:108F600021462846FFF75AFFD6F8CC3F241A05447D
:108F7000DB1B322BF2D9F8BDF819012010B5032004
:108F80000C464DF0F7FB03280AD0074B93F8D03F6F
:108F9000012B4FF012030CBF04480548238010BD7D
:108FA00012230448238010BDF8190120B4020120C7
:108FB000A00201208C0201202DE9F04FDFF8188378
:108FC000B94D44462DED068B89B0CDE906010592D9
:108FD0000FCD0FC40FCD0FC4B44B95E8070093F825
:108FE000D63F84E80700042B00F20C81DFE813F081
:108FF00036010A010501050044019FEDAD8A9FED90
:10900000AD9AAD4AAD4B0598AD49002818BF13463F
:10901000AC4AC8E9062139EE087ADFEDAB7AF5EE05
:10902000006AAA4A28EE278AA94FB0EE67AA02F181
:10903000150BC6EE879A0026DFEDA68A0292C8F8C5
:109040002430079BB34200F0D280029A731C12F8BE
:10905000014B0393DBB20292002C00F01B81002233
:1090600003E00132152A00F0158102EB42015500A0
:109070001BF80100A042F4D104938C4B194491F8E1
:10908000F11F002900F00E81204639F0B5F9824623
:1090900000684CF05FF99AF8051039F0EBF90178A7
:1090A000002940F0F78020090322DFF8409204F005
:1090B0000F0C441E049B4D44944205F8C73C05F830
:1090C000C82C00F2C580784901EB4401888D40FA34
:1090D0000CF111F0010100F0BB8001210493A9F112
:1090E0009C0501FA0CF10139084051F0A5FB6E4BCB
:1090F000032202211C44049B94F83440204405EBD5
:10910000C00078618271C3719AF808203DF0C2FFF7
:10911000059B002B7BD0654B6449B3F8D43F91F895
:10912000D61F07EE903AD9F864310429F8EEE77AB1
:10913000FCEEE77A17EE900AB3FBF0F202F57F42FD
:1091400002F1FF024FEA1242B3FBF2F2B2FBF0F07F
:1091500083B272D007EE902AF8EE676A66EE887ADC
:1091600028EEE77A5149C7ED027A91F8D70FA9EEB8
:10917000267A0699019038460091514687ED037A88
:1091800031F062FB002E65DD7B68D8F83820934211
:1091900062D0012E5ED0D8F8502093425CD0022ECF
:1091A00058D0D8F86820934256D0032E52D0D8F821
:1091B0008020934250D0042E4CD0D8F8982093426F
:1091C0004AD0052E46D0D8F8B020934244D0062E7F
:1091D00040D0D8F8C820D31A18BF0123039E01221B
:1091E0003B741837082E07F8072C7FF42AAF3A484B
:1091F00009B0BDEC068BBDE8F08F9FED388AB0EE6C
:10920000489AFEE69FED368AB0EE489AF9E6FAFEF5
:10921000697AFCEEE77AD9F864114FF6FF7317EE1E
:10922000902A1846B1FBF2F21A44120CB1FBF2F28A
:109230001E4991F8D61F04298CD107EE900A07EE3B
:10924000102AF8EE677AF8EE476A67EE8A7A87E7BF
:1092500079615DE70123C1E70023BFE70023184AD6
:1092600001219FED198A0693164BB0EE489A05919D
:10927000C8E90632104BCEE60023114A01219FEDCA
:10928000198A06930F4BB0EE489A0591C8E9063249
:10929000094BC0E6144A0020074BC8F81C20C8F848
:1092A0002430A5E70B68FFDEF8E20508F819012075
:1092B000ACC5A737ACC5A736750A0408059A0308DC
:1092C0004D9F0308810A04086F12833AD3290120B5
:1092D0004800002000007A4414000020282930387B
:1092E0006F12033900000000F19C0308F02A0120EE
:1092F00070B5D0F89062E6B101EB810500EB850511
:10930000EB695BB1D0F8A802C1EBC10400EB8404A7
:10931000626CB3FBF2F402FB14341CB10020C6F8FB
:10932000140270BD23462246EC610BF081FA204600
:1093300070BD022070BD00BF002310B504241A4682
:109340001946C0F86C42D0F8A8020BF071FA002060
:1093500010BD00BF10B5134602240A460021C0F814
:109360006C42C0E90733D0F8A8020BF061FA002084
:1093700010BD00BF10B50C7882B00023D0F8982241
:1093800014F06004ADF8063016D0202C0ED14B78C6
:10939000023B092B0AD8DFE803F033390909090930
:1093A00009093F2F90F87432032B5AD00224FFF79B
:1093B0002BFD204602B010BD4B780B2BF6D80FF2D8
:1093C000080C5CF823F000BF4D940008AD93000832
:1093D000AD930008AD930008AD930008AD9300086D
:1093E00023940008AD930008AD930008AD930008E6
:1093F000A59300083F9400088B7800241360D8E7F9
:10940000111D01220024FFF7A5FFD2E7114601221A
:109410000024FFF79FFFCCE74B8800241B0A536012
:10942000C7E74B881B0A222B1FD0212BBED1CA882D
:109430001149092A28BF0922FFF78CFFB9E790F8E4
:109440007432032BB2D18B789360B2E790F8742218
:10945000032AABD102220DF106011C46FFF77AFF69
:10946000A7E702F108010122E6E7CA880349362A84
:1094700028BF3622E0E700BF00030120C802012018
:109480002DE9F0430D784FF0010883B0044680F8D1
:10949000805205F01F0C4F7800F5207EC44580F8FF
:1094A0008172CB788E7806EB0326B6B2A0F8826282
:1094B0004A790B7903EB02239BB2A0F8843291F82E
:1094C00007908A79C0F86C8202EB092292B2A0F868
:1094D0008622C0F870220DD0BCF1020F3ED0BCF144
:1094E000000F19D005F08001FFF732FC002003B017
:1094F000BDE8F08305F06002402A67D06A0665D5B2
:1095000080212046FFF724FC20460021FFF720FCA5
:10951000002003B0BDE8F08305F06005202D6FD07A
:10952000402D6DD0002DEBD1092FE9D801A151F8C4
:1095300027F000BF4B9600087996000801950008B7
:109540009796000801950008A7960008079700085D
:1095500001950008359700081596000805F060058C
:10956000202D4DD0402D4BD0002DC9D1012FD9B287
:1095700000F00481032F00F0EF80002FC0D190F89D
:109580007422022A00F0CC81032AB9D113F0800F93
:1095900001F00F0303EB830300EB830340F0D8815A
:1095A000D3F84431002BABD001F07F03142202FB2F
:1095B000030202F5A072002B40F00D82002313601D
:1095C000114620460222FFF7C5FE8FE794F8742269
:1095D000013A022A94D8DBB2032B91D8D4F88C320A
:1095E000714620469B689847B4F88632002B7FF47A
:1095F0007DAF00287FF47AAF2046FFF79DFE75E728
:10960000D4F88C32714620469B689847002003B0FE
:10961000BDE8F083F6B2C14D012E85F868613FF6D2
:109620006FAF90F87432022B00F0BE81032B00F074
:10963000A9818021FFF78CFB00212046FFF788FBE2
:1096400031462046FFF72CFB50E790F87432013B7F
:10965000022B3FF655AF022A7FF452AF0122D0F819
:109660007C32C2600BB10323C360022204F10C01FF
:109670002046FFF76FFE39E790F87432013B022B6A
:109680003FF63EAF012E7FF431AF0023C0F87C32AD
:10969000FFF752FE2AE7012E7FF428AFC0F87C6264
:1096A000FFF74AFE22E713437FF42AAF7F2E3FF6EF
:1096B00027AF90F87432032B3FF422AFF1B2D0F809
:1096C000A83280F8761293F8BC23012A11D01A68C8
:1096D000002083F83810D2F8001821F4FE61C2F897
:1096E0000018D2F8001841EA0611C2F8001883F8F1
:1096F000BC032046FFF720FE002E00F07E810223EF
:1097000084F87432F2E6330A013B062B3FF6F8AEDA
:1097100001A252F823F000BF999800087F98000832
:109720006D980008019500080195000857980008F9
:1097300011980008012A7FF4E3AE90F87432022BEE
:1097400000F2FF80002B3FF4DBAE0023014641F81E
:10975000083FFFF7FFFDC9E690F87432022B00F0D6
:10976000D380032B7FF4CCAE4F063FF445AF56EACF
:1097700002037FF441AFFFF7EBFA3DE790F8742264
:10978000022A00F0C180032A7FF4BAAE002E7FF4D3
:10979000ADAE48063FF430AFD4F8A80201F00F0197
:1097A000426891423FF628AF13F0800F4FF01C0340
:1097B00040F0278103FB01020025134602F5FE72EB
:1097C00083F8FD5100231170937090F8BC33012B86
:1097D0003FF412AF0121036880F8BC13557811786B
:1097E000012D0CBF03F5106303F5306303EB411348
:1097F000196821F400111960D278023A012A03D8BD
:109800001A6842F080521A60002380F8BC33F3E6F5
:10981000037C002B7FF474AED0F88C320DF106007F
:109820001B6B984707234370BDF806306BB1B4F843
:109830008622002A3FF4E0AE9A420146204628BF25
:109840001A46ADF80620FFF785FDB4F88632002BE6
:109850007FF44CAED0E6037C002B7FF451AED0F801
:109860008C320DF106005B6B9847DDE7F6B2052EF2
:109870003FF646AEDFE806F0302820184038037C7B
:10988000002B40F09F80D0F88C320DF106009B6ACF
:10989000984702234370C7E7D0F888320DF10601DC
:1098A000007C1B689847BFE7D0F888320DF10601AD
:1098B000007C1B699847B7E7D0F888320DF10601A4
:1098C000007CDB689847AFE7D0F888320DF10601DD
:1098D000007C9B689847A7E7D0F888320DF1060115
:1098E000007C5B6898479FE7D0F888320DF106014D
:1098F000007C9B69984797E7D0F888320DF1060104
:10990000007C5B6998478FE74D063FF4F9ADFFF7A0
:109910001FFA20468021FFF71BFAE7E5F02A012015
:109920004A067FF4EDAD1B064FF000034FF0020234
:109930004CBF00F1140100F5A0710B60FFF70AFDA8
:10994000D4E5032B7FF4DCAD011DFFF703FDCDE56E
:109950009B69002B3FF4D4AD01F07F035A1C02EB4E
:10996000820200EB8202002B3FF428AED0F8A8124E
:109970001C2000FB031393F83E30002B3BD0012347
:1099800013601DE67EB3416801293FF435AEC9B2CC
:10999000FFF786F995F8681120466160FFF788F9AE
:1099A00002287FF429AEABE5002E3FF425AE01215D
:1099B0000323416080F87432FFF77AF902287FF4BC
:1099C0001BAE9DE5D0F88C320DF10600DB6A98479E
:1099D0000223437028E7D0F8A8321C2000FB013393
:1099E00093F8FE31C9E702233146466080F87432AD
:1099F000FFF756F900E61360E2E5012384F87432BC
:109A000074E503FB0102012513463C3283F83D5007
:109A1000D8E600BF38B5044600250121D0F8A802D9
:109A20000AF02AFF8121D4F8A802C4F858510AF09C
:109A300023FFD4F8A002E56254F0F6FA2846C4F8F1
:109A4000A05238BD38B504468321D0F8A8020025BD
:109A50000AF012FFD4F89802656518B154F0E4FAE0
:109A6000C4F89852002038BD38B50446002581213D
:109A7000D0F8A8020AF000FF0121D4F8A802E5629C
:109A80000AF0FAFED4F8A8028221C4F858510AF06C
:109A9000F3FED4F8903225644BB1D4F894325B686D
:109AA0009847D4F8900254F0BFFAC4F890520020BE
:109AB00038BD00BF10B50823032283210446FEF7FA
:109AC0006DFF01231020636554F0A6FAC4F89802D4
:109AD00018B103460020187310BD022010BD00BF4E
:109AE000154BDB68C3F3022310B4C3F107041A1D3E
:109AF000042C28BF0424062A4FF0FF328CBF033BFE
:109B00000023A240002821EA020101FA03F108DB48
:109B100009010A4BC9B2034483F800135DF8044BF2
:109B2000704700F00F000901054BC9B203441976D4
:109B30005DF8044B704700BF00ED00E000E100E07D
:109B4000FCEC00E030B5264C0022264841F287317B
:109B5000D4F8643183B0244DA0FB030304F5B67040
:109B6000C4F86C51DB0C013BC4E95E12C4E95C3201
:109B70000AF02AF91D4B062137201A6C42F0200208
:109B80001A641B6C03F020030193019BFFF7A8FFED
:109B9000D4F86C314FF400001549164A4860D96872
:109BA00041F00101D96099680A40062A06D0B2F551
:109BB000803F03D01A6842F001021A600E4B002069
:109BC0000E49D3F8B02F03F5A464C3F81C05C2F8FE
:109BD0001002C3F81405C2E9811403B030BD00BF00
:109BE000F02A012083DE1B430014004000380240AD
:109BF00000E100E007000100F81901209C2C012081
:109C000038B50F4B0F4AD3F86431A2FB03239B09ED
:109C1000013BB3F1807F10D20B4A0024F0200B49A6
:109C20000725536081F82300214694604FF0FF30F0
:109C30001560FFF755FF204638BD012038BD00BF35
:109C4000F02A0120D34D621010E000E000ED00E0AA
:109C50004309012200F01F0084B0013B02FA00F02A
:109C6000032B0BD8DFE803F015021E0C124B5A6CC5
:109C700002435A645A6C10400090009B04B0704735
:109C80000D4B1A6B02431A631A6B10400390039B2F
:109C9000F4E7094B5A6B02435A635A6B1040029027
:109CA000029BEBE7044B1A6C02431A641A6C1040D7
:109CB0000190019BE2E700BF0038024018B100228A
:109CC00001213DF0E7B9704718B1002220213DF095
:109CD000E1B9704700487047B42A012058B1838821
:109CE0004FF00042B3FA83F332FA03F303D0024990
:109CF0000A6813430B607047003C0140F0B589B01F
:109D000004463EF0EBF9031E1CDB164E0022164DF6
:109D1000F118B4F804C005EB830305F6EC1091F8D4
:109D2000387003A9C3F8AC093D44104B2068079272
:109D3000CDE903C3CDE905220AF0EAFE95F8F03932
:109D4000802B01D809B0F0BD3E448023022196F952
:109D5000480085F8F0390190FFF7C2FE01980BF03A
:109D600051FEEFE7F8E20508F02A0120000031106B
:109D7000002800F08F80B0F804C0BCFA8CF3202BD0
:109D8000C3F11F0200F086806F4B2DE9F04F9D1844
:109D9000DFF8E48185B0036808EB820095F838208D
:109DA0000024DFF8D8E10192C0F8AC19674A02E05C
:109DB0000134102C65D04FF0010909FA04F10CEAC6
:109DC000010531EA0C01F3D14FF0030A04FA09F757
:109DD00018684FF00F0B0AFA07F704EA0A0124F09B
:109DE000030620EA0700890006F1804618600BFA96
:109DF00001F0D3F80CB006F59C362BEA0707DF60BC
:109E0000DEF8447047F48047CEF84470DEF84470C2
:109E100007F480470397039FB76827EA00004C4F79
:109E2000BB421AD007F58067BB4234D0494FBB42D2
:109E300035D0494FBB426BD0484FBB4271D0484FE1
:109E4000BB4269D0474FBB4278D0474FBB420CBFA3
:109E50000727082707FA01F10843B06001341168A9
:109E6000102C41EA05011160516821EA0501516099
:109E7000916841EA05019160D16821EA0505D56044
:109E800099D1019B984498F8F039F02B0CD805B083
:109E9000BDE8F08F704709FA01F10843DDE70227BA
:109EA00007FA01F10843D8E7F021304B264888F83B
:109EB000F019D968019AC1F302210244C1F10700E7
:109EC0000B1D92F84840042892F9482028BF04202E
:109ED000062B4FF0FF338CBF033900218340002A4B
:109EE0006FEA030303F0030303FA01F31EDB2048C8
:109EF00001211B0104F01F0485185209DBB201FA8D
:109F000004F485F8003340F8224005B0BDE8F08F36
:109F10000AFA01F10843A0E7052707FA01F108430F
:109F20009BE7042707FA01F1084396E704F00F04C2
:109F30001B01104ADBB222441376A8E7062707FA72
:109F400001F1084389E700BFF8E20508003C014041
:109F50000000024000080240000C024000100240D5
:109F60000014024000180240001C024000ED00E016
:109F700000E100E0FCEC00E0F02A012000380240A3
:109F80002DE9F041D0F800E00C46DFF8588084B0AD
:109F9000DEF804501746DFF850C0194605EA0805F8
:109FA000DDF82880064603932C43424644EA0C0C15
:109FB000CEF804C00AF006FD78B931680246039B6A
:109FC00030468F624021CDF800800AF02BFD00382A
:109FD00018BF012004B0BDE8F081012004B0BDE845
:109FE000F08100BF009800FC00200180F8B5134FFD
:109FF00004460D460AE09B69DB0602D50AF0A2FC86
:10A00000D0B9D7F8F8395B1B0A2B08D823682A4641
:10A010000A2120469E69B606EDD50020F8BD636C86
:10A020002021002201200B4384F84020636484F83F
:10A03000411084F84220F8BD0120F8BDF02A01202B
:10A040002DE9F84FCB4C054694F8FC19D4F8040AD6
:10A05000C1F340013DF050FA94F8FC19D4F8000A1D
:10A06000C94301F001013DF047FA002D00F0E780FF
:10A0700005F1FF39C04E4FF01008C04F5FFA89F963
:10A08000BF4DD4F8043A33B11A689B8851690B422A
:10A0900018BF1B049361D4F8003A33B11A689B8847
:10A0A00051690B4218BF1B049361B4F80C3A002BA2
:10A0B00040F0578194F80E1AD4F8100A3DF01CFABB
:10A0C000FA204FF47A714FF0010C7B68C3F3080358
:10A0D000002B40F01981EFF31183002B40F0148125
:10A0E000D6F8CC2FD5F808E0D6F8CC3F9A42F7D175
:10A0F000D4F8343A9E45F3D8D4F830AA01FB0AF3D9
:10A10000A3EB0E03B3FBFAF301FB02327B68C3F34C
:10A110000803002B40F0B680EFF31183002B40F0D2
:10A12000B180D6F8CC3FD5F808B0D6F8CCEF73455F
:10A13000F7D1D4F834EAF345F3D8D4F830AA01FBC8
:10A140000AFEAEEB0B0EBEFBFAFE01FB03E39B1A0D
:10A15000B3F57A7FDAD30138B7D1D4F8043A33B102
:10A160001A689B8851690B4218BF1B049361D4F88D
:10A17000003A33B11A689B8851690B4218BF1B041F
:10A180009361B4F80C3A002B40F0DF8094F80E1A7B
:10A19000D4F8100A81F001013DF0AEF9FA204FF435
:10A1A0007A714FF0010C7B68C3F30803002B40F079
:10A1B0008A80EFF31183002B40F08580D6F8CC2FF6
:10A1C000D5F808E0D6F8CC3F9A42F7D1D4F8343A23
:10A1D0009E45F3D8D4F830AA01FB0AF3A3EB0E0393
:10A1E000B3FBFAF301FB02327B68C3F3080343BB02
:10A1F000EFF311832BBBD6F8CC3FD5F808B0D6F8D7
:10A20000CCEF7345F7D1D4F834EAF345F3D8D4F85A
:10A2100030AA01FB0AFEAEEB0B0EBEFBFAFE01FB01
:10A2200003E39B1AB3F57A7FDED30138BBD109F182
:10A23000FF395FFA89F9B9F1FF0F7FF422AFBDE86A
:10A24000F88FEFF3118A88F31288D5F808B02B68DD
:10A25000DB0303D5C4F82CCAD5F808B0D6F8CC3F38
:10A260005FFA8AFAD4F82CEA8AF31188D4F830AA73
:10A27000734401FB0AFEAEEB0B0EBEFBFAFE01FBC4
:10A2800003E3CEE7EFF3118A88F31288D5F808B01C
:10A290002B68DB0303D5C4F82CCAD5F808B0D6F870
:10A2A000CC3F5FFA8AFAD4F82CEA8AF31188D4F802
:10A2B00030AA734401FB0AFEAEEB0B0EBEFBFAFEA6
:10A2C00001FB03E343E7EFF3118E88F31288D5F81F
:10A2D00008A02B68DA0303D5C4F82CCAD5F808A067
:10A2E000D6F8CC3F5FFA8EFED4F82C2A8EF3118874
:10A2F000D4F830EA1A4401FB0EF3A3EB0A03B3FBD4
:10A30000FEF301FB02326FE7EFF3118E88F3128840
:10A31000D5F808A02B68DA0303D5C4F82CCAD5F801
:10A3200008A0D6F8CC3F5FFA8EFED4F82C2A8EF324
:10A330001188D4F830EA1A4401FB0EF3A3EB0A03A8
:10A34000B3FBFEF301FB0232E0E6D4F8283A002B1F
:10A350003FF424AF0023D4F8142A136084F8253A7C
:10A360001CE7D4F8283A002B3FF4AAAE38F0B4FD2D
:10A37000A6E600BFF02A0120F819012000ED00E058
:10A3800010E000E02DE9F04FCA4C83B00523CA4E1F
:10A3900094F8FC194FF01009D4F8040AC1F34001F5
:10A3A00001933DF0A9F894F8FC19D4F8000AC943C8
:10A3B000DFF80C83C14D01F001013DF09DF8D4F8A8
:10A3C000043A33B11A689B8851690B4218BF1B04C9
:10A3D0009361D4F8003A33B11A689B8851690B42F3
:10A3E00018BF1B049361B4F80C3A002B40F059815C
:10A3F00094F80E1AD4F8100A3DF07EF832204FF48B
:10A400007A710127D8F80430C3F30803002B40F019
:10A410001B81EFF31183002B40F01681D6F8CC2F6F
:10A42000D5F808E0D6F8CC3F9A42F7D1D4F8343AC0
:10A430009E45F3D8D4F830AA01FB0AF3A3EB0E0330
:10A44000B3FBFAF301FB0232D8F80430C3F308037C
:10A45000002B40F0B780EFF31183002B40F0B28067
:10A46000D6F8CC3FD5F808B0D6F8CCEF7345F7D185
:10A47000D4F834EAF345F3D8D4F830AA01FB0AFE45
:10A48000AEEB0B0EBEFBFAFE01FB03E39B1AB3F52A
:10A490007A7FD9D30138B5D1D4F8043A33B11A68E8
:10A4A0009B8851690B4218BF1B049361D4F8003A92
:10A4B00033B11A689B8851690B4218BF1B04936122
:10A4C000B4F80C3A002B40F0E08094F80E1AD4F85F
:10A4D000100A81F001013DF00FF832204FF47A713B
:10A4E0000127D8F80430C3F30803002B40F08B8019
:10A4F000EFF31183002B40F08680D6F8CC2FD5F8EF
:10A5000008E0D6F8CC3F9A42F7D1D4F8343A9E45C9
:10A51000F3D8D4F830AA01FB0AF3A3EB0E03B3FB84
:10A52000FAF301FB0232D8F80430C3F3080343BB4B
:10A53000EFF311832BBBD6F8CC3FD5F808B0D6F893
:10A54000CCEF7345F7D1D4F834EAF345F3D8D4F817
:10A5500030AA01FB0AFEAEEB0B0EBEFBFAFE01FBBE
:10A5600003E39B1AB3F57A7FDDD30138B9D1019BA0
:10A570005F1E17F0FF0301937FF421AF03B0BDE826
:10A58000F08FEFF3118A89F31288D5F808B02B68A1
:10A59000DB0303D5C4F82C7AD5F808B0D6F8CC3F45
:10A5A0005FFA8AFAD4F82CEA8AF31188D4F830AA30
:10A5B000734401FB0AFEAEEB0B0EBEFBFAFE01FB81
:10A5C00003E3CEE7EFF3118A89F31288D5F808B0D8
:10A5D0002B68DB0303D5C4F82C7AD5F808B0D6F87D
:10A5E000CC3F5FFA8AFAD4F82CEA8AF31188D4F8BF
:10A5F00030AA734401FB0AFEAEEB0B0EBEFBFAFE63
:10A6000001FB03E342E7EFF3118E89F31288D5F8DB
:10A6100008A02B68DA0303D5C4F82C7AD5F808A073
:10A62000D6F8CC3F5FFA8EFED4F82C2A8EF3118830
:10A63000D4F830EA1A4401FB0EF3A3EB0A03B3FB90
:10A64000FEF301FB02326EE7EFF3118E89F31288FD
:10A65000D5F808A02B68DA0303D5C4F82C7AD5F80E
:10A6600008A0D6F8CC3F5FFA8EFED4F82C2A8EF3E1
:10A670001188D4F830EA1A4401FB0EF3A3EB0A0365
:10A68000B3FBFEF301FB0232DEE6D4F8283A002BDE
:10A690003FF423AF0023D4F8142A136084F8253A3A
:10A6A0001BE7D4F8283A002B3FF4A8AE38F014FC8E
:10A6B000A4E600BFF02A0120F819012010E000E014
:10A6C00000ED00E010B4B8B10D4CD4F8383A102BBE
:10A6D00005D1052100205DF8044B38F0CFB803EB1D
:10A6E0004302224482F83D1A012182F83C0A0B44BD
:10A6F00082F83E1AC4F8383A5DF8044B704700BF40
:10A70000F02A01202DE9F04FD04C002387B004F649
:10A710006C2894F8802AC4F86C3AC8E90133C8E977
:10A7200003331AB194F8813A84F86C3A94F8823A77
:10A730001BB194F8833A84F87B3A94F8863A1BB1BB
:10A7400094F8873A84F8763A94F8843A1BB194F8EE
:10A75000853A84F8713A94F8883A013B4FFA83FAC3
:10A76000DBB2BAF1FF3F029300F01381B022B84987
:10A77000B84D002302FB0A112E4605F12800503186
:10A780001F469B46019353F00DFC039535785146C7
:10A7900028463FF0B5FC8146002840F0FD80013797
:10A7A0000536042FF2D194F8980A039DFFF750FA6A
:10A7B0004FF44032A84E00230121C4F8A02A3046AD
:10A7C000D4F8942AC4F8B8BAC4F8B41AC4F8AC1AC5
:10A7D00084F8CC1AC4F8A43AC4F8C43AC4F8C83A05
:10A7E000C4F8A83A84F8BC3AC4F8C03AC4F8B03AFD
:10A7F000C4F89C2AFDF704FCBAF1000F40F0EB808E
:10A80000019B83F0010919F0FF0F40F0E480A6F1ED
:10A8100008004EF001FF012308F11408EA78002A2D
:10A8200040F032810535A845F8D104EB0A030299BE
:10A83000022093F9902A39F0D1FB0546002800F058
:10A84000A880002740684BF025FB06213A46DFF838
:10A8500024824EF039FABBF1010F4FF400638CBF34
:10A860004FF480613946D5E90102C4F8F41A4FF477
:10A8700000554FF48071C4F8E82AC4F8F83A4FF450
:10A8800000320323C4F8E40A4046C4F8EC7AC4F862
:10A890000C3BC4F8F07AC4F8087BC4F8107BC4F809
:10A8A000147BC4F8FC5AC4F8001BC4F8042B0BF04A
:10A8B00007F894F8D83AC4F8D48A012B0597C4F85D
:10A8C0001C6B66D00123D4F89C5A84F8D83AAB6844
:10A8D000DE0713D4D4F864316049AA68B3FBF1F3FE
:10A8E00042F0010203EB4303AA600593059B2BB1E1
:10A8F000059B013B0593059B002BF9D1AB68D8075D
:10A9000047D5D4F8DC2A564B134043F48073C4F87F
:10A91000DC3A6B68590507D5D4F8DC3A23F4405388
:10A9200043F48053C4F8DC3AD4F8DC3A13F480538F
:10A9300040F03C81C4F8E03A4A4800234A496FF0AD
:10A940002202C4F8240B494884F8D83A5B46C4F87C
:10A95000201B05F14C01C4F8300B2A606E68444A94
:10A9600046F0806643486E60AE6846F48076AE601E
:10A970000AF01EFF404B5A68D20640F02481D4F8FA
:10A980009C3A9A6812F0405F03D19A6842F0804284
:10A990009A6007B0BDE8F08F28463CF051FCFB1DE3
:10A9A00003210022DBB2CDF8049008B18371C2719B
:10A9B0003CF02CFC30783FF0D5FB0BF1010386F81E
:10A9C00002B05FFA83FB4FF00703707033714FF0F2
:10A9D0000103F370E3E6B02200212848482753F032
:10A9E00053FBB0220021254853F04EFB244B384640
:10A9F00084F8487BC4F8443BFFF72AF94FF4403011
:10AA000000230121D4F8442BC4F8500B1D48C4F88E
:10AA1000641BC4F85C1B84F87C1BC4F8543BC4F86A
:10AA2000743BC4F8783BC4F8583BC4F8683B84F8DE
:10AA30006C3BC4F8703BC4F8603BC4F84C2BFDF78A
:10AA4000DFFA0E484EF0E8FDE5E600BFF02A0120EF
:10AA5000F8E205085C3501208C35012040420F00EA
:10AA6000FEF8FFFFA91A0108AD1A0108991A01089A
:10AA700008010020D4350120002301403436012094
:10AA8000002001403C36012094F8D80A00215A1CCD
:10AA90002F7901280491D2B269783DD04FF001009E
:10AAA000092984F8D80A4ED94FF0030E6FF01D0023
:10AAB000D4F89CCA4FF007091EFB0100DCF80CE03B
:10AAC00009FA00F907FA00F02EEA0907CCF80C7031
:10AAD000DCF80C703843CCF80C00062B4FF0050066
:10AAE0001CD86FF0040710FB0373D4F89C7A1F2066
:10AAF00000FA03FC786B01FA03F320EA0C00786398
:10AB0000786B03437B63D4F89C3A3E48834230D051
:10AB10004FF0000384F8D83A134683E60C2B32D862
:10AB20006FF0220710FB0373D4F89C0A1F2707FA63
:10AB300003FC076B01FA03F327EA0C070763076BB3
:10AB40003B430363DFE7D4F89C0A01EB41094FF074
:10AB5000070ED0F810C007FA09F70EFA09FE2CEA22
:10AB60000E0CC0F810C0D0F810C047EA0C070761FF
:10AB7000B3E7122921D01129CAD123494B6843F4E4
:10AB800000034B60C4E76FF0400710FB0373D4F879
:10AB90009C0A1F2707FA03FCC76A01FA03F327EA96
:10ABA0000C07C762C76A3B43C362ACE7D4F8E03A1C
:10ABB00023F00603C4F8E03ABEE613494B6843F4B9
:10ABC00080034B60A4E7D4F89C2A0E498A420DD03A
:10ABD0005B68DB063FF5DDAE0C4B9A427FF4D9AEE5
:10ABE0009A6812F0405F7FF4D4AECEE6936813F01B
:10ABF000405F03D1936843F080439360024B5B68EE
:10AC0000C7E600BF002001400023014000220140B0
:10AC10002DE9F041D0F800E00C46DFF8588084B010
:10AC2000DEF804501746DFF850C0194605EA08055B
:10AC3000DDF82880064603932C43424644EA0C0C78
:10AC4000CEF804C009F0BEFE78B931680246039B15
:10AC500030468F628021CDF8008009F0E3FE003895
:10AC600018BF012004B0BDE8F081012004B0BDE8A8
:10AC7000F08100BF009800FC002001810A4610B15D
:10AC800002213CF007BA7047034690F83C000128C7
:10AC900000F03E810220F0B4012483F83D0083F8E7
:10ACA0003C40142A45D8DFE812F04D00440044002F
:10ACB00044007B00440044004400DA0044004400A7
:10ACC0004400AA004400440044000601440044003B
:10ACD000440015001A688E68156A0F6825F48015FF
:10ACE000AB4C1562106A556820F40010D2F854C0BD
:10ACF00040EA0650A74E0CEA0404B24244EA072494
:10AD000000F0088106F58066B24200F003814E68CB
:10AD100055605465D6651062506D0C6940F4006052
:10AD20005065506D20F480605065516D41EA0421FA
:10AD3000516500220121104683F83D1083F83C2024
:10AD4000F0BC70471A68D1F808C0156A0F6825F082
:10AD50000105914C1562106A5668956920F0020051
:10AD60002C408C4D40EA0C00AA4244EA070400F053
:10AD7000DD8005F58065AA4200F0D8804D685660F8
:10AD800094615563106290690C6940F0080090610D
:10AD9000906920F004009061916921439161C8E7B6
:10ADA0001A68D1F808C0156A0F6825F010057B4CA9
:10ADB0001562106A5668956920F020002C40754D88
:10ADC00040EA0C10AA4244EA072400F0C38005F5CB
:10ADD0008065AA4200F0BE804D685660946195631C
:10ADE000106290690C6940F400609061906920F4F1
:10ADF00080609061916941EA0421916199E71A6844
:10AE00008E68156A0F6825F48055644C1562106AC7
:10AE1000556820F40050D2F81CC040EA06305D4E60
:10AE20000CEA0404B24244EA072400F08D8006F5DF
:10AE30008066B24200F088804E685560D461166426
:10AE40001062D0690C6940F40060D061D06920F4D0
:10AE50008060D061D16941EA0421D16169E71A6853
:10AE6000D1F808C0156A0F6825F480754A4C156240
:10AE7000106A5668D56920F400702C40454D40EAB0
:10AE80000C20AA4244EA070473D005F58065AA4263
:10AE90006FD04D685660D461D5631062D0690C697B
:10AEA00040F00800D061D06920F00400D061D16981
:10AEB0002143D1613DE71A688E68156A0F6825F451
:10AEC0008035374C1562106A556820F40030D2F88E
:10AED00054C040EA06402F4E0CEA0404B24244EA51
:10AEE00007041DD006F58066B24219D04E68556041
:10AEF000546596651062506D0C6940F0080050650D
:10AF0000506D20F004005065516D2143516510E7EC
:10AF10000220704725F480254E6945EA8625F6E62D
:10AF200025F480354E6945EA0625DFE726F4407CA6
:10AF300020F008008E69CF684D693843354320F012
:10AF4000040045EA0C0619E725F480454E6945EAF8
:10AF5000861571E726F4406C20F080008E69CF687A
:10AF60004D6940EA0710354320F040004CEA850661
:10AF700032E726F4405C20F400608E69CF684D69AA
:10AF800040EA0720354320F480604CEA051680E74C
:10AF9000FF8FFFFE000001408CFFFEFFFF8CFFFED5
:10AFA0008FFFFEFF064B93F8F42B002AFBD141F2F2
:10AFB000587204499B5801F10D001B68184700BFE7
:10AFC000F02A0120E7360120F0B5D823884E83B05F
:10AFD00003FB0063D3F86426002A00F0C38093F8D3
:10AFE0006E160022044683F872260846FEF730FEED
:10AFF00001F01F02490901230139934003290AD8AE
:10B00000DFE811F0E9000400EF00E30079494A6A43
:10B0100022EA03034B62D823651C03FB0463EDB2F1
:10B0200093F868063CF00CF9074610B11223C5717D
:10B030008371D82303FB046393F869063CF000F99D
:10B0400010B11323C5718371D82303FB046393F8F4
:10B050006A063CF0F5F810B11423C5718371D82548
:10B060002E21384605FB046595F86B263CF0D6F991
:10B0700095F869063CF0E4F895F86C262E213CF032
:10B08000CDF995F86A063CF0DBF895F86D260E21AF
:10B090003CF0C4F9D5F8643657491A688B4222F05F
:10B0A00040021A6060D0554A934200F0848002F555
:10B0B0008062934265D14F4A116A41F400411162A6
:10B0C000116A21F400411162D82000FB046494F855
:10B0D0007226002A52D1012402255A68484942F4B6
:10B0E0008052C1E9C6545A601A68520632D4D1F867
:10B0F00020C3D1F82873D1F82C630197D1F82473B9
:10B10000B6F5005FDFF808E1D1E9C32042EA0002AA
:10B11000186842EA0C0200EA0E0ED1F8140342EA63
:10B120000702019F40EA1C4042EA0702354F42EA0B
:10B13000060242EA0E0242EA040242EA05021A60EC
:10B140005A6807EA020740EA0700586002D1B1F8DE
:10B1500030231A61DA6922F40062DA611A6842F077
:10B1600040021A6003B0F0BD224A516A41F4805196
:10B170005162516A21F480515162A5E700242546AD
:10B18000ABE7214A934209D11A4A516A41F400516E
:10B190005162516A21F40051516295E71B4A934272
:10B1A00092D1144A516A41F480115162516A21F4DA
:10B1B0008011516288E70F4A116A41F4804111629F
:10B1C000116A21F4804111627EE70A490A6922EA84
:10B1D00003030B611FE707494A6922EA03034B6136
:10B1E00019E704490A6A22EA03030B6213E700BF66
:10B1F000E83B0120003802400030014000380040A8
:10B2000000000120FBF0FFFF00340140005001402E
:10B210004000FFFF03680B4A23F0400390420360A5
:10B220000DD0094B98420AD01022036823F038034E
:10B2300013430360036843F0400303607047082230
:10B24000F3E700BF00380040003C00402DE9F0412A
:10B250006B4C00234FF4F0722021064604F6C81010
:10B2600084F8C43952F010FF04F6A8304FF4F0729D
:10B27000202152F009FF94F8890D10B194F88A2D1D
:10B280001AB900252846BDE8F0813BF0D9FF0746F2
:10B29000C4F8980D3CF016F905460028F1D00FB11E
:10B2A0002323FB800D2138463BF0B0FFD4F8980DE6
:10B2B0003CF01CF994F88A0D524F013840B23DF031
:10B2C000BBF902232021C4F8900D84F88C3D49F08D
:10B2D0006FFAB7F834134C483DF01AF9D4F8980DCA
:10B2E0003CF0FEF8FF218C204CF056F98046D4F853
:10B2F000980D3CF0FBF8D4F8900DFFF78BFFB8F1F8
:10B300001B0F05D0D4F8980D0025FEF7DDFCB9E73A
:10B310000122D4F8983D84F8C4290BB12322DA80A5
:10B32000B7F8341338483DF0F3F8D4F8980D3CF0F2
:10B33000D7F840210A204CF02FF9FF218A204CF049
:10B340002BF90346D4F8980DC3F3801384F89C3D81
:10B350003CF0CCF8D4F8900DFFF75CFF94F8883DF2
:10B36000012B43D0022B39D0E3B394F89D3D182B29
:10B3700009D194F89C2DB7F83433A4F8A06DA4F843
:10B38000A22DA4F8A43DB7F834131F483DF0C0F82F
:10B39000B7F834131C483DF0BBF8D4F8980D3CF0D6
:10B3A0009FF8022100204CF0F7F8D4F8980D3CF0FB
:10B3B0009DF8D4F8900DFFF72DFF94F8AD2D94F87B
:10B3C000AE3DC2F1200294F8AC1DC3F1100384F825
:10B3D000AF2D84F8B03D84F8A81D53E71023A7F8DB
:10B3E0003433C2E72023A7F83433BEE7002EF5D06C
:10B3F00094F89C3D002B14BF10232023EFE700BFDF
:10B40000E83B01200000012074490120F8B5474EB7
:10B4100096F8B14D04EB4403650006EBC30393F8C3
:10B42000B43D032B77D8DFE803F0492A1F022544F7
:10B4300006EBC505D5F8B83D002B6ED196F8142E55
:10B44000944268D0013404F003018A4286F8B11DA9
:10B4500061D001EB41040222184606EBC404C4F893
:10B46000B83D84F8B42DF8BD2B1906EBC303D3F80F
:10B47000B82D72B1013A0020C3F8B82DF8BD2B19D0
:10B4800006EBC303D3F8B82D002AF3D1022283F8C8
:10B49000B42D254406EBC50595F8C03D013BDBB254
:10B4A00085F8C03DF3B1224B0120D3F8382302F2D6
:10B4B000E733B3FBF2F3C5F8B83DF8BD3DF00AFD44
:10B4C00048B31B4A42F20F732C440121D2F83823AF
:10B4D00006EBC404134484F8B41DB3FBF2F3C4F8C0
:10B4E000B83DF8BD124B601C0327D5F8BC1DD3F83E
:10B4F0003823384096F8144E531E85F8B47D001B4F
:10B500000B4418BF01209A42B3FBF2F188BF002020
:10B51000C5F8B81D30B90120F8BD013B0020C5F8C1
:10B52000B83DF8BD0139C5F8B81DF8BDE83B0120AC
:10B530000000012003689B0AA3F58013522B00D959
:10B5400070470E4A134470B593F8604284B00D2CD6
:10B5500012D800294FF0000309494FF0010514BF2C
:10B560001E460226427901EB84106946CDE900654A
:10B57000CDE9023308F028FB04B070BDF8E20508FD
:10B58000004A01200378012B01D00020704790F978
:10B590000420084902EB420201EB421292F83511F5
:10B5A000202901D018467047D2F8F4309869C0F3CA
:10B5B000C0307047E04C012070B5174C82B00D468A
:10B5C000134694F86062022E08D00A46014604F53C
:10B5D000187002B0BDE870403DF006B9D4F86C2296
:10B5E0001AB1918816680904B1610146D4F8640261
:10B5F00001934BF023FE019B2A460021D4F86402FC
:10B600004BF0D6FBD4F86C3213B11A689B88936167
:10B61000012002B070BD00BFE04C01202DE9F04FC9
:10B62000037883B00446022B00F08C80012B04D0F9
:10B630000025284603B0BDE8F08F90F90400554E70
:10B64000042886F8A432D4BF00250125B0F1FF3FBD
:10B6500008BF45F00105002DEAD100EB40024FEA9A
:10B66000400C06EB4212D2F8F470002FE0D092F8B2
:10B6700035E1BEF1200FDBD1BF6917F40047D7D108
:10B6800092F834E1BEF1010FD2D04FF04008DFF85C
:10B6900018E1DFF818B14FF0210A94F80590DBF8B3
:10B6A000F84982F835A182F8368106F52978C2F882
:10B6B0003871A2F81E31C2F820E1B2F81EE182F81A
:10B6C00034311FFA8EF3DFF8E8E0C2F81881FF2B5F
:10B6D000C2F828E159D8B2F81EE14FF000781FFAFD
:10B6E0008EFE84442C4800944FEA490900EB4C102C
:10B6F0000A4606EB4C14494614301923A4F81CE101
:10B70000FFF786FA002836D1D4F8F420234953688D
:10B7100094F81C610B40224DD4F8281143EA090328
:10B72000A94243EA064343EA0803536084F834011C
:10B7300003D01C4B994218BFF227136801251F4301
:10B74000176076E7C3681BB19A8818681204826193
:10B7500060684BF073FD012160684BF06FFDE3689A
:10B760003BB101251A689B882846936103B0BDE868
:10B77000F08F01255DE7B6F8A6320022013384F888
:10B7800034219BB2A6F8A63253E74FF0FF0E4FF0DC
:10B790008078A6E7E04C0120C04D0120009C00FC11
:10B7A000DD530108E55401080000FFFFF02A0120E5
:10B7B000295601080848002302461178063202295A
:10B7C00004D00133062BF8D10020704703EB43036C
:10B7D00000EB4300704700BF884F0120F0B59C4C40
:10B7E00085B02422002104F52A7052F04DFC94F813
:10B7F000CD62002E3AD13546D4F8E4325BB39B6A71
:10B800004BB39448984783682BB303880021DFF833
:10B810006CC2013B604666469BB237780636032F02
:10B820001CD001310629F8D1002201780630022906
:10B8300000F0A4800132062AF7D1D4F80C130529B0
:10B8400009D002FB01C20131C4F80C13022000210F
:10B85000938010705180284605B0F0BD062303FB8D
:10B860000141B1F8AA32013B9BB2DDE704F5357323
:10B8700094F8CC02C4F8D03208B90025BCE73BF0FC
:10B88000DFFC0746C4F8E0023BF01CFE054600283A
:10B89000F3D0013E022370B284F8D4323CF0CCFEE7
:10B8A0000028EAD0C4F8D8020FB12023FB800D2174
:10B8B00038463BF0ABFCD4F8D0320126D8683BF0D8
:10B8C00015FED4F8D0322021586848F071FF624B41
:10B8D000D4F8D02284F808630026C4F8042393E83F
:10B8E0000300009032208DF8041037F02BFA052366
:10B8F00002AA6946D4F8D0028DF80A608DF8096072
:10B900003CF088FE9DF80A209DF8090012029DF87F
:10B910000B10524B42EA00420A439A4200F09080D8
:10B9200030DCA3F5F1139A425DD041DD4C4B9A42D5
:10B9300051D002339A4261D14FF400724FF48073B8
:10B94000A4F8E822A4F8F432B4F8F4220020B4F801
:10B95000E8324FF48071120284F8F602A4F8EA1279
:10B9600002FB03F3B3F1807FC4E9BB2357D8012264
:10B970003C4B84F8FD22C4F8E4323DE7062101FB8C
:10B9800002C263E7384B9A4235DC053B9A4235DD0B
:10B99000364B1344032B4BD801A252F823F000BFBF
:10B9A000E7B90008D7B90008C9B9000839B90008D3
:10B9B000A3F52203013B9A423AD02CDD2C4B9A424C
:10B9C00009D001339A4219D14FF48073A4F8E832B8
:10B9D000A4F8F432B8E780224FF48073A4F8E82288
:10B9E000A4F8F432B0E740224FF48073A4F8E822C0
:10B9F000A4F8F432A8E71F4B9A42E5D0002394F84C
:10BA0000CC021D46A4F8E832A4F8F432C4E9BB33F2
:10BA10003CF05CFDF0E6184B9A42D5D0EEE70123EE
:10BA2000B721D4F8040384F8FC324BF0F7FC9EE70E
:10BA300020224FF48073A4F8E822A4F8F43283E7BC
:10BA40004FF480621023A4F8E822A4F8F4327BE7D4
:10BA5000E04C0120C44F0120ACE505081640E00091
:10BA60001720C200B4E505081940EF00EABF10FF37
:10BA700017BA20001870EF0018600100884F0120ED
:10BA80002DE9F04F0421B94C002340264FF0A0428D
:10BA900004F552656160022194F8BD038BB0C4F8CF
:10BAA000C84F6661C4F80054226023632361E362D7
:10BAB0006362A161E160C4E90733002800F05C81A2
:10BAC00003201E46114684F8BD03936823F001034A
:10BAD0009360CB68084643F04003CB60FDF7F2F873
:10BAE0008B6B012E054643F480338B6316D0FDB17A
:10BAF00094F8D05F0223012D84F8BD3300F0FA8062
:10BB000023688021012059625A6A42F480029A62B5
:10BB1000FCF706FE00200BB0BDE8F08F8B6843F009
:10BB200006038B608B6843F020038B60002DDFD110
:10BB300023683220DA6822F0C042DA60DA6842F024
:10BB40008042DA6009F06CFF606848B32A4601273A
:10BB50002946C2EBC203561C04EB830383F83C2046
:10BB6000A3F84220F2B283F83D70824283F83F107E
:10BB70001965C3E91111ECD300221146C2EBC203CF
:10BB8000561C04EB830383F8FC21F2B283F8FD1109
:10BB9000824283F8FF11C3F81012C3E98111EDD37B
:10BBA00000222368D4F80CC01646D4F81080D4F8CC
:10BBB0002CE0D4E90671019102F14001013203EB5E
:10BBC00081010F2A4E60F7D19A6BBEF1000F40F051
:10BBD0003D8122F400129A631A6842F040021A6012
:10BBE0001A6842F080021A600022012F03F50066F5
:10BBF000C3F8002ED3F80028C3F80028D3F8002893
:10BC000000F01B81032F00F0188142F00302C3F8FB
:10BC100000284FF48461564A196102E0013A00F0AD
:10BC20002C8119698F06F9D41021514A196102E05B
:10BC3000013A00F020811969C906F9D40021316167
:10BC40007161F161E0B103F510624FF0904A4FF07D
:10BC5000006B0F464FF67F399C4607E017600131B5
:10BC60001761C2F808902032814260D01368002B1F
:10BC7000F4DA11B1C2F800A0F1E7C2F800B0EEE7C3
:10BC80003269B8F1010F22F48072326100F0E7806E
:10BC900000216FF0804299615A61B8F1000F03D121
:10BCA0009A6942F010029A619969324A0A439A618C
:10BCB000019A1AB19A6942F008029A61BEF1010F25
:10BCC00000F0C880002D7FF413AF0121626A84F870
:10BCD00038508A4284F8BD1300F0D1807368032085
:10BCE00043F00203736009F09BFE94F8D05F012DCE
:10BCF0007FF406AF03204AF03DFD03283FF400AF78
:10BD000023688022284640215A625A6A42F400126F
:10BD10009A62FCF705FD20210220FCF701FD40217D
:10BD20000320FCF7FDFC00200BB0BDE8F08F0021E4
:10BD300063460CF530624FF0904A4FF0006B0F46AF
:10BD40004FF67F39844607E0176001311761C2F86A
:10BD500008902032614593D010680028F4DA11B1C0
:10BD6000C2F800A0F1E7C2F800B0EEE7F819012030
:10BD7000400D030000383C8000F0FF064B4B0320D1
:10BD80004FF4C05584F8BC631A6B42F001021A6389
:10BD90000A221B6B069105A903F001030890444891
:10BDA0000493049B07960595099208F0B1FEE36A97
:10BDB000012B71D03D4B062143205A6B42F080028B
:10BDC0005A635A6B02F080020292029A5A6C42F451
:10BDD00080425A645B6C03F480430393039BFDF73A
:10BDE0007FFE34490820A269032388602168012A64
:10BDF00084F8BD338B68266923F001038B607FF4E0
:10BE000068AE8A6B2C4B22F48032606B8A63012807
:10BE1000CA6803EA0203CB60CB6823F44013CB600B
:10BE200003D1CB6843F48013CB600846FCF74AFF8C
:10BE3000012E05467FF45BAE70E6BCF1000F3FF4C7
:10BE4000E6AE42F00102C3F80028E2E642F4001236
:10BE50009A63C9E69969194A0A439A6132E718490F
:10BE60000020184A31636FF08041376B3A433263E8
:10BE70009861596118E70125E0E60125D4E684F8C8
:10BE8000F4539969C4F8FC2341F000610E4A9961AA
:10BE9000596D0A435A6521E74FF4007305A9044818
:10BEA0000593CDE9066608F033FE83E700380240CB
:10BEB0000000024000E100E0BFFFBDFF04000040C1
:10BEC00000018000030001000300001099B10A6B1B
:10BED000824216D9154BD3F83C23914221D34C39D9
:10BEE00091421ED30B6B9842F9D38B6B9842F6D8D4
:10BEF0000B46184670470D4BD3F83C130A6B904223
:10BF000012D30B680BB9F4E70A6B90420B4602D3CD
:10BF10008A6B9042EDD951F84C3F002BF4D1184672
:10BF200070470023184670470A46D8E7E04C0120C6
:10BF30002DE9F047CC0143D1034622494FF0FF32AF
:10BF4000022443F8081B7E2642601846DFF87880FA
:10BF50002644051D6FF07047D8F840934FF0010A52
:10BF6000013E494608E0A3421CD0631C45F8043C4E
:10BF7000321B1C460435CAB10B6BA34202D88B6B33
:10BF8000A34204D22046FFF7A1FF014690B10A79EF
:10BF90004B6B002AE7D1A34204D0E6D2631C45F8DC
:10BFA000042CE5E7631C45F8047CE1E7C8F840137E
:10BFB000BDE8F087321B631C494645F804ACD8E75E
:10BFC0008026C3E7F8FFFF0FE04C0120F0B5002307
:10BFD0000E680DE0BCF1050F17D9BEF1050F18D89A
:10BFE0000A2C16D103EB830316F8010B04EB430371
:10BFF000A0F13005A0F1610CA0F1410EA0F13704D1
:10C00000EFB2092FE6D82C46ECE7A0F157040A2C32
:10C01000E8D00E601360F0BD036870B55E6A26B1AB
:10C0200033460522BDE87040184704460D464E1DB4
:10C0300000E023689B68204698470028F9D02368D1
:10C04000204615F8011B1B689847B542F1D170BD19
:10C05000036870B55E6A26B133460822BDE87040B9
:10C06000184704460D4601F1080600E023689B6866
:10C07000204698470028F9D02368204615F8011B70
:10C080001B689847B542F1D170BD00BF2DE9F0475C
:10C090000023194D84B0074695F94D9305F5557663
:10C0A0004FF0B60A00EB010805F2F4551C46D6F82D
:10C0B00000C0304600226946E036BCF1000F14D0C3
:10C0C0009CF838C0BCF1140F0FD019F1020F01D049
:10C0D000CC450AD1CDE90244CDE90078ADF808A0FD
:10C0E0008DF80E402EF0AAFF0346B542DFD1184668
:10C0F00004B0BDE8F08700BFE04C01202DE9F74314
:10C10000A0230124114E18255FFA84F8FF2B14DCBC
:10C11000E9B2D6F8F4055F1CDBB2C1F11C02C1F133
:10C120001B0180F80B808272C9B202680093002361
:10C13000D2F818904246C8473B46013DE6D101344B
:10C14000052CE0D103B0BDE8F08300BFE04C012036
:10C1500010B50A4C94F81106003818BF0120FFF7FB
:10C1600075F850B1064904F5BF603CF03FF904F59D
:10C17000BF6011F08FFB04F5BF6010BDE04C0120E3
:10C18000E0E50508094B93F8D63F042B08D9053B99
:10C19000032B08D801231A4600B1037010467047DC
:10C1A00000230122F8E700231A46F5E7F8190120D9
:10C1B0002DE9F0479AB004460D4617469846DDF83B
:10C1C0009090DDE9226A02E0206837F065FF206880
:10C1D00037F06AFF0028F7D10146642201A851F028
:10C1E00053FF264B8DF80450CDF85CA00293002D30
:10C1F00040D0AB1E012B3FD9042D14BF00230323D5
:10C200001F4A8DF805300123D2F8CC2F039616442F
:10C210008DF85B30CDE90594049637B14246394636
:10C2200007A851F0BFFE8DF85A80164E002396F8ED
:10C2300062961893B9F1000F19D196F8610664223D
:10C2400001A902FB006000F2646051F0ABFE012323
:10C2500086F8619686F86236236843B143463A46CB
:10C26000294620461AB0BDE8F04713F0FFBA1AB0CD
:10C27000BDE8F0870523C3E70223C1E7005301208F
:10C28000F8190120E04C01209FED747A07EE901A16
:10C2900020EE070AF8EE677A27EE800AFDEEC07AF4
:10C2A00017EE903A2033402B00F2C880DFED6C7A15
:10C2B000B4EEE70AF0EE407AF1EE10FA0CDD9FEDF5
:10C2C000696ADFED696AB0EE677A77EEC67AB4EE36
:10C2D000E67AF1EE10FAF6DC9FED647AF4EEC77AB6
:10C2E000F1EE10FA0CD59FED5F6ADFED616AB0EEFA
:10C2F000677A77EE867AB4EEE67AF1EE10FAF6D443
:10C300009FED5C7AF4EEC77AF1EE10FA40F3868086
:10C310009FED537A77EE677A67EEA75A9FED565AEC
:10C320009FED566AB6EE007ADFED556AA5EE856A96
:10C3300027EEA55AE5EE866AE5EE267A27EE877A9D
:10C34000DFED4C6A70EE267ABDEEE76A16EE103A23
:10C350002033402B6FD8B4EEE60AF1EE10FA0CDD74
:10C36000DFED405A9FED406AF0EE676A77EEE57ABE
:10C37000F4EEC66AF1EE10FAF6DCDFED3C6AF4EE9C
:10C38000E67AF1EE10FA0CD5DFED365A9FED386AF9
:10C39000F0EE676A77EEA57AF4EEC66AF1EE10FA6F
:10C3A000F6D4DFED346AF4EEE67AF1EE10FA48DD09
:10C3B000DFED2B6A76EEE77A67EEA75ADFED2E4ABD
:10C3C0009FED2E6AB8EE005ADFED2D6AA5EEA46A45
:10C3D00067EEA54AE5EE866AE4EEA67A67EE857A10
:10C3E000C7EE206A0023836143610362B7EE006AEF
:10C3F000C36176EE865A76EE666A86EE257A67EE39
:10C40000277A80ED007A66EE876A80ED027AC0EDC9
:10C41000017AC0ED037AC0ED046A70479FED197A86
:10C42000F4EEC77AF1EE10FA7FF576AF9FED0F7A52
:10C4300077EE677A70E7DFED147AD1E79FED127A35
:10C440007EE7DFED106AF4EEE67AF1EE10FAB3D58E
:10C45000DFED066A76EEE77AAEE700BF27D4D23684
:10C46000DB0F4940DB0FC940E4CB1641DB0F49C06D
:10C47000E4CB16C1DB0FC93F92E741B99730083CC6
:10C4800015A82ABEDB0FC9BF0000000030B400238E
:10C49000314D32494CF25034C5F8E436304AD1F8C7
:10C4A000F80904E0D1F8F8391B1AA3420FD8D36871
:10C4B000DB03F7D4D16811F4F9710BD1D06810F017
:10C4C000010002D001230846D36030BC704703202E
:10C4D00030BC7047D3689B0705D5D5F8E43643F0E8
:10C4E0002003C5F8E4361E4BDB68DC0605D5D5F81D
:10C4F000E43643F01003C5F8E436194BDB689806C0
:10C5000005D5D5F8E43643F00803C5F8E436144BF6
:10C51000DB68590605D5D5F8E43643F00403C5F8C1
:10C52000E4360F4BDB681A0605D5D5F8E43643F040
:10C530000203C5F8E4360A4BDB68DB0505D5D5F800
:10C54000E43643F04003C5F8E436054B4FF4F97286
:10C550000120DA6030BC7047E04C0120F02A012055
:10C56000003C02400C480D4BD0F8001710B48A1E56
:10C570000B4C2231C0F8F036B0F81A371B01A4FB7F
:10C5800003C3DB08A3F5B06322F8023F9142F3D165
:10C590005DF8044B704700BFE04C01203D2C0208C1
:10C5A000CDCCCCCC70B5084C251D2E4614F8010B13
:10C5B0002EF00EFF28B10378B44205F8013BF5D107
:10C5C00070BDFF23F8E700BF1C5401202DE9F047A0
:10C5D0001C4F01264FF03C094FF0000807F10805F9
:10C5E000B24617F8010B3AF02BFE044690B180F8E2
:10C5F0000690C671FB7803F07F02012A17D013F072
:10C60000800F20460CD185F804803AF069FF85F848
:10C6100005802C6001360835052EE2D1BDE8F08793
:10C6200085F804A03AF062FF85F805A0F1E71B0643
:10C6300004D42046FDF742FBFB78E0E73AF056FFD2
:10C64000F7E700BF245401202DE9F04F454B85B09A
:10C65000DFF824810126DFF8249103F57F6A08F1D1
:10C660000C0718F801BBBBF1000F66D04FEA1B1591
:10C670000BF00F01013D032D6DD809EB4502908DA4
:10C6800040FA01F414F0010468D001224D44364C04
:10C690008A40013A10404EF0CFF895F8342004213A
:10C6A000104404EBC0047C61E671A171002102E03A
:10C6B0000131152941D001EB41004A001AF8005020
:10C6C0005D45F5D1274B0392184490F8F11F0029DE
:10C6D00046D0584635F090FE0546006848F03AFED0
:10C6E000697935F0C7FE90F800B0BBF1000F24D196
:10C6F0001E490420039A0A4402F8C76C02F8C80CC9
:10C70000F4B120461A4C2A7A02213AF0C3FC294699
:10C71000184A3846B4F86E57B4F86C47CDE9004B68
:10C72000B2FBF5F301369BB22EF08EF80123F6B280
:10C73000183707F8073C092E93D105B0BDE8F08FF4
:10C740000B4B29460B4A3846B3F86E57B3F86C3793
:10C75000CDE90034E4E700247C61A7E77C61A5E72C
:10C760000B68FFDEF8190120542A0120F02A01206D
:10C77000E04C012040420F0050540120F8E205082F
:10C780008E4B2DE9F04193F83C2882B00190002AAD
:10C7900040F00E8193F86028B7EE007AB3F8647821
:10C7A000012107EE902AB3F86208F0EE475ADFED58
:10C7B000846AB8EEE76A07FA01F507EE900AB3F863
:10C7C0005E08804CE6EE665A8542A6EE267AA4F80C
:10C7D0000871F8EEE77AB8BF054683F83C18AEB2A8
:10C7E00067EEA67AA4F80C61C4ED3F5A84ED407A56
:10C7F000C4ED417A002A00F0D880DDED017AADB2B7
:10C800009FED710AF8EE677A6D0080EE270A4FF00F
:10C81000C3F88046B0FBF5F5012DB8BF0125EDB298
:10C82000B0FBF5F39BB284F8105100EE103ABBEE6A
:10C83000ED0A84ED450A4FF0AFF8644BDFED646A12
:10C84000A3FB0838DFED630A9FED636A00234FEA1C
:10C85000D8089FED621ADFED625A07EE908ADFED8D
:10C86000611A9FED612AF8EEE77ADFED602A9FED0D
:10C87000603ADFED603A86EEA77A5F49B7FBF0F0E9
:10C880000228B8BF022084F8180184ED477A07EE29
:10C89000903AB8EEE77AF0EE467AE7EE207AFDEECF
:10C8A000E76A16EE902A2032402A7BD8B4EEC17A8D
:10C8B000F1EE10FA0CDDDFED516A9FED517AB0EE2A
:10C8C000675A77EEE67AB4EEC75AF1EE10FAF6DC64
:10C8D000F4EEE57AF1EE10FA0CD5DFED486A9FED43
:10C8E000497AB0EE675A77EEA67AB4EEC75AF1EEFF
:10C8F00010FAF6D4F4EEC67AF1EE10FA4ADD73EED1
:10C90000E77A67EEA76AB0EE424AB7EE007A67EEC2
:10C91000E64AA6EEA14A77EE677AB0EE627AB6EE04
:10C92000005AA6EE847AE4EE877A67EE857A0133C0
:10C93000E1EC017A202BAAD107EE905AB7EE006AFB
:10C94000314A1020F8EEE76A07EE906A2F4B02F1A9
:10C950002806F8EE677A202186EE267A84F821569A
:10C96000C4F8C42702F1A8051422C4F8C067C4F8AB
:10C97000D057C3EDAC7AC3EDAD7AC3EDAE7AA4F86F
:10C98000BC07A4F8CC17A4F8C82783ED007A02B03E
:10C99000BDE8F081F4EEC37AF1EE10FA48BF75EE0F
:10C9A000E77AAEE7F6EE007AC1E7194B1A7024E792
:10C9B000044C94F81051B4F80C61BDE7E04C012030
:10C9C0000AD7233C1400002000247449ABAAAAAA69
:10C9D000DB0FC9413C8C4F3EDB0FC93F0100F840E3
:10C9E000DB0F49C092E741B99730083C15A82ABE31
:10C9F000DB0FC9BFDB0F494034010020DB0FC9400A
:10CA0000E4CB1641E4CB16C130E605083806002019
:10CA10000000002070B5044684B04FF4004030F0B0
:10CA2000F9F888B3002303214FF4E13590F90400AD
:10CA30001A46029301914FF40041009530F049F9F4
:10CA4000124BC3F86808F8B1012C40F698024FF475
:10CA500061714FF00A0608BF4FF496620C4D83F8DF
:10CA60006C4801200B4CA3F874280B4AC3F870687B
:10CA7000A3F87618A3F87818C3F87C58C3F8804850
:10CA8000C3F8842804B070BD0020FBE7E04C01200F
:10CA9000798E010845D901086D8E01082DE9F8430A
:10CAA000204D0023204E4FF0050895F8A77805F695
:10CAB000A40506F5206486F8FC7915F8010B03F14E
:10CAC000010908BB20604B460434032BF5D1F94320
:10CAD000D6F8000A01F001013AF00EFD96F8FC19B3
:10CAE000D6F8040A81F00201C1F340013AF004FDD6
:10CAF00096F8FC19D6F8080A81F00401BDE8F8435D
:10CB0000C1F380013AF0F8BC3AF09AFB20605FFA7A
:10CB100089F310B180F80680C3712068FDF7CEF864
:10CB2000D1E700BFE04C0120F02A01202DE9F041BF
:10CB30002A4C82B02A4DB4F8AC68A5F80C6AEEB95C
:10CB400094F8A8083AF07CFB94F8A928C5F8100AD4
:10CB5000003A18BF012285F80E2A48B194F8AA18A5
:10CB60002B220029C28014BF112101213AF04EFB73
:10CB7000002002B0BDE8F0413BF072BA94F8A888FA
:10CB800000222B21404635F0C7FC074640463AF0CC
:10CB900057FB00B117B902B0BDE8F0812B22C5F8F0
:10CBA000280A4FF00008C280397AFEF767F80D4A6C
:10CBB000CDF804803946A4F8AE6805F61420B2FB1F
:10CBC000F6F3C3F34F049BB200942DF03DFED5F86D
:10CBD000143AC3F8008085F8258ADCE7E04C012090
:10CBE000F02A012040420F002DE9F84F254B002686
:10CBF00093F8BC2803F6B30703F50D6483F8B02857
:10CC00005FFA86FB4FF0010917F8010F01360BEBB5
:10CC1000090A49464FF000085FFA8AFA524635F091
:10CC20007BFC054640B3387804F80E8C04F80D8C74
:10CC300004F80FBC04F8109C44F8045C3AF000FBC4
:10CC400018B180F8069080F807A0297AFEF716F848
:10CC50000D4A002128464BF0C5FC0C4B221D2146F5
:10CC6000236028460A4BC4E9013848F0F3FA4246EB
:10CC7000697928682DF044FD082E04F11C04BFD109
:10CC8000BDE8F88FE04C012040420F00D1A7030817
:10CC9000E197030870B52C4C00222C4B022194F82C
:10CCA000E809C4F8E039C4F8A029C4F8A429C4F8F4
:10CCB000A829C4F8DC29A4F8E42935F02DFC0028C3
:10CCC00040D0234B0546026803F1C000597C11B1E6
:10CCD00059688A422BD018338342F7D1002394F845
:10CCE000E809C4F8CC5884F8C0383AF0A9FA08B179
:10CCF0000223C380297A0026FDF7C0FF2846154A83
:10CD000000214BF06FFC144A1448154B111FC4F856
:10CD1000D0082846C4F8D438C4F8D86848F09AFA3D
:10CD2000324669792868BDE870402DF0E9BC926A06
:10CD30000C4801320C49D0F86431B3FBF2F381F8AE
:10CD40003C33CBE770BD00BFE04C012000FFFF008B
:10CD50004800002040420F00B45501200998030804
:10CD6000A5990308F02A0120000001202DE9F04FC9
:10CD7000B64D85B00E46DFF80C930446C02205F18F
:10CD800034000021019651F07FF999F8E939002B20
:10CD900070D099F8EA39002B00F08B80DFF8CCB224
:10CDA0009BF8E43F012B00F0AE80022B00F08E8058
:10CDB000A74BA84E1C4602939BF8DA7F0FCE0FC4F8
:10CDC0000FCE0FC4391EA44A9BF8D63F18BF0121CD
:10CDD000C5F83C29072B85F85C1996E8070084E81C
:10CDE000070000F20981042B00F21381DFF898821A
:10CDF0000026DFF880A2019B5FFA86F90321B34287
:10CE000009F101072BDD1AF8014BFFB220463A4623
:10CE100035F082FB034620461C4613B33AF010FA65
:10CE2000C8F8140018B14FF00303C77183719BF861
:10CE3000D73F9BF8D62F002B00F0E980E37983F0F1
:10CE4000010349462046013648F0C0FA48B14FF088
:10CE50000103082E08F1180808F8073CCBD1029B03
:10CE600006E07E4900237E4AC5F84019C5F84829E6
:10CE7000C5F85839D5F8583963B100220121019815
:10CE800083F82D1083F82C001A6383F82E2005B048
:10CE9000BDE8F08F734E744C0FCE0FC40FCE0FC48D
:10CEA00096E80700A4F1200384E80700C5F8583984
:10CEB000EDE76E4B2046019993F8D82F003A18BF42
:10CEC0000122FCF779F8C5F85809D3E79BF8DA3F57
:10CED000002B3FF46DAF9BF8D63F082B13D105F61E
:10CEE00024135C4E5C4F1C460293012385F85C3989
:10CEF0000FCE0FC40FCE0FC496E80700C5F83C79DB
:10CF000084E807007BE0019B0026DFF880C1584CD5
:10CF1000C5F8603989F8EC69BCE80F000FC4BCE8BB
:10CF20000F000FC49BF8DA3F04F15C079BF8D62F83
:10CF30009B1B89F8242A18BF012385F85C39A4F6C5
:10CF4000DC039CE8070003934A4B84E80700029344
:10CF50000BE03AF0C5FAFB68082E039A07F12007A8
:10CF6000536102F1180303934DD0D5F86039B342F1
:10CF700049DD029B13F8018B4046029335F0FEFA1F
:10CF8000044640463AF05CF99BF8D72F824694F865
:10CF900007800AB188F0010808F0010495F85C29BF
:10CFA000013489F8EB490AB188F0010850463AF09B
:10CFB00089FA00283DD0504601363BF08FF8C7F87B
:10CFC0000CA061017860F2B287F8108041F00D0189
:10CFD0007961BAF1000F05D04FF003038AF80720FA
:10CFE0008AF8063050463AF011F918F0010F504611
:10CFF000AFD13AF07BFAAEE7082B7FF4F7AE1E4BC9
:10D00000C5F86439F2E61A48C5F8580932E7E379F9
:10D0100017E79BF8D93F194A012BC5F8642905D0B9
:10D020009A1E53425341002F18BF002385F86839D8
:10D03000DCE6134B01220949C5F80839084BC5F84D
:10D040000C1989F8EC29C5F81439DDE71400002023
:10D050003809002084E70508D52F05087D0A040853
:10D06000750A040858E70508D0560120F819012070
:10D0700004090020D3290120DD3300001134000011
:10D08000810A0408E04C012048000020B0E70508B0
:10D09000F8B5704F97F814073AF0D2F897F815578B
:10D0A00058B12D230446C380FCF70EFE0A2035F04C
:10D0B0002DFD20463BF008F818B9D7F8283ADA00D9
:10D0C00000D5F8BD013D092DFBD897F81347D4B919
:10D0D00040202FF09FFD0028F3D090F9043097F8FE
:10D0E000E916092BC8BF143B0A293B4493F82C4A84
:10D0F00000F0A28093F8383A97F81227002A08BF68
:10D100001C46002CDDD020463AF09AF8054600284F
:10D1100000F08B802D23C380FCF7D0FD0121084651
:10D120003AF0F2F92B68AA889A613C2035F00AFEA1
:10D13000002101203AF0E8F997F81537002B38D094
:10D140000026454C94F8FC19D4F8000AC94301F0B4
:10D1500001013AF0D1F994F8FC19D4F8080A81F0E9
:10D160000401C1F380013AF0C7F97820002D38D0CE
:10D17000AB8801362A681B04936135F0C7FC94F82C
:10D18000FC19D4F8000A01F001013AF0B5F994F85D
:10D19000FC19D4F8080AC1F380013AF0ADF92B6804
:10D1A000AA8878209A6135F0B1FC97F815379E422D
:10D1B000C8DB97F8133783BB97F81437002B80D15F
:10D1C00097F81637012B7FF47CAFD7F8283A13F085
:10D1D00080537FF476AF87F81537BDE8F8403FF00D
:10D1E00071BE7820013635F091FC94F8FC19D4F822
:10D1F000000A01F001013AF07FF994F8FC19D4F823
:10D20000080AC1F380013AF077F9782035F07EFC06
:10D2100097F815379E4295DBCBE7322035F092FD2B
:10D220002846002139F0F2FFC6E7FCF747FD01214F
:10D2300008463AF069F978E7D7F8503A5B057FF588
:10D2400040AF0AF0A1FD00287FF43BAF002C7FF433
:10D250005AAF36E7E04C0120F02A0120344870B480
:10D2600090F8543AA3F13001092958D800F6542413
:10D2700000F66320224612F8015FA5F1300109296A
:10D2800004D88242F7D1002070BC7047141B022CD6
:10D290004BDD2848002101E010F8013B01EB810142
:10D2A000161A044603EB4103022EA3F1300303F0E8
:10D2B000FF01F1DC204B03FB01F1A2424FF0000320
:10D2C0000ED903EB830314F8016B5B00A242A3F1B8
:10D2D0003003334403F0FF03F3D1184800FB03F39A
:10D2E0002E2D06D01648A0FB032370BC01EB930043
:10D2F000704701320425002404EB84041078013DBA
:10D30000303864000928A4B2204401D8013284B224
:10D3100015F0FF05F0D1642202FB0433E2E700219F
:10D320001D4600F654220B46DAE70021054CC4E7FF
:10D33000E04C0120355701208096980040420F00B4
:10D34000ABAAAAAA34570120094BD3F8640AD3F830
:10D35000682AD3F86C3A904202DC1146024608462D
:10D36000984204DD9A42B8BF1A461046704770478B
:10D37000E04C0120124A02F52760D2F87C1AD2F85C
:10D38000802A30B419C8984202DC1D46034628465C
:10D39000914202DC15460A4629468842A8BF084643
:10D3A0009342B8BF1346844202DB2246044610462D
:10D3B000984203DD9C422046B8BF184630BC7047F7
:10D3C000E04C01200B6810B414681B1B0360546808
:10D3D0004B681B1B5DF8044B43608B6892689B1A7B
:10D3E0008360704738B50D460446FF2100682A4621
:10D3F00050F04AFE22682A44226038BD2DE9F047E9
:10D40000041E0D4612DB092C26DC0B46814A82489D
:10D410000021A0FB04605970C00800EB8000A4EB61
:10D420004000125C28461A70BDE8F08764422D2344
:10D43000092C01F8013B24D8764A774B0020A3FB46
:10D44000046348702846DB0803EB8303A4EB430323
:10D45000D35C0B70BDE8F0876F4B632CA3FB0426F5
:10D460004FEAD60621DC0B466A4A6B49A1FB06014E
:10D47000C90801EB8101A6EB4101515C03F8011BD6
:10D48000C5E7654A632CA2FB04364FEAD60637D8B7
:10D49000604A614BA3FB0603DB0803EB8303A6EBA7
:10D4A0004303D35C01F8013BC7E7A3FB0627B4F5B0
:10D4B0007A7F4FEAD7070DD20B46564A5649A1FB51
:10D4C0000701C90801EB8101A7EB4101515C03F899
:10D4D000011BCAE7A3FB072842F20F7294424FEAEE
:10D4E000D80836D80B464B4A4B49A1FB0801C9085E
:10D4F00001EB8101A8EB4101515C03F8011BDDE761
:10D50000A2FB0637B4F57A7F4FEAD7070CD2414A1F
:10D51000414BA3FB0703DB0803EB8303A7EB4303A8
:10D52000D35C01F8013BB4E7A2FB073942F20F7369
:10D530009C424FEAD90921D8364A374BA3FB09034D
:10D54000DB0803EB8303A9EB4303D35C01F8013B46
:10D55000DEE7A3FB0829314A94424FEAD90921D8D2
:10D560000B462C4A2C49A1FB0901C90801EB81019A
:10D57000A9EB4101515C03F8011BB5E7A2FB093A95
:10D58000264B9C424FEADA0A21D8224A224BA3FBBF
:10D590000A03DB0803EB8303AAEB4303D35C01F824
:10D5A000013BCAE7A3FB09231D4A94424FEAD30A71
:10D5B00021D80B461849174AA1FB0A01C90801EBFB
:10D5C0008101AAEB4101515C03F8011BCAE7A2FBF0
:10D5D0000A38134B9C424FEAD80813D80E4B0D4A19
:10D5E000A3FB0803DB0803EB8303A8EB4303D35C33
:10D5F00001F8013BCAE70A22BAFBF2F03FF094FCC3
:10D600000346D7E70A22B8FBF2F03FF08DFC014653
:10D61000E4E700BFB0700608CDCCCCCC9F860100FB
:10D620003F420F000C461646054683B52DF024FFF9
:10D6300020462DF021FF0021204B0846002E08BF78
:10D640001E4639F061FF0021012039F05DFF2846B8
:10D6500036F02AFDB0B10121002039F055FF2846EF
:10D6600036F01AFD0746204636F01AFD0028FAD09B
:10D670003946204636F01CFD3846B04700210846A2
:10D6800039F042FF204636F00FFD0028DFD001219F
:10D69000002039F039FF204636F0FEFC01462846CE
:10D6A000019136F0FDFC01990028F8D0284636F0AB
:10D6B000FFFC0021084639F027FFC8E7099F03084F
:10D6C000F0B5002289B0DFF898C004AF13460A60B5
:10D6D0004A603E468A60CA600A610268C2F38550A9
:10D6E00040FA03F43546E40704D513F80C4005F876
:10D6F000014B2E460133062BF2D1174DC2F3032402
:10D700000023C2F305302C4405F2F44C33700DF1C4
:10D71000190694F8EC448DF8184040FA03F43546A5
:10D72000E40704D513F80C4005F8014B2E460133ED
:10D73000062BF2D10023C2F3834506AC08463370B2
:10D7400002F00F030549C2F303120097CDE901452A
:10D7500046F0FAFA09B0F0BDF8E20508D8700608FC
:10D76000DCE7050870B5094C0546D4F8842A62B197
:10D77000002601362D21D4F8840A3BF079FBAE4215
:10D78000F7DBBDE870403CF08FBD70BDE04C012080
:10D7900038B50546084640F0E9FB041E0D4B0FDB8B
:10D7A00093F86C2A944205DA21460B483DF034FD8B
:10D7B000204638BDFF2C03D108483DF02DFDF7E78A
:10D7C00093F86C2A284606494FF0FF34013A3CF0A2
:10D7D00013FDEDE714000020E7700608F870060856
:10D7E0000B710608114A0130002302EBC000F0B4AF
:10D7F000D0F800C50E4E3360336133623363336457
:10D80000336533663367BCF1000F0DD090F8FC74BC
:10D8100057B13F0100240CEB0403351910340FCB32
:10D82000A74285E80F00F6D1F0BC7047F8E2050882
:10D830006857012038B50F4C034694F80F1B04F6C7
:10D84000083084F80B3B01F03F0101F10A058B1C05
:10D85000083184F80A5B254484F80D3B1CF0A0FFD6
:10D8600085F8060B94F80A3B000A1C4484F8070B61
:10D8700038BD00BFE04C012038B51E4C0968D4F813
:10D88000345B0068491B1C4DDFED1C6A00EE901AEA
:10D89000D4F8301BD5EDD07A1C46F8EEE00A401AD9
:10D8A00060EEA70A07EE900AF8EEE77A20EEA07A7B
:10D8B000B1EE670AA7EEA77AF1EEC77A67EEA67A0D
:10D8C000FCEEE77AC2ED007A46F054FA9FED0C7A4E
:10D8D000DFED0C7AE0EE077AFDEEE77A17EE902A9C
:10D8E000002A02DBC4ED007A38BD48F6A043134499
:10D8F000236038BDE04C0120000001202C7D8E3FCC
:10D90000A00CB34500A00C4638B50A4C00250122F6
:10D91000802120462FF06AF930B194F904002FF0ED
:10D9200099F908B1006838BD01350C34092DEED1E4
:10D930000020F8E72858012038B5041F00F1080539
:10D9400054F8043FD81780EA430018F0C5FCA542FC
:10D95000F6D138BD084B4FF6FF70002103F5276262
:10D9600010B40024C3F81C0BC2F8A410C3F8184B61
:10D970005DF8044B704700BF140000202DE9F04112
:10D98000BB4CDFEDBC7AD4F8242B94F8053B07EEB2
:10D99000102A2DED028BB8EE478A28EE278A002B3D
:10D9A00045D094F8707A002F40F0B680B24E002532
:10D9B000DFEDB28A4FF0000894F8283B2B41DB07DB
:10D9C00012D594F8043B1BBBB4F8063B07EE103AA3
:10D9D000002F46D0B8EE477AC8EE877A77EE887A7D
:10D9E00088EE277A86ED027A01352436042DE3D1BC
:10D9F00094F8095BB4F80C6BB5BB2FB994F8203BD5
:10DA000084F8307B84F82C3BBDEC028BBDE8F081C0
:10DA1000B4F8063B301DD4F8241B00EE103AB8EEE3
:10DA2000400ACFB946F078FA94F8707ADCE794F8B7
:10DA3000041B94F8212BB1FA81F1D4F8100BB4F83F
:10DA4000065B490925F03EFC80B28542A4F8060B2E
:10DA5000A7D094F8707AA9E750F03EFC94F8707A59
:10DA6000C2E7C6F80480B5E7854A94F80A3BD2F8C5
:10DA7000B82B92F8832013435ED1A5F1010194F8ED
:10DA8000212BD4F8100BB1FA81F1490925F01AFCC9
:10DA900080B2A4F80C0B002F61D194F8203B84F8DD
:10DAA000305B84F82C3B0028AED007EE900A0123AF
:10DAB000B8EE678A9D42DFED717A84F8343BC7EE99
:10DAC000888A00F08B80022D9ED1D4F8241BB0EE02
:10DAD000480A6C4846F020FA94F8303B012B00F0DD
:10DAE000C180022B90D1B0EE480AD4F8241B6648BE
:10DAF00046F012FA94F8303B012B00F0AE80022B76
:10DB000082D1B0EE480AD4F8241B6048BDEC028BE9
:10DB1000BDE8F04146F000BA94F8095BB4F80C6B2C
:10DB2000002D3FF471AF564A94F80A3BD2F8B82B57
:10DB300092F88320134304D0002F7FF465AF304662
:10DB4000ABE7A5F1010194F8212BD4F8100BB1FA41
:10DB500081F1490925F0B6FB80B2A4F80C0BB04264
:10DB60003FF452AF00283FF44FAF94F8303B002B06
:10DB70003FF44AAF07EE900A012BB8EE678ADFED5B
:10DB80003F7AC7EE888A47D0022B7FF43DAFD4F8A6
:10DB9000241BB0EE480A3B4850F09EFB94F8303B03
:10DBA000012B52D0022B7FF42FAFB0EE480AD4F8ED
:10DBB000241B354850F090FB94F8303B012B47D0A4
:10DBC000022B7FF421AFB0EE480AD4F8241B2F4873
:10DBD000BDEC028BBDE8F04150F07EBB2C4A002129
:10DBE000D2ED007A134678EEA76A43F8041F87EE59
:10DBF000A67A83ED017A78EEA76A0021996087EE14
:10DC0000A67A83ED037A77EEA88A00221A6187EE5E
:10DC1000A87A83ED057AF7E61D4A1346F3EC017AFC
:10DC200078EEA76A87EEA67A83ED017AD2ED007AC4
:10DC300078EEA76A87EEA67A83ED037A77EEA88A54
:10DC400087EEA87A83ED057ADEE6114A131DEDE72B
:10DC50000F4A131DD2ED007AF0E70D4A131DD2EDE5
:10DC6000007AD0E70A4A131DD2ED007AC3E700BF5D
:10DC700014000020BD378635840A002083F9223E37
:10DC8000E04C01204C0B0020700B0020940B002076
:10DC9000B80B0020012816D02F4B93F8C03B012B66
:10DCA0002CD02E4BF6EE006ABEEE007ADFED2C7A19
:10DCB00003EB800090ED000A80FE660A80FE070AF2
:10DCC00020EE270A7047274AF6EE006A224BBEEE86
:10DCD000007A02F6D431DFED227A93F8C43B91ED5D
:10DCE000010A80FE660A80FE070A20EE270A23B199
:10DCF000B5EEC00AF1EE10FA03DC70479FED1A0A88
:10DD0000704707EE903AB2F9BE1BB2F9D23BDFED95
:10DD1000176AF8EEE77ACB1A07EE103AB8EEC77A30
:10DD200027EE267AB4EEE77AF1EE10FAE6DA77EE2D
:10DD3000C77AB2EE047AF4EEC77AF1EE10FADCD8C4
:10DD4000B1EE047A67EEA67A30EE470AA7EE807A43
:10DD5000B0EE470A704700BF14000020B4580120FD
:10DD600000004843E04C012000000000CDCCCC3D39
:10DD7000F8B5774B40F60301B3F8E02B0A402DEDE0
:10DD8000048BB0EE408A04D0B0EE480ABDEC048BA0
:10DD9000F8BD03EB4003B5EEC00ADFED6E6AF7EEA7
:10DDA000007AB3F9BC1BBFEE007AB3F9D03BF1EEB9
:10DDB00010FA694E4FEA8007A1EB030306EB8004DB
:10DDC000C8BF012100EE103AD8BF4FF0FF31D4F8A0
:10DDD000C85BB8EEC00A20EE260AB5EEC00AF1EE26
:10DDE00010FACCBF4FF0010C4FF0FF3C77FE877A62
:10DDF0006B1A18BF0123002D08BF0023002B49D147
:10DE000006F53D62F0EEC06A92ED007AF4EEC76A64
:10DE1000F1EE10FA07DD614508BF002D0CBF0123AC
:10DE2000002300F08580002D42D0B0EE408A4B4A9E
:10DE3000DFED4B8AD2ED006A97EE278A9FED497A93
:10DE4000DFED497A28EE268A88FE478A88FE278AEF
:10DE5000002B61D196F8183C984295D1434C94F828
:10DE60009D3D262B90D1B2EE049A20EE090A4DF08A
:10DE700093FDB0EE480AA4F8A25DA4F8A00D4DF001
:10DE80008BFD28EE890AA4F8A40D4DF085FDA4F8B9
:10DE9000A60D79E706F53D63F0EEC06AC4F8C82B1D
:10DEA00093ED007AF4EEC76AF1EE10FA3EDC134609
:10DEB00006EB80029FED2E6AD2ED6F7AF0EEE76AF4
:10DEC000F4EEC66AF1EE10FA2DDC9FED2A6A66EEDA
:10DED000866A294AF0EE408AB7EE006A92ED005A4F
:10DEE000FFEE005A67EE857AE6EEA78AF5EEC08A65
:10DEF000F0EEE87AF1EE10FAF4EE477ACCBF0124A6
:10DF00004FF0FF3436FE256AF1EE10FA01DDA14232
:10DF100014D00025002B9DD00744184B002203EBA2
:10DF200087035A6096E7F7EE006AD2E76145BED1F3
:10DF3000F21965460123C2F8C8CB74E7B0EE688ACF
:10DF400052ED017A002597EE068A28EE278AE3E74C
:10DF5000E04C0120CDCCCC3D14000020E80B00208B
:10DF60000000000000007A4400007AC4E83B012071
:10DF7000FFFFF9436F12033BEC0B0020F00B002076
:10DF800070B46F4C0A7804F6D43304EB80066D4D00
:10DF900007EE902A03EB8001D6F8E43BB8EEE76A7F
:10DFA000D1ED006A514207EE101A85FB0315DB170D
:10DFB000B8EEC77AC3EB651307EE903AF8EEE77A4E
:10DFC000E6EE267AF4EEC77AF1EE10FA05D407EE03
:10DFD000102AF8EE476A86FEE77A04EB400040F626
:10DFE0000101B4F8E02BB0F9BC3BB0F9D00B114201
:10DFF000DFED556AA3EB000307EE903AF8EEE77AFF
:10E00000A7EEE67A06D0514B93ED000A70BC27EEDE
:10E01000000A7047B4F9BC3BB4F9BE2B002B4C4846
:10E020004C49B8BF5B42002AD0ED017AB8BF5242DA
:10E030009BB290ED006A92B291F8200C87FE866A3E
:10E040009342B8BF134607EE903AF8EEE77A67EED0
:10E05000A67AE0BB01F62C43DFED3F5AD3ED006A10
:10E06000F4EEE56AF1EE10FA61D5F7EE005A9FED95
:10E070003B4A9FED3B5A01F6244175EEE65AD1ED3D
:10E08000004A75EE677A65EE845AE5EEA76A66EE99
:10E09000A46ADFED347AF4EEE76AF1EE10FA4BD9B8
:10E0A000DFED314AF7EE005A84EEA65AF0EE656ACB
:10E0B000E6EE456AC6FEE56AC6FEA76A2B4BD3EDBF
:10E0C000007A67EE277A70BCA7EEA60A704701F6C1
:10E0D00024439FED245AD3ED005AF4EEC55AF1EED5
:10E0E00010FA21DD01F62841D1ED004AF4EEC54ACF
:10E0F000F1EE10FA18DDDFED1E6A74EEE77AB7EE86
:10E10000004A26EE266AC7EEA46AC6EE257AC6FE47
:10E11000C46AC6FE856A77EE847A66EEA76AC6FE92
:10E12000C46AC6FE856AC9E7F0EE456AC6E701F62D
:10E130002441D1ED006AACE7F0EE676ABEE700BFAC
:10E14000E04C01201F85EB51CDCCCC3D300C0020A4
:10E15000CC58012014000020AE47813F610BB63B34
:10E1600000003443000000000000C842440C0020BE
:10E170000000C8C22DE9F04F0C4F97F89D5D102D9F
:10E180002DED048B83B000F06184094C002694F8D7
:10E19000B987B8F1060F00F24484DFE818F0D30421
:10E1A000940565040B00D800A8056903E83B01202D
:10E1B00014000020E34B102D1A4693ED037AD3EDA3
:10E1C000057AB2EC011A27EE073A67EEA73A93ED0B
:10E1D000077A92ED006AD3ED097A27EE074AD3ED6C
:10E1E0000B6A66EE062A93ED0D7A67EEA74AD3ED29
:10E1F0000F7A26EEA65AD3ED021A67EE075A93ED70
:10E20000042A27EEA76AD3ED116AE1EE012A93ED05
:10E21000137AA1EEA13AD3ED157AE2EE023AD3EDEC
:10E22000060A66EEA66A93ED081A27EE077AD3ED82
:10E230000A1A67EEA77A93ED0C2AA0EEA04AE1EE47
:10E24000014AD3ED0E0AA1EEA15A93ED101AE2EEA7
:10E25000025AD3ED121A93ED142AA0EEA06AE1EE51
:10E26000016AE2EE027AA1EEA17AB1EEE22AF1EEC3
:10E27000C32AB1EEE33AF1EEC43A03ED202AB1EE3F
:10E28000E44A43ED1F2AF1EEC54A03ED1E3AB1EE12
:10E29000E55A43ED1D3AF1EEC65A03ED1C4AB1EEC4
:10E2A000E66A43ED1B4AF1EEC76A03ED1A5AB1EE76
:10E2B000E77A43ED195A03ED186A43ED176A03ED47
:10E2C000167A93ED177AD3ED197A67EE075AD3EDE4
:10E2D0001B6A27EEA76A93ED1D7AD3ED1F7A66EECF
:10E2E000A66AD3ED164A27EE077A93ED185A67EE21
:10E2F000A77AE4EEA45A93ED1A4AA5EE056AD3ED87
:10E300001C4A93ED1E5AE4EE046AA4EEA47AE5EEEC
:10E31000057AB1EEE55AF1EEC65AB1EEE66AF1EED3
:10E32000C76A03ED155AB1EEE77A43ED145A03EDCF
:10E33000136A43ED126A03ED117A00F0758794F8C1
:10E34000B98708F101085FFA88F884F8B98794F86A
:10E3500018310F2B00F3B6877B490D2B03F1010C0D
:10E3600001EB830200F2C38701F2844A02F5C66220
:10E370000AEB8301D2ED007A91ED6C7AB4EE677A04
:10E38000F1EE10FA05DDB5EEC07AF1EE10FA00F309
:10E3900046870020DFED6D7A0AEB8C02D2ED6C6AC5
:10E3A000F4EE476AF1EE10FA08DDF4EE676AF1EE7A
:10E3B00010FA03DDF0EE667A5FFA8CF0D91C03F1F7
:10E3C000020C0E29624600F3EE800AEB830292ED06
:10E3D0006E7AB4EE667AF1EE10FA08DDB4EE677A82
:10E3E000F1EE10FA03DDF0EE477A5FFA8CF00AEBFB
:10E3F0008302D2ED6F6AF4EE476AF1EE10FA07DDA0
:10E40000F4EE676AF1EE10FA02DDF0EE667AC8B259
:10E41000591D03F1040C0E29624600F3C4800AEB77
:10E42000830292ED707AB4EE667AF1EE10FA08DDAE
:10E43000B4EE677AF1EE10FA03DDF0EE477A5FFA98
:10E440008CF00AEB8302D2ED716AF4EE476AF1EECA
:10E4500010FA07DDF4EE676AF1EE10FA02DDF0EE75
:10E46000667AC8B2D91D03F1060C0E29624600F384
:10E470009A800AEB830292ED727AB4EE667AF1EE3C
:10E4800010FA05DDB4EE677AF1EE10FA00F3E786D4
:10E490000AEB8302D2ED736AF4EE476AF1EE10FAEA
:10E4A00005DDF4EE676AF1EE10FA00F3D38603F1AE
:10E4B000090103F1080C0E29624674DC0AEB8302A1
:10E4C00092ED747AB4EE667AF1EE10FA05DDB4EEF0
:10E4D000677AF1EE10FA00F3CD860AEB8302D2EDF3
:10E4E000756AF4EE476AF1EE10FA05DDF4EE676A3C
:10E4F000F1EE10FA00F3B98603F10B0103F10A0CF7
:10E500000E2962464FDC0AEB830292ED767AB4EE76
:10E51000667AF1EE10FA05DDB4EE677AF1EE10FAE4
:10E5200000F3B3860AEB8302D2ED776AF4EE476A12
:10E53000F1EE10FA0CDDF4EE676AF1EE10FA00F37A
:10E540009F8605E068080020B4010020000000005C
:10E5500003F10C01012B0A4625DC0AEB830292ED44
:10E56000787AB4EE667AF1EE10FA07DDB4EE677AE7
:10E57000F1EE10FA02DDF0EE477AC8B20AEB830240
:10E58000D2ED796AF4EE476AF1EE10FA09DDF4EEA5
:10E59000676AF1EE10FA04DD03F10D00F0EE667A21
:10E5A000C0B203F10E0202F16C030AEB82010AEB26
:10E5B000830CD1ED6B6A9CED007AF4EE476AF1EEC4
:10E5C00010FA07D5B4EE677AF1EE10FA02DDF0EE3C
:10E5D000477AD0B20F2A02F1010C00F0F3830AEB64
:10E5E00083030AEB8201D3ED006A91ED6D7AF4EEBC
:10E5F000476AF1EE10FA05D5B4EE677AF1EE10FA3B
:10E6000000F37D860E2A02F1020300F0DB830AEBA1
:10E61000830191ED6C7AD1ED6B6AF4EE476AF1EE0D
:10E6200010FA05D5B4EE677AF1EE10FA00F37186B0
:10E630000F2B03F1010200F0C5830AEB820191ED7B
:10E640006C7AD1ED6B6AF4EE476AF1EE10FA05D5FB
:10E65000B4EE677AF1EE10FA00F364860F2A02F145
:10E66000010300F0AF830AEB830191ED6C7AD1EDE9
:10E670006B6AF4EE476AF1EE10FA05D5B4EE677AEC
:10E68000F1EE10FA00F357860F2B03F1010200F0B0
:10E6900099830AEB820191ED6C7AD1ED6B6AF4EE0D
:10E6A000476AF1EE10FA05D5B4EE677AF1EE10FA8A
:10E6B00000F34A860F2A02F1010300F083830AEB7C
:10E6C000830191ED6C7AD1ED6B6AF4EE476AF1EE5D
:10E6D00010FA05D5B4EE677AF1EE10FA00F3408631
:10E6E0000F2B03F1010200F06D830AEB820191ED23
:10E6F0006C7AD1ED6B6AF4EE476AF1EE10FA05D54B
:10E70000B4EE677AF1EE10FA00F336860F2A02F1C2
:10E71000010300F057830AEB830191ED6C7AD1ED90
:10E720006B6AF4EE476AF1EE10FA05D5B4EE677A3B
:10E73000F1EE10FA00F329860F2B03F1010200F02D
:10E7400041830AEB820191ED6C7AD1ED6B6AF4EEB4
:10E75000476AF1EE10FA05D5B4EE677AF1EE10FAD9
:10E7600000F31C860F2A02F1010300F02B830AEB51
:10E77000830191ED6C7AD1ED6B6AF4EE476AF1EEAC
:10E7800010FA05D5B4EE677AF1EE10FA00F31C86A4
:10E790000F2B03F1010200F015830AEB820191EDCA
:10E7A0006C7AD1ED6B6AF4EE476AF1EE10FA05D59A
:10E7B000B4EE677AF1EE10FA00F30F860F2A02F139
:10E7C000010300F0FF820AEB830191ED6C7AD1ED39
:10E7D0006B6AF4EE476AF1EE10FA05D5B4EE677A8B
:10E7E000F1EE10FA00F302860F2B03F1010200F0A4
:10E7F000E9820AEB820191ED6C7AD1ED6B6AF4EE5D
:10E80000476AF1EE10FA05D5B4EE677AF1EE10FA28
:10E8100000F3F5850F2A02F1010300F0D3820AEB21
:10E82000830191ED6C7AD1ED6B6AF4EE476AF1EEFB
:10E8300010FA05D5B4EE677AF1EE10FA00F3E88528
:10E840000E2B40F0BF82B84B93ED007A53ED016A76
:10E85000B4EE667AF1EE10FA40F3B482B4EEE77AE1
:10E86000F1EE10FA40F3AE82F0EE477A0F20ACE200
:10E8700094F8BA2794F83436DFF8C0E203F5937CB5
:10E88000C3F120030CEB421C13F0FC0FC3F3850013
:10E890005FFA83F80EEB8C0C00F00D8501300CF163
:10E8A0001003AEF170010EF244624FEA00190CEB56
:10E8B000001013ED026A103311ED027A103253ED9D
:10E8C000076A103153ED057A26EE076A51ED074AC3
:10E8D00013ED087A834211ED085A66EEA46A51EDF1
:10E8E000055A27EE057A02ED066A67EEA57A42ED33
:10E8F000076A02ED087A42ED057ADAD18B49A9F16F
:10E90000100301F2B4629C44C818134418F00302C7
:10E910001BD0DCED007A013A90ED007A67EE877A41
:10E92000C3ED007A11D0DCED017A012A90ED017A75
:10E9300067EE877AC3ED017A07D0DCED027A90EDBD
:10E94000027A67EE877AC3ED027A94F834060028DB
:10E9500063D094F8BA370EEB880C5FEA90090EEB9F
:10E96000C31E0CF2346C01EB88080EF5936E35D0A3
:10E9700009F101090EF1100308F110010CF1100268
:10E980004FEA091A0EEB091913ED026A103311ED63
:10E99000027A103253ED076A103153ED057A26EEF4
:10E9A000076A51ED074A13ED087A4B4511ED085AF5
:10E9B00066EEA46A51ED055A27EE057A02ED066A65
:10E9C00067EEA57A42ED076A02ED087A42ED057A14
:10E9D000DAD1AAF110039E4498449C4410F003003D
:10E9E0001BD0DEED007A013898ED007A67EE877A69
:10E9F000CCED007A11D0DEED017A012898ED017A94
:10EA000067EE877ACCED017A07D0DEED027A98EDD9
:10EA1000027A67EE877ACCED027A102D7BD094F8DB
:10EA2000B98708F10108424BA3FB0823A8EB0302B6
:10EA300003EB52039B08C3EBC303A8EB030384F867
:10EA4000B93703B0BDEC048BBDE8F08F34F0FCF8AF
:10EA5000384C97F89D5D064694F8B987102D08BF8D
:10EA6000A7F8A08DFFF795BBDFF8CC80DFF8D0E0EA
:10EA7000B0EE006AD8ED005AF6EE006ADEED007ADC
:10EA80000EF18C03B4F8BC0777EEA77AD4F8D01750
:10EA90000138B0EE664A1031B0EE677A08EBC0027A
:10EAA000E5EE867A083A95EE867A67EEA67A27EE44
:10EAB000267ACEED1F7A8EED207AD2ED036A0138E8
:10EAC000D2ED027A01F1080153ED215AA2F10802B8
:10EAD00053ED224A03F1080335EEE67A11ED036A9D
:10EAE00037EEE45A77EEA47A76EEA56A51ED045A31
:10EAF000A6EE057AE5EE857AA5EEE67AE6EE267ACA
:10EB000027EE047A67EE847A03ED037A43ED047A04
:10EB1000D3D1102D83D134F097F8801B94F8B987A6
:10EB2000A7F8A20D7DE700BF2408002034010020D3
:10EB30002549922414000020E8070020B401002099
:10EB4000EC070020B4F8BC379A485908D4F8C0271D
:10EB500000EB8308DB084FEA810C00EB810A00F030
:10EB6000A38003F1010E0CF1100C0AF11003103018
:10EB70000AEB0E1AC44402F1100908F1100E5EED02
:10EB8000047A103310ED041A09F110095CED041A2F
:10EB9000103013ED086A71EE278A5EED032A31EE1C
:10EBA000671A1CED032A36EE218A5EED013A71EEFA
:10EBB000C61A13ED064A0EF1100E53ED054A0CF17C
:10EBC000100C5EED066A53ED075A5CED067A1CEDFB
:10EBD000057A35EE820A10ED063A72EE655A10EDAE
:10EBE000075A74EE270A10ED056A77EEC47A40EDF5
:10EBF000088A35EE229A36EE232A35EE625A73EEF3
:10EC0000268A00ED079A74EE872A00ED052A37EE72
:10EC1000647A40ED068A73EE666A43ED052A36EEA5
:10EC2000636A03ED088A03ED070A43ED060A5345BC
:10EC300059ED074A19ED084A24EEC12A24EE653A37
:10EC400065EE242AA5EE042A61EE843AB0EE435A1A
:10EC5000E1EE042AE5EEA43AA1EEA45A0EED072A4D
:10EC60004EED082A4CED073A0CED085A59ED055ABD
:10EC700019ED065A26EE253A65EEE63A27EE854A64
:10EC800065EE474AE6EE053AA6EE853AA7EE254A36
:10EC9000E7EEA54A0EED063A4EED053A0CED054AB3
:10ECA0004CED064A7FF46BAF89B242480191F9F707
:10ECB00051FA01994046D4F8C027F9F74BFA102DC4
:10ECC0007FF4ADAE27E7DFF8EC80D4F8C4274046E8
:10ECD000B4F8C8174AF0DCFF97F89D5D102D00F0DE
:10ECE000FE8294F8B937013384F8B937BEE6324B67
:10ECF0001B78002B00F06882304A94F8BA3702F192
:10ED0000DC08D4ED3F7A03EBC300D4F8A41108EB80
:10ED10008303D4ED410A02EB800093EDAC0AD0F8F6
:10ED20001CA0D0F8209020EE270A90ED054AD0F8DC
:10ED300018B0FDF7A9FA80ED054A6C32C0F818B09A
:10ED4000C0F81CA0C0F8209094F8BA37D4ED407AEF
:10ED500008EB8308D4F8A41103EBC30098EDAC0AC8
:10ED600002EB800020EE270AD0F814A0D0F818900B
:10ED7000D0F81C80026AFDF787FA102DC0F814A0A5
:10ED8000C0F81890C0F81C80026200F0A08294F8CD
:10ED9000BA270B4B013294F8B907A3FB02130130D9
:10EDA00003F4FF7184F8B90701EB5303D21A84F816
:10EDB000BA275FE5E8070020000000205C0500207E
:10EDC000ABAAAAAA002800F04E81431E012B40F3F3
:10EDD000C4820AEB8002811E92ED6B7A1346D2ED5B
:10EDE0006A6AF4EEC76AF1EE10FA00F38280012934
:10EDF0007FD093ED697AC21EB4EEE67AF1EE10FA96
:10EE000000F34982012A00F04682D3ED686A021FAE
:10EE1000F4EEC76AF1EE10FA6BDC012A69D093EDCB
:10EE2000677A421FB4EEE67AF1EE10FA00F333820D
:10EE3000012A00F03082D3ED666A821FF4EEC76AC1
:10EE4000F1EE10FA55DC012A53D093ED657AC21F1A
:10EE5000B4EEE67AF1EE10FA00F31D82012A00F01A
:10EE60001A82D3ED646AA0F10802F4EEC76AF1EEEB
:10EE700010FA3EDC012A3CD093ED637AA0F109023E
:10EE8000B4EEE67AF1EE10FA00F30582012A00F002
:10EE90000282D3ED626AA0F10A02F4EEC76AF1EED3
:10EEA00010FA26DC012A24D093ED617AA0F10B023E
:10EEB000B4EEE67AF1EE10FA00F3ED81012A00F0EB
:10EEC000EA81D3ED606AA0F10C02F4EEC76AF1EEBC
:10EED00010FA0EDC012A0CD093ED5F7AA0F10D023E
:10EEE000B4EEE67AF1EE10FA00F3D581022A07FEBD
:10EEF000267A431C0E2B00F33C820AEB800100F1C2
:10EF0000020CD1ED6D6A0A4691ED6E6AB4EEE66AC6
:10EF1000F1EE10FA00F36E81BCF10F0F00F08E805D
:10EF2000D2ED6F6AC11CB4EEE66AF1EE10FA00F1A0
:10EF30005F810F2900F0B28192ED706A011DB4EE7D
:10EF4000E66AF1EE10FA00F355810F2976D0D2ED82
:10EF5000716A411DF4EEC66AF1EE10FA00F34881C1
:10EF60000F2900F09B8192ED726A811DB4EEE66A72
:10EF7000F1EE10FA00F33E810F295FD0D2ED736AF3
:10EF8000C11DF4EEC66AF1EE10FA00F331810F29CB
:10EF900000F0848192ED746A00F10801B4EEE66A33
:10EFA000F1EE10FA00F326810F2947D0D2ED756AF1
:10EFB00000F10901F4EEC66AF1EE10FA00F31881CF
:10EFC0000F2900F06B8192ED766A00F10A01B4EE30
:10EFD000E66AF1EE10FA00F30D810F292ED0D2ED82
:10EFE000776A00F10B01F4EEC66AF1EE10FA00F355
:10EFF000FF800F2900F0528192ED786A00F10C0138
:10F00000B4EEE66AF1EE10FA00F3F4800F2915D0A1
:10F01000D2ED796A00F10D01F4EEC66AF1EE10FA54
:10F0200000F3E6800E2940F03981E14A92ED006A52
:10F03000B4EEE66AF1EE10FA00F3DC8087FE667A41
:10F04000C7EE878A94F8BA9709F1AC0BB2EE007A52
:10F050000AEB8B02F7EE007A92ED008AC8FEC78AAF
:10F06000C8FEA78A17E0F2EE008AB7EE007AC7FE64
:10F07000E88AC8FE878A94F8BA9794ED450A09F1A0
:10F08000AC0B0AEB8B0393ED008A88EE000A4CF080
:10F0900083FCC0B2431C0AEB800207EE900ADBB28D
:10F0A00092ED6C7AF8EEE76A0F2B27EE077A66EEA0
:10F0B000876A69D80AEB830207EE903A012892ED3D
:10F0C0006C6AF8EEE77A26EE066AE6EE276A37EE15
:10F0D000067A59D8B5EEC07AB4F80C31F1EE10FAD0
:10F0E00069DD86EE879A94ED457A29EE077AB4F8C1
:10F0F000082107EE902AF8EE677AF4EEC77AF1EE6F
:10F1000010FA05DC07EE903AF8EE677AC7FEC77A88
:10F1100094ED477A77EEC87A0AEB8B0A28EE877A65
:10F12000A7EE278A8AED008A27F028FA0028B8BFC0
:10F130004042C0B214280DD9B4F8343C07EE903ADE
:10F14000F8EEE77A87FE888ABCEEC88A18EE103A95
:10F15000A4F8343CB9F1000F32D10F2D00F0A1809A
:10F16000112D6AD1934B9FED940AD3ED007A28EECE
:10F17000800AFDEEE77A17EE903AA7F8A03D4CF032
:10F180000BFCA7F8A20D4AE40138C0B20AEB8003D9
:10F1900007EE900A93ED6C6AF8EEE77AB4F80C315A
:10F1A00026EE066A37EE067AE6EE276AB5EEC07AF4
:10F1B000F1EE10FA95DCB0EE487A9FED809A96E772
:10F1C000102D7FF42EACA6E494F8BA377C4803EBFC
:10F1D000C302D4ED410A00EB8303D4F8A41100EB81
:10F1E000820093EDE30AD0F814A0D0F81890BFE5A0
:10F1F000F0EE466A87FE667AC7EE878A94F8BA9779
:10F2000009F1AC0BB2EE007A0AEB8B02F7EE007A52
:10F2100092ED008AC8FEC78AC8FEA78A3BE7F0EED7
:10F22000477A1846FFF7B8B833F00EFD801B97F801
:10F230009D5DA7F8A40DFFF782B82B2DC0D15D4BC3
:10F24000D3ED007AFDEEE77A17EE903AA7F8A23DEB
:10F25000FFF7E5BBF0EE667AC8B2FFF728B9F0EE2B
:10F26000477A5FFA8CF0FFF713B9F0EE667AC8B20E
:10F27000FFF742B9F0EE477A5FFA8CF0FFF72DB94D
:10F28000F0EE667AC8B2FFF763B9F0EE477A5FFA3C
:10F290008CF0FFF747B9B0EE667A2AE6F0EE466AE0
:10F2A000CCE69FED450A29EE000A4CF075FBA7F865
:10F2B000A60DFFF7B6BBAEF180010EF2346308462F
:10F2C000FFF724BBF7EE008ADFF8F8A0D3E633F0AF
:10F2D000BBFC801B97F89D5DA7F8A20D57E533F0A6
:10F2E000B3FC801B97F89D5DA7F8A20DF9E41A46C0
:10F2F00001F2844A0020DFED317AFFF754B90E2A7B
:10F30000F0EE477A5FFA8CF002F102037FF47FA9F6
:10F310005BE50F2BF0EE477AD8B203F101027FF4E0
:10F320008CA952E50F2AF0EE477AD0B202F1010320
:10F330007FF499A949E50F2BF0EE477AD8B203F193
:10F3400001027FF4A6A940E50F2AF0EE477AD0B279
:10F3500002F101037FF4B3A937E5B7EE007AC8E5FF
:10F360000F2BF0EE477AD8B203F101027FF4BDA96A
:10F370002BE5F7EE006A61E60F2AF0EE477AD0B28D
:10F3800002F101037FF4C7A91FE50F2BF0EE477AC6
:10F39000D8B203F101027FF4D4A916E50F2AF0EEEA
:10F3A000477AD0B202F101037FF4E1A90DE500BF75
:10F3B00024080020E80800200000C84200000000E7
:10F3C0005C050020380600200F2BF0EE477AD8B2FB
:10F3D00003F101027FF4E1A9F7E40F2AF0EE477A86
:10F3E000D0B202F101037FF4EEA9EEE40F2BF0EEB0
:10F3F000477AD8B203F101027FF4FBA9E5E40F2AB2
:10F40000F0EE477AD0B202F101037FF408AADCE4FF
:10F410000E2BF0EE477AD8B23FF415AAD5E4F8B532
:10F42000214C1D270E46054684F8F87B1BF0DCFABC
:10F4300000201BF07DFA08201BF07AFA0E201BF04A
:10F4400077FA38461BF074FA04201BF071FA042096
:10F450001BF06EFA00201BF06BFA30201BF068FAEC
:10F4600000201BF065FA30461BF062FA00201BF00A
:10F470005FFA1BF0A5FA04F6F9301BF0AEF923464B
:10F4800070B194F8F92B62B994F8FA2B302A00D0B5
:10F490003AB993F8FB2B22B993F8FC3B01202B706F
:10F4A000F8BD0120FCE700BFE04C0120104B0344F5
:10F4B00010B5044693F8D40510F05EFD0D480A23FC
:10F4C00000EB44040920B4F90C1CB1F5FA6FA8BF95
:10F4D0004FF4FA61B1F57A7FB8BF4FF47A71A1F5B4
:10F4E0007A71B1FBF3F1BDE81040C9B210F072BD02
:10F4F000F8E20508E04C01201C4991F8542A9AB31F
:10F50000F0B4002605463346304637461BB991F81D
:10F51000544A2D2C22D02E2A18D0CA1800EB800075
:10F5200092F8544A4000A4F13002092A02D8A0F10E
:10F530003002A0180E2B14D80133CA1892F8542A9E
:10F54000002AE3D106B14042F0BC70470133002DE0
:10F55000F8D0CA182A4482F8547ADEE701231E46FE
:10F56000EBE70020F0BC704700207047E04C012022
:10F570001FB503AC8DF80C30002300948DF80D30CE
:10F580000FF012F804B010BDF8B5054626201FF0A4
:10F59000C9FF134C0146F8B9D4F8300C90F8383054
:10F5A0001E3B012B01D934F083FD0E4F0026AE42E5
:10F5B0000ADBB4F8543C0133A4F8543C0A4BD3F8AA
:10F5C000CC3FC4F8643CF8BD17F8011B0136D4F8F1
:10F5D000300C34F06DFDEAE7002384F8623CEDE77F
:10F5E000E04C012014590120F819012010B5FAF758
:10F5F00071FB0446112137F009FE204637F070FFF9
:10F60000C82033F09FFB2046BDE8104037F06EBFA6
:10F6100008B5002037F014FE054BC3F8680C08B19C
:10F620002A23C3804021BDE8084037F0EFBD00BF6A
:10F63000E04C01202DE9F0416A4CD4F86C110B69C3
:10F640009E0702D5CB689D074CD40B69580702D59D
:10F65000CB685A073ED40B691B0702D5CB681F073E
:10F6600030D40B69DE0602D5CB68DD0622D40B69E7
:10F67000D80702D5CB68DA0741D40B691B0603D53E
:10F68000CB681F0600F192800B69DE0503D5CB68BD
:10F690001D0600F18F800B695C0603D5CB68580608
:10F6A00000F18C800B699A0602D5CB689B0621D4A9
:10F6B000BDE8F0816FF0100200230A61CA6984F886
:10F6C0008831D4E76FF0080200230A61CA6984F820
:10F6D0008831C6E76FF0040200230A618A6984F862
:10F6E0008831B8E76FF0020200230A618A6984F862
:10F6F0008831AAE76FF020030B61BDE8F0813A4B37
:10F700006FF0010299420A61B7D1384DD5F8B06F58
:10F71000D6F81432002BB0D1DFF8D880D8F86C2C92
:10F7200092B1D5F8047502F03F003A44C5F80425BB
:10F73000D5F80425B2F5006F01D1C5F804350023D2
:10F74000C8F86C3C002843D0D5F80425D5F8083516
:10F750009A4292D0D5F80425D5F808359A4231D985
:10F76000D5F80475C7F50067D5F80405B7F5007F2F
:10F770001F4A28BF4FF40077D6F814320244C6F867
:10F780001072C6F80822002B7FF477AF0123D5F85A
:10F79000C80F8121C5F8507DC6F814323B4605F0EC
:10F7A00047F8D4F86C11C8F86C7C66E76FF08003FA
:10F7B0000B6169E76FF480730B616CE76FF04003D6
:10F7C0000B616FE7D5F80875D5F80435FF1ACBE75C
:10F7D000D5F80425064BC6F810021344C6F80832C3
:10F7E0004BE700BFF02A012000140040F819012067
:10F7F000181F0120E04C01204B78012BF0B50D784B
:10F8000026D000F53060404C404B00EB45104D6970
:10F810000669344004610469234003618B6805B1C3
:10F820004B610469C3F31203012A44F40024046108
:10F83000046943EA0403036105D0036843F0044309
:10F8400003600020F0BDCB68002BF6D04361F4E7E5
:10F850004B6993B300F510642B4FD1F808C004EB4B
:10F8600045142A4E6345D4F810E00EEA07072761D5
:10F87000276906EA07062661266938D946F4002674
:10F88000C1F814C0CCF31203012A2661266943EAA9
:10F890000603236126D0BCF1000F08D005F00F024B
:10F8A0000125D0F8343895401D43C0F834582368FA
:10F8B000002043F004432360F0BD00F51060134EB8
:10F8C000A3F50023012A00EB4514206906EA00068F
:10F8D0002661206940F400202061206903EA0003CA
:10F8E0002361E4D10B69002BE1D06361DFE746F4CB
:10F8F0000026C3F31203012A2661266943EA0603A0
:10F900002361CBD1EEE700BF0000F8FFFFFF07E067
:10F910002DE9F0434D780F78012D4DD000F530637F
:10F920006F4E4C6903EB47136E4D1F693E401E61DD
:10F930001E6935401D616CB38D68012A6A4E2C44E6
:10F940001F6904F1FF34B4FBF5F41FFA84FC06EAE6
:10F95000C44405FB0CF544EA0704C5F312051C6119
:10F960001C6945EA04051D6121D0CA78012A0AD123
:10F97000D0F8082812F4807F1A680CBF42F00052B9
:10F9800042F080521A601A6842F004421A60002065
:10F99000BDE8F0838C68012A1D69C4F3120444EAAF
:10F9A00005041C611C6944F400241C61DDD1CA6893
:10F9B000002ADAD05A61D8E74B6900F51064002BB1
:10F9C00037D104EB4714474E454D012AD4F810C0F7
:10F9D0000CEA06062661266946F400262661266999
:10F9E00005EA06052561CE7872D0012E59D1D0F8EE
:10F9F000085815F4807F25680CBF45F0005545F088
:10FA000080552560256845F004452560002ABED153
:10FA10009BB203339C08BAD0CA6800F5805302EB4E
:10FA2000840403EB073352F8041BA2421960FAD195
:10FA3000ADE704EB4714D1F808E0DFF8A490C3F376
:10FA40001206D4F8108003EB0E0C08EA09090CF139
:10FA5000FF3CDFF89080C4F81090D4F81090BCFB05
:10FA6000FEFE09EA0808DFF880C0C4F810800CEA3E
:10FA7000CE4CD4F810E04CEA0E0CC4F810C0D4F808
:10FA800010C046EA0C062661CE78012E10D0012A5D
:10FA900022D007F00F03D0F834789D403D43C0F8E2
:10FAA00034582368002043F004432360BDE8F0830A
:10FAB0002569012A25F0C0452561256945F00055D5
:10FAC000256194D10D69002D91D0164665618CE7B2
:10FAD0000D69002D89D0F9E70D69002DF6D1E0E719
:10FAE0000000F8FFFFFF07E00000F81F70B5D0F836
:10FAF000A852C1EBC1000C46002605EB80001C217A
:10FB0000C0F80822C0F8103280F8FC41C0F8146236
:10FB100080F8FD612B6901FB0451012B01F5FE7199
:10FB200008BFC0F80C22DAB228681CB9FFF764FEDF
:10FB3000002070BDFFF7ECFE002070BD0E48D0F82D
:10FB4000B03F10B5A3B190F8304D00F55260D3F836
:10FB5000042234B1002440230121FFF7C7FF2046CF
:10FB600010BD4FF400730121FFF7C0FF204610BD08
:10FB70000224204610BD00BFF819012010B50C4C1E
:10FB8000D4F80C3563B10B49013BD1F8702CC4F8A3
:10FB90000C3512F8014BC1F8702C047013B101231D
:10FBA000184610BDFFF7CAFF0123184610BD00BF5D
:10FBB000F8190120E04C012013B5074CD4F8703C33
:10FBC00003B9FEE701A8FFF7D9FF0028F6D09DF89A
:10FBD000040002B010BD00BFE04C012010B50B685E
:10FBE000064C074AC4F80C35C2F8700C0BB1002063
:10FBF00010BDFFF7A3FF002010BD00BFF8190120C2
:10FC0000E04C012070B5037C044601259BBB4FF4FA
:10FC1000007302222946F8F7C1FE4FF40073C4F8BE
:10FC20005851022281212046F8F7B8FEE5624FF4D0
:10FC30001B704EF0F1F90546C4F8A00220B300266F
:10FC4000D4F8A43206813046A5F85C621B68984758
:10FC50000121D4F8A80204F0B9FD8121D4F8A8024A
:10FC600004F0B4FD05F5037220461F230121FFF7C0
:10FC70003DFF304670BD402302222946F8F78EFE34
:10FC80004023C4F85851CCE7022070BD70B5D0F8BD
:10FC9000A052044695F8183213B9D5F814323BB97E
:10FCA00081212046F9F754F86B7A022B07D070BDFA
:10FCB0006B7A002BF4D10121F9F74AF8F0E705F54A
:10FCC000037220461F230121BDE870400EE700BFEC
:10FCD0002DE9F0410A46D0F8A05200270B4E044609
:10FCE00085F838222F7205F50B720D238121C5F896
:10FCF0002C62D0F8A80204F09BFD05F503722046A3
:10FD00001F230121BDE8F041F0E600BF55534253E7
:10FD10002DE9F047137882B0914604468A465A2B63
:10FD20005CD8DFE813F0CE005B005B007D005B0079
:10FD30005B005B005B005B005B005B005B005B00EB
:10FD40005B005B005B005B005B00B2005B005B0084
:10FD50005B005B005B005B005B00A90174005B0063
:10FD60005B0074005B005B005B005B00CD015B002F
:10FD7000F7015B005B003B015B00E0005B005B00A8
:10FD80005B005B0028015B005B005B005B005B00CD
:10FD90005B005B005B005B005B005B005B005B008B
:10FDA0005B005B005B005B005B005B005B005B007B
:10FDB0005B005B005B005B005B005B005B005B006B
:10FDC0005B005B005B005B005B005B005B005B005B
:10FDD0005B005B005B005B005B001802D0F8A012C8
:10FDE0000524002091F85D325A1C01EBC303D2B206
:10FDF00083F83C4283F84002042A00F003824FF06B
:10FE0000FF3581F85D22284602B0BDE8F087D0F8C2
:10FE1000A032002005465881284602B0BDE8F08790
:10FE2000D0F8A042002104F10B0304F11D0003F8F7
:10FE3000011F8342FBD1702094F85C320C252073A3
:10FE400094F85D02E574984213D004EBC3000133CB
:10FE500090F83C52DBB2A573042B90F84152257602
:10FE600090F8400218BF84F85C32607608BF84F8CE
:10FE70005C121223638199F80430122B98BF6381BE
:10FE80000025284602B0BDE8F08799F80130D0F887
:10FE9000A002DB0740F18381072100F1120300F18A
:10FEA0000B0583224181C3F10604D54901E092F894
:10FEB000EC2503F80129E218AB4211FA82F2F6D1DF
:10FEC000DEE7D0F8A062D6F81472002F40F02D8241
:10FED000D0F8A43208469B6898470546002840F0B1
:10FEE0006D8270818FE7D0F8A062357A002D40F0E6
:10FEF000908196F91832002BC0F27081D0F8A432AC
:10FF000008469B6898470746002840F07182D4F85D
:10FF1000A4325046DB6898470546002840F08D82A1
:10FF2000D9F80210D4F8A00209BAD0F86072C6F865
:10FF30006412B9F807305BBA9BB21944C6F868324C
:10FF4000B94200F26882B6F85E12D6F8142203FBBA
:10FF500001F3934240F09E81B3F5007F4FF0010121
:10FF6000204606F10C0228BF4FF4007331729BB299
:10FF7000FFF7BCFD47E799F80150D0F8A03215F023
:10FF8000020040F0F781D3F86012D3E999242244AB
:10FF90008A4200F201820546588134E7D0F8A082F7
:10FFA00098F80860002E40F0328198F91832002B42
:10FFB00080F2CE81D0F8A43208469B689847054667
:10FFC000002840F04E82D9F80200D4F8A06200BAAE
:10FFD000D6F86072C8F86402B9F807305BBA9BB211
:10FFE0001844C8F86832B84200F2F880B8F85E22C7
:10FFF000022003FB02F3D8F8142288F808009A4282
:020000040801F1
:1000000040F0EC80B6F85E324FF4007CD6F86872AF
:1000100006F10C05D4F8A422504607FB03F7294645
:10002000A8F80AC06745D2F81080D6F8642228BF25
:100030006746B7FBF3F39BB2C0470028C0F25F816D
:100040002A463B46D4F8A802812104F0F1FBB6F819
:100050005E52D6F83432B7FBF5F5D6E99920DF1BAE
:100060002A44451BC6F83472C6E99925002D7FF451
:1000700007AF03233372C6E6D0F8A072082000222F
:100080005F4E07F11303788107F10B05C3F10700F9
:1000900001E092F8F42503F80129C2189D4216FAEE
:1000A00082F2F6D1D4F8A4325046DB689847002893
:1000B0003FF4E6AEBB7B002563F07F03BB73A2E693
:1000C000D0F8A062002506F10B0306F1170203F831
:1000D000015F9342FBD1D4F8A43250460DF10202E5
:1000E00001A95B689847002840F0F780019B082130
:1000F000BDF802200220013BF17352BA0C211C0E04
:10010000F374F2821A0C1B0A34747274B374B082E2
:100110007181B5E6D0F8A0620846D4F8A43206F2A0
:100120005E2206F518715B6898470546002840F086
:10013000C180D6F860320821B6F85E22013B3082D9
:1001400052BA7181180EF373190C72821B0A307344
:100150007173B37357E6D0F8A07208200022284EBE
:1001600007F11303788107F10B05C3F1070001E0E4
:1001700092F8FC2503F80129C218AB4216FA82F264
:10018000F6D1D4F8A4325046DB68984700283FF4F3
:1001900077AEFB7B002563F07F03FB7333E6D4F877
:1001A000A44201EBC10199F80430E46904EB810435
:1001B00022790532934228BF13464381002B3FF436
:1001C0005FAE013B9AB2531C0C322344024413F835
:1001D000011D9C4202F80119F9D151E696F85D32F1
:1001E00005211A460133DBB206EBC202042B82F86A
:1001F000405282F83C1200F0A88086F85D323FE65B
:10020000F8E205084FF0FF3581F85D02FBE5464650
:10021000F8E6B6F85E5206F10C08D6F868720846A1
:10022000D4F8A432414607FB05F7D6F86422D3F888
:100230001490B7F5007F28BF4FF40077B7FBF5F3B4
:100240009BB2C8470028C0F22781B6F85E02D6F8F4
:100250003432B7FBF0F1D6E99925DB1B0A446D1A5D
:10026000C6F83432C6E9992525B920462946FFF754
:100270002FFDC8E505FB00F3424620460121B3F5FA
:10028000007F4FF0000528BF4FF400739BB2FFF7CB
:100290002DFCB8E590F85D3205215A1C00EBC30334
:1002A000D2B283F8405283F83C12042A3AD080F844
:1002B0005D22E5E5D4F8A0220220002592F85D3207
:1002C000591C02EBC303C9B283F83C0283F84052C5
:1002D000042924D082F85D12D2E5D4F8A0220220AD
:1002E00092F85D32591C02EBC303C9B283F8405245
:1002F00083F83C020429EDD182F85D52C0E5D4F8C0
:10030000A0220420002592F85D32591C02EBC303A1
:10031000C9B283F83C0283F840528142DAD182F8B4
:100320005D5270E580F85D526DE596F85D3205210D
:1003300000251A460133DBB206EBC202042B82F819
:100340003C1282F840527FF458AF86F85D525AE56D
:1003500098F85D3205211A460133DBB208EBC20280
:10036000042B82F8406282F83C1200F0918088F8F9
:100370005D3285E593F85D220520002511460132A6
:10038000D2B203EBC101042A81F83C0281F8405249
:100390007BD083F85D2273E593F85D220524114636
:1003A0000132D2B203EBC101042A81F8400281F884
:1003B0003C42EED1054683F85D0224E5D4F8A02244
:1003C0000220002592F85D3219460133DBB202EBC0
:1003D000C101042B81F8407281F83C0218BF82F8F9
:1003E0005D324FF0050308BF82F85D7233720AE593
:1003F000D4F8A022022092F85D3219460133DBB214
:1004000002EBC101042B81F8405281F83C0286D0F6
:1004100082F85D3234E590F85D3205211A460133E9
:10042000DBB200EBC202042B82F8405282F83C128D
:100430003FF478AF80F85D3222E5D4F8A0220220A4
:1004400092F85D3219460133DBB202EBC101042B95
:1004500081F8407281F83C02DAD13D4682F85D7243
:10046000D1E4D4F8A022022092F85D32194601337B
:10047000DBB202EBC101042B81F8406281F83C023F
:10048000C6D1354682F85D62BDE483F85D52BAE4B8
:10049000354688F85D62B6E4D4F8A0220420002531
:1004A00092F85D3219460133DBB202EBC10183429F
:1004B00081F83C0281F84052AAD130E7F8B5D0F873
:1004C000A0420546267A5EB1012E07D104F21B2216
:1004D00094F81912FFF71CFC00282FDB0020F8BD50
:1004E000D0F8A832D4F81012D3F83032D4F814224D
:1004F0001F2BC4E98C1208D12D4BD4F80C229A4240
:1005000003D194F8191201291DD994F85D32002104
:1005100005205A1C04EBC303D2B283F83C0283F8D3
:1005200040120223042A2846637214BF84F85D2215
:1005300084F85D12FFF7AAFB0020F8BD28460121D0
:10054000FFF7C6FBCAE794F81A32013B0F2BDCD841
:1005500004F21B22FFF7DCFB0028237A1DDB013BA2
:10056000022BBBD96189F1B1D5F8A07204F10C025C
:100570000420D7F83432D7F814425B1A87F838626F
:10058000A1423872D5F8A802C7F834320B4628BF0A
:100590002346812104F04CF9A0E7052BCED0284654
:1005A000FFF774FB9AE72846FFF792FB96E700BF38
:1005B00055534243D0F8A01210B50B7A022B07D046
:1005C000033B012B02D80021FFF782FB002010BD66
:1005D00001F21B2291F819120446FFF799FB00283B
:1005E000F4DA20460121FFF773FBEFE7F0B50023B3
:1005F00083B00E460446ADF806300B78D0F8A072F2
:1006000013F0600522D0202D19D14A78FE2A11D08E
:10061000FF2A14D14A8892B9CD8885B91B060ED419
:100620004FF4807107F503721F2339810121FFF711
:100630005DFA08E04D8815B9CE88012E73D02046AA
:100640000225F8F7E1FB284603B0F0BD4B780B2BF1
:10065000F5D801A252F823F097060108BF06010859
:100660003F0601083F0601083F0601083F06010852
:100670003F0601083F0601083F0601083F06010842
:10068000AD0601088906010890F87432032BD6D113
:100690008B787B60D7E790F87422032ACFD10222AF
:1006A0000DF106011D46F8F755FECCE790F87432BF
:1006B000032BC4D1391D0122F8F74CFEC3E7097999
:1006C000D0F8A80204F082F83179D4F8A80204F036
:1006D000D3F8B38896F9042003F00F03002A4FF0F3
:1006E000000203EB830304EB83032ADBC3F84421FA
:1006F000237C9BBB4FF40073022201212046F8F7B4
:100700004DF90123C4F85831D4F8A0727B7A022B3A
:1007100032D03279D20996D0012B94D020460121D3
:10072000FFF7D6FA8FE71A0689D5D0F8A4329B696D
:10073000984703463246204639463B60F8F70AFEA2
:1007400081E79A61237C83B94FF4007302228121EF
:100750002046F8F723F90123E362D5E7402302227C
:1007600001212046F8F71AF9CBE740230222812124
:100770002046F8F713F9EEE720468121F8F7E8FA6A
:1007800000237B725FE700BF2DE9F0410A7884B057
:1007900000270D4612F060060446D0F890328DF81E
:1007A0000D70ADF80E7016D0202E1AD1CE8806B37B
:1007B000120643D519460193D4F89432324668782C
:1007C0003E46D3F80880C047019BEA882046194678
:1007D000F8F7C0FD09E04B780A2B20D00B2B28D06E
:1007E0008BB120460226F8F70FFB304604B0BDE877
:1007F000F081D0F89432324648789B68984730466A
:1008000004B0BDE8F08190F87432032B29D00226A1
:100810002046F8F7F9FA304604B0BDE8F08190F8C8
:100820007432032BF3D101220DF10D01F8F792FD83
:10083000DBE790F87432032BD7D0E8E74A7803253A
:1008400083F80162394683F800221A46C0F84861ED
:100850003346C0F84C613E46C0F86C52FFF746F98B
:10086000C3E702220DF10E01F8F774FDBDE700BFEA
:100870002DE9F041037C04460125BBBB4FF4007316
:1008800002228121F8F78AF829464FF400730222E8
:100890002046E562F8F782F8C4F858514FF0010895
:1008A0000823032282212046F8F778F84FF40770D6
:1008B000C4F840804DF0B0FB0546C4F8900258B330
:1008C000D4F8943200271B689847267CC5F8147228
:1008D0004146D5F804222046C5F81872AEB140232F
:1008E0003E46FFF703F93046BDE8F081402302227F
:1008F0008121F8F753F82946402302222046E56279
:10090000F8F74CF8C4F85851C8E74FF40073FFF7F4
:10091000EDF83046BDE8F0814646E4E770B505469F
:1009200041B9D0F86C320C46032B10D0052B1FD0E8
:10093000002070BDD0F88C329B6933B190F87422DE
:10094000032A02D19847002070BD022070BDD0E973
:1009500053639E4212D8D0F88C321B6923B190F8B1
:100960007422032A00D198472846F8F7E5FCDFE710
:10097000C5F86C12F8F7ECF9204670BDF61AB342D0
:10098000C0F84C6128BF33469BB2FFF7AFF8204652
:1009900070BD00BF2DE9F04F854E83B035686C699E
:1009A00014F0010402D003B0BDE8F08F6A69AB69AE
:1009B0001A42F8D06B69AA6913409F0703D56B6987
:1009C00003F002036B616B69AA691340180379D4C1
:1009D00028464369826913405F0300F1D58042696C
:1009E00083691A4200F1BA8043698269134019058C
:1009F00008D5D5F80838DA0700F14783436903F4CE
:100A0000006343614369826913401B0110D5436948
:100A100003F00063436196F8F433002B40F0488202
:100A2000012386F8F433436DC3F38303C6F8F83328
:100A3000436982691340DF0400F1CD814369826913
:100A400013409A0400F17081436982691340DB0608
:100A500012D5836923F0100383612B6AC3F34342E9
:100A600003F00F01022A00F0E582062A00F05E8200
:100A7000836943F0100383614369826913401F0750
:100A800000F10B82436982691340DD0200F10082AC
:100A90004369826913409C0200F1F58143698269D0
:100AA0001340590000F1EA814369826913405A07F3
:100AB0007FF579AF4468630700F1F18243681C4316
:100AC000446070E7D5F81878D5F81C381F403F0C03
:100AD0003FF47EAFDFF8D8A028464FF0000800941E
:100AE00006E07F0808F101080AF11C0A00F03282D2
:100AF000F907F6D55FFA88F100F5306B0BEB411280
:100B00009268D0F8143802EA030919F0010F40F096
:100B1000268219F0080F40F0598219F0100F05D005
:100B200005F53063102203EB48139A6019F0200F8B
:100B300009D03169012900F0558305F53063202281
:100B400003EB48139A6019F4005FCAD005F53063CF
:100B50004FF4005203EB48139A60C2E7D5F804380B
:100B600023F00103C5F8043896F8F433012B00F0A4
:100B7000B681D6F8003493F8752283F8742243695D
:100B800003F0004343612FE7D0F81838D0F81C2851
:100B900013409BB2002B3FF422AF05F51062009585
:100BA000034F4FF0000A1D469046019409E000BF34
:100BB000F81901206D080AF1010A07F11C0700F07D
:100BC000CB81E907F6D55FFA8AF9D0F81028D0F87A
:100BD000344800F5106309F00F0103EB4913CC40D2
:100BE0009B68E401E4B214431C40E20732D54FF0A5
:100BF000010E009B0AF00F0C08EB4A12D3F83418D0
:100C00000EFA0CFC21EA0C01D6F810C0F445C3F82A
:100C10003418C2F808E003D1D7E911231344BB64A8
:100C2000D6F800B4B9F1000F40F0E981DBF86C327E
:100C3000022B00F0E78233F0040300F01B839BF8E3
:100C40007832012B02D100238BF87832BCF1010FEE
:100C500000F0CD82230703D508EB4A1308229A60DF
:100C6000E10603D508EB4A1310229A60620603D509
:100C700008EB4A1340229A60A30703D508EB4A13F6
:100C800002229A60240695D5D7E91441A14291D851
:100C9000621A7B6C00EB4A1C93420CF5106C28BF67
:100CA0001346DCF81820033392B2B2EB930F2CD327
:100CB00009F10109864600EB09392CB3A14223D280
:100CC000621A7B6C307C9A4228BF1A46BB6C02F1D8
:100CD000030B4FEA9B0B70B990B2033080080AD027
:100CE00003EB800153F8040B8B42C9F80000F9D1E3
:100CF000BB6CD7E91441DCF818001344114480B2EE
:100D0000BB6479658345D8D97046A142FFF452AFE0
:100D10000AF00F010124D0F8342804FA01F122EA84
:100D20000102C0F8342845E7D0F8001900F5006347
:100D3000BB4A0A40C0F800299A6802F00602042A59
:100D400000F0D1805A6842F480725A609B6813F0B8
:100D5000060340F0B081C268F36022F47052C260B2
:100D6000C36843F41053C3604FF00009D6F8004441
:100D70004FF0400800220127434620461146F7F76E
:100D80000DFE4346002220468021C4F84471C4F879
:100D90005081F7F703FE0023D4F8A022A761C4F81E
:100DA000248084F87472C4F86C326360C4F87C32B6
:100DB000002A00F0F281D4F88C32204600215B68D2
:100DC0009847D6F80034306883F81090436903F4EC
:100DD0000053436138E6D5F804284FF4846105F5E3
:100DE000006C904B22F00102CCF80420016101E07C
:100DF000013B02D002699106FAD4D6F804E0BEF1B4
:100E0000000F15D005F510634FF67F31996001345E
:100E10001A682033744522F4001243F8202CC3F8DA
:100E2000E811D3F8E02122F40012C3F8E021EDD15B
:100E3000DCF81C30326B43F00113CCF81C30002A74
:100E400040D1DCF8142042F22B031343CCF81430C9
:100E5000DCF8103043F00B03CCF81030D5F8003834
:100E6000317C23F4FE63704AC5F80038F7F744FF7D
:100E70003068436903F480534361DFE5436903F05D
:100E80008043436110E6436903F40013436105E6C0
:100E9000436903F480134361FAE5D6F8003493F80C
:100EA0007422032A39D0436903F008034361E9E55A
:100EB000D6F80034042193F8742283F8741283F86E
:100EC0007522B5E5DCF8843043F00B03CCF88430B0
:100ED000DCF8443043F00B03CCF84430BEE7002389
:100EE00086F8F4334BE6D0F8002942F00302C0F84C
:100EF00000295A6842F480725A609B6813F0060316
:100F000040F0D980C368002223F47053F260C360BC
:100F1000C36843F41053C36026E7D3F88C22D26928
:100F2000002AC0D0184690473068BCE7C1EBC10129
:100F300005F58055C3F30A1306EB81022C68D2F83D
:100F40001412C6F8C4430B442968C2F81432C6F818
:100F5000C8138DE5009C3CE5DDE900543FE505F54F
:100F600030634FF0010C32690BEB481B03EB481464
:100F70006245C4F808C0D0F840E0DBF8083000F063
:100F800017812A4A964540F0FC801A0440F1F4800B
:100F90004FF4004219F0080FCBF808203FF4BDAD24
:100FA000026CDBF80800214B9A4200F0D1801E4908
:100FB000D6F800040192F8F763FA1D4B019A9A42A1
:100FC00000F2D18008223068A260A6E54FEA4813FB
:100FD0003169026C03F5306B012905F530618344FA
:100FE00001EB0304DBF80800DDD1114B9A4200F25B
:100FF000AF800D49D6F80004F8F742FAE2E7DBF8D3
:101000008C325B69002B3FF425AE9BF87422032AD7
:101010007FF420AE58464946984730681AE600BF2C
:1010200000F8FFFF400D0300BC1D01200A31544FA2
:101030000A30544F47F6F07213423FF419ADC3F330
:101040000A14C1EBC1024FEAC10C2346033406EB7C
:101050008202A408D2F8082208D005F5805502EBD8
:1010600084072C6842F8044BBA42FAD1ACEB010277
:1010700006EB8202D2F80842D2F814121C440B4448
:10108000C2F80842C2F81432F2E4D6F8003404215F
:1010900093F8742283F8741283F87522AEE4D6F8BC
:1010A00000040122D0F88C3280F8742201795B6848
:1010B0009847306802E523F00403002B3FF422AF89
:1010C000A64A0324A64BD2F86421A6491344F4602F
:1010D0008B4240F2BF80A44BA44913448B4240F2A0
:1010E000D180A34BA34913448B4240F2EF80A24B23
:1010F000A24913448B42C0F02181A14BA149134462
:101100008B4240F21E81A04BA04913448B42C0F099
:101110001B819F4B9F4913448B42C0F01B819E4B08
:101120009E4913448B42C0F012819D4B9D4913444C
:101130008B4234BF4FF4E0534FF4C053C2684FF0BA
:10114000010922F47052C260C2681343C3600DE605
:10115000030403D54FF40042CBF808209249D6F897
:101160000004F8F78DF9316901297FF42BAF8E4A1D
:101170003068F7F7C1FD25E79A0602D52023CBF8A2
:101180000830C1EBC103D6F8000406EB8303D3F8A3
:101190000822FFF7C3FB3068BBE4D4F89032002B81
:1011A0007FF409AED4F89832002B7FF404AE08E641
:1011B0001A0752D57D4A964505D9190403D54FF42F
:1011C0000043CBF808307849D6F80004F8F758F90E
:1011D000754A01213068F7F78FFD08233068CBF896
:1011E000083096E4704AF7F787FD3068A5E4336D60
:1011F0005AEA03037FF42EAD61466B4AF7F77CFD94
:10120000306827E5DBE908239A423ED8DBF81C105A
:10121000B1FBF3F203FB12120AB98B4259D9DBF886
:101220008C32DB682BB19BF87422032A01D158461B
:10123000984780215846F7F78BFD00230522584632
:101240001946CBF86C221A46FEF750FCD6F810C0AF
:101250003068F4E44FF4705370E79A0629D52022E1
:10126000CBF8082019F0080F3FF457AC026CDBF8FC
:101270000800BAE680215846F7F76AFDD6F810C094
:101280003068DCE44FF4605358E7D31A4946B26C37
:10129000DBF8A802CBF820309BB203F0C9FA4B462A
:1012A0004A4649465846FEF721FCD6F810C0306839
:1012B000C5E413F0280FD5D13C4A964517D91B0435
:1012C00015D54FF40042CBF80820CBE74FF450532C
:1012D00034E7DBF870329942A1D24B464A46494680
:1012E000DBF8A80203F0A4FACBF87092D7E7DBF89A
:1012F0001020C1EBC100DAF80432C2F3120CDAF8A4
:10130000082206EB80001A44A3EB0C03CAF808225B
:10131000D0F80822D6F80004CAF81432FFF7FEFA13
:10132000D6F8103258EA03037FF435AF1E4A012184
:101330003068F7F7E1FC3068FFF7EBBB4FF4405340
:10134000FCE64FF43053F9E64FF42053F6E64FF441
:101350000053F3E64FF41053F0E600BFF02A0120EB
:10136000405327FFFF340C00401E1BFF3F420F007D
:1013700000DC0BFF7F4F1200808CF9FE20D613009B
:1013800060B6E5FE5FE3160000D3CEFE40771B009B
:10139000C05BB3FEC091210000CA91FE20753800E9
:1013A000E05459FEE09C4100BC1D01200A30544F1E
:1013B0000121032008B545F091F972B643F000F819
:1013C0002DE9F04FCD4C8DB00027DFF83C93A4F20F
:1013D0005F3504F6211A009054F80B0C002800F039
:1013E000FE8032F061FE0646002800F0D281D9F876
:1013F000CC3FE026A4F10B0B44F8073C00237E43CE
:1014000004F8033C54F80B0C32F04EFE002800F0B8
:10141000E68054F80B0C32F03FFE14F8023C804694
:101420005A1E0B2A0DD8DFE812F01F003A004600C2
:10143000530083009B00E200150134013F0171015C
:10144000880124280CD0009A3AB995F8B62B82422C
:1014500040F07981012204F8032C0D2BD2D186E0D3
:10146000012304F8023CCDE700234D28C4F8C53021
:1014700084F8CD3084F8CE3004D0582808D004F851
:10148000023CBFE7022284F8C43004F8022CB9E71A
:10149000032304F8023C022384F8C430B2E7042397
:1014A0003C2804F8023C0BD0B8F13E0F0CD00023CE
:1014B00004F8023CA6E70A233C2804F8023CF3D1D6
:1014C000002304F8013C9DE7012304F8013C99E75F
:1014D000D4F8C500AB19421C0344C4F8C520022A45
:1014E00083F85F8394F8CD0088EA000184F8CD107A
:1014F00088D12378C02BDAD86278FF2A08D1052B4F
:10150000D5D9012384F8C430072304F8023C79E7D5
:10151000A4F8C1200022C4F8C930934284F8C32043
:10152000C4F8C52014BF0523062304F8023C69E76C
:10153000D4F8C500AB19421C0344C4F8C52083F895
:101540005F8394F8CD00D4F8C93088EA00019A424C
:1015500084F8CD107FF456AF062304F8023C51E71F
:1015600094F8CD308342A2D10D2304F8023C14F844
:1015700001CCBCF1000F40F0ED80614B04AE08944B
:10158000ADF82CC0CDF80CC00FCB86E80F00D4F816
:10159000C930324608A9D4F8D10023440993B4F8DD
:1015A000C130ADF8283094F8C3308DF82A300123CB
:1015B0008DF82E3003AB2BF0A5FF48B1049B3146CC
:1015C00094F8C420584605934E4B049329F036FDF9
:1015D0000023039E04F8023C002E40F0D280013725
:1015E000E034032F7FF4F8AE0DB0BDE8F08FD4F8EF
:1015F000C500AA194146431C0244C4F8C53082F80C
:101600005F8394F8CD2094F8CE0088EA020201931B
:1016100084F8CD2042F0E0FD019B84F8CE00072B3A
:101620007FF4F0AEB4F80530C02B3FF640AFB4F80D
:101630000320C4F8C930A4F8C120A27884F8C320DC
:1016400000229342C4F8C52014BF0823092304F8DC
:10165000023CD7E6014694F8CE0042F0BDFD94F876
:10166000CD3084F8CE0088EA0303D4F8C50084F8AE
:10167000CD30AB19421C0344C4F8C52083F85F8306
:10168000D4F8C9309A427FF4BDAE092304F8023C75
:10169000B8E694F8CD30434084F8CD3094F8CE309D
:1016A00083427FF404AF57E7D4F8C500AA19414636
:1016B000431C0244C4F8C53082F85F8394F8CE001E
:1016C000019342F089FD019B84F8CE00052B7FF445
:1016D00099AEB4F80120B4F80330A4F8C120227800
:1016E000C4F8C93084F8C32000229342C4F8C5204E
:1016F00014BF0B230C2304F8023C83E63F50012067
:10170000FCE8050898D10120F8190120014694F859
:10171000CE0042F061FDAB1984F8CE00D4F8C500CC
:10172000421C0344C4F8C52083F85F83D4F8C93051
:101730009A427FF467AE0C23A1E694F8CE30834240
:101740007FF4B5AE10E723287FF487AE022204F8B9
:10175000032C82E6BCF1010F4FF0000602D004F822
:10176000026C3CE7D4F8C93008A8089423440993D4
:10177000B4F8C130CDE90A66ADF8283028F038FF5A
:10178000EDE754F80B0C29F077FE54F80B0CB0473A
:1017900025E714F8033C002B3FF421AFD9F8CC2FF8
:1017A00054F8071C521A632A7FF619AF012B30D068
:1017B000022B7FF414AF54F80B3C012285F8890CFE
:1017C000C5F8783CC5F87C3CC5F8843C402385F8D6
:1017D000742C85F8883C95F80F360F4A003B0F486B
:1017E000C5F8802C18BF01230D4AC5F884AA82F8D9
:1017F000383CC5F8CCAC38F05BFD4FF400502BF012
:101800003FFD084838F04AFD85F8D06C85F8D16C6A
:10181000E5E6FFF7CDFD00BF190A0408317106089F
:1018200014000020677106080022836BA3F85A2079
:10183000A3F85220704700BF836B1A6810B45C6F26
:10184000986F9168090601D5212C1AD09168490634
:1018500001D5222806D0DA6F5DF8044B42F0100261
:10186000DA67704700202024A3F85A00116821F499
:1018700090711160916821F00101916018669C6778
:10188000E9E700212024A3F85210116821F0C001DB
:1018900011605C67DAE700BF704700BF704700BFA8
:1018A000C369B3F5807F12D0826B002120201368BA
:1018B000A2F85A10196821F480711960996821F012
:1018C00001019960996821F0400199609067704723
:1018D000C369B3F5807F0CD0826B00211368A2F836
:1018E00052109A6822F080029A601A6842F0400210
:1018F0001A607047836B0121002283F83D101A772C
:10190000704700BF0122836B83F83D20704700BF02
:1019100011F0010307D090F8413003F02803282B81
:101920000CBF4223F2238A0709D590F8412002F028
:101930002802282A0CBF43F0440343F0F4034A076B
:10194000016848BF43F0B8030A6822EA03030B604A
:10195000704700BFC16838B5022903689A699C695D
:101960009A68DD680DD1C2F3C21282EA144212F005
:10197000060206D1816C01318164816C022907D095
:1019800038BD0421FFF7C4FF002380F8403038BD84
:1019900008218264D96180F8402038BD836B002221
:1019A000D3E90E0102650A6593F84120602A02D14D
:1019B000202283F8412070470023202210B5134CC9
:1019C0004363C462036380F8412080F842304B07D0
:1019D00012D50268436A526A1A70436A028D013353
:1019E00043624AB1438D013A013B02859BB2438574
:1019F000436C43F0040343640721FFF789FF102180
:101A000002680023D16180F8403010BD0000FFFF64
:101A100038B5002580F8425090F84130292B04D089
:101A200090F841302A2B0BD038BD282221230121E8
:101A300080F841200363FFF76BFF80F8405038BD0A
:101A400028222223022180F841200363FFF760FF50
:101A500080F8405038BD00BF38B50025202280F8FE
:101A6000425090F84130212B0AD0122380F84120B7
:101A7000022145630363FFF74BFF80F8405038BDF8
:101A8000112380F84120012145630363FFF740FFE4
:101A900080F8405038BD00BF836B40221A645A6CF6
:101AA00042F004025A647047704700BF836B1A6C9F
:101AB00012F0500F1A6C20D142F4007219681A64A7
:101AC0008A6812F0405F1AD19A69C2B9CA6A12F4E0
:101AD000700F02D08A68500511D44A6822F02002A3
:101AE0004A601A6C22F480721A641A6CD10406D40B
:101AF0001A6C42F001021A647047D20600D5704792
:101B00009B6BDB6C184700207047704730B1044B6B
:101B100093F900000028D4BF00200120704700BFC7
:101B2000185C012008B5FFF7F1FF50B1054A537862
:101B300092785B0003F00203002A18BF43F0010310
:101B40000B6008BD185C012008B5FFF7DFFF10B17E
:101B5000014B5B680B8008BD185C012070B5FFF776
:101B6000D5FF78B1084A158965B1D6680023B3421C
:101B70001C4607DA02EB44040133248ADBB2AC4290
:101B8000F5D30B7070BD00BF185C012008B5FFF7DE
:101B9000BDFF10B100230B70137008BD0420704707
:101BA00028B1034B93F90000003818BF012070479B
:101BB0004403012008B5FFF7F3FF40B1054B93F94B
:101BC0000020012A04DDDB78C3F340030B6008BD6D
:101BD0000020FCE74403012008B5FFF7E1FF10B146
:101BE000014B9B780B7008BD4403012070B5FFF7D3
:101BF000D7FF30B10D4CE378DB0703D500230B7022
:101C0000137070BD0A4D94F9013095F8206093FB74
:101C1000F6F301330B7094F9014095F8201094FB12
:101C2000F1F301FB134301331370EAE7440301208E
:101C3000185C0120032070470A4A70B592F82430DE
:101C400006255E1CB6FBF5F405FB146492F82550DE
:101C5000AC4205D002EBC30382F82440C3E90A0179
:101C600070BD00BF185C0120002230B5044610464C
:101C7000914200DC30BDA35C0825584010F0800F75
:101C80004FEA400318BF83F0D503013DD8B2F5D128
:101C90000132EDE710B5C9B10D4B986D814215DCED
:101CA000A2B11B6A9A4211DC013A0139094C03FBCB
:101CB000012104F10A00A1730521FFF7D5FF0621D8
:101CC000E07304F10A00BDE81040B5E710BD00BFA5
:101CD000185C01204403012000230380837083806B
:101CE000C3800372704700BF074A084992F85C300E
:101CF00009780133DBB2994282F85C3002D10023CB
:101D000082F85C30704700BF185C0120800A002018
:101D1000F8B5764C236E83B1754B1B6893F82E3063
:101D20005BB1744B94F86420A3FB0013012A4FEAC3
:101D300093132ED0022A08D002B1F8BD6E4B984200
:101D4000FBD9012384F86430F8BDA26E64329A4254
:101D50003CD894F85C3004EB031393F87C20FF2A02
:101D600005D001326549012083F87C200874FFF713
:101D7000BBFF634B01221B7884F86420092BDCD164
:101D8000B4F8FE305F4A01339BB2A4F8FE305380B2
:101D9000F8BD94F85C1004F170055B48002701EB76
:101DA0008106A366E566022500EB461354480A2621
:101DB00084F87A7000789A70092884F87B6084F837
:101DC0006450BAD101314F4B1980F8BD94F87A2094
:101DD00094F87B309A42B0D104F16F0004F1780599
:101DE000002310F8011F08224B4002E0013ACBB259
:101DF00009D013F0800F4FEA4301F7D081F00703B9
:101E0000013ADBB2F5D18542EBD194F879109942D1
:101E100037D1B4F87360012794F85C5076BA94F81F
:101E200077C004EB0511B4F87500B6B294F87830B9
:101E300040BA81F87C2043EA0C23C1F8806094F812
:101E400071C080B294F872601BB2C1F88400032D97
:101E500046EA0C2294F97000A1F88830A1F87E209F
:101E6000264A81F87D00177408D8254A12780C2A72
:101E700028D00D2A02D1234B23F81500FFF734FF99
:101E80005FE794F85C3004EB031393F87C20FF2A9F
:101E900005D001321949012083F87C200874FFF72E
:101EA00023FF174B01221B7884F86420092B7FF451
:101EB00044AFB4F8FC30134A01339BB2A4F8FC30B1
:101EC0009380F8BD03EB83031049114A03EB8303AE
:101ED000897E0C48F9409B0093FBF1F382FB0312CF
:101EE000DB17C3EBA20320F81530C7E7185C01200D
:101EF0006C090020D34D62103F4B4C00440301207D
:101F00008549012088490120500C0020CC2901205E
:101F1000676666660A4B93F87A1093F87B209142C5
:101F20000DD0C0B210B493F87A20DC6E511CD2B23E
:101F3000C9B283F87A10A0545DF8044B704770471B
:101F4000185C01200E4B0F4AD3F80031B2F900059E
:101F50005B0707D400EB8000400080B200F5C8703A
:101F600080B27047084B094ADB6B323382FB0312A5
:101F7000D817C0EBA20080B200F5C87080B27047DD
:101F8000185C0120500C0020404F012067666666F7
:101F900080F08003042B70B520D941281ED0FD2885
:101FA00006D0F0281DD0EF281FD00224204670BD97
:101FB0000B2004260F4D2E4400240135FFF7E8FFC7
:101FC0002044AE42C4B2F1D015F8010BFFF7E0FF98
:101FD0002044AE42C4B2F7D1204670BD042420464E
:101FE00070BD03200526044DE5E70C200626034DB1
:101FF000E1E700BF2CEE050830EE050824EE0508E9
:102000000C4AD2F81831F0B41C680027D2F81061DD
:102010004FF6F6751981611C9F81C3E90016207087
:10202000D2F81831D2F810111A689D81C3E9001254
:10203000F0BC7047185C01200E4BD3F8BC0203F5CE
:10204000CE7203F58E7130B403F52B75441CC3F8C2
:10205000142103F5D672C3F81851C3F80C11C3F854
:102060001021C3E9AF40C3E9671130BCC3E9AB221B
:10207000704700BF185C012000B5034683B03221D1
:10208000074A68468DF8001019689B88D2F8C42268
:10209000CDF80110ADF80530904703B05DF804FBB2
:1020A000185C01205E2810B511D05D2805D00D4BBD
:1020B000BDE81040D3F8C83218470A4CD4F8C832EB
:1020C0009847D4F8C8323D20BDE810401847054C69
:1020D0005D20D4F8C8329847D4F8C8323E20BDE815
:1020E00010401847185C0120134B002210B483F8ED
:1020F000CE12090A0F2483F8CD0283F8CF1203F51C
:1021000033700121C3F8D022C3F8D422C3F8D822F7
:1021100083F8CC4210F8014F013122440E29D2B28B
:10212000F8D183F8DA2210220449D3F8DC025DF8F2
:10213000044B31F089BF00BF185C0120E45E012030
:10214000054B002183F8E012C3F8E412D3F8DC3227
:1021500003B1C9E7704700BF185C012013B50446FE
:10216000FFF71EFDE0B100230DF106022046ADF899
:1021700006300EF0E7F898B10A4C9DF8062094F965
:1021800000106275032902D162F07F026275052199
:102190000548FFF769FD0621A0750348FFF74CFDD0
:1021A00002B010BD44030120550301202DE9F84F72
:1021B0001B4C05461E2094F8E8A294F8E9B294F866
:1021C000EA62B4F8EC92B4F8EE8294F8F0721DF082
:1021D000A9F930B1B8F1000F03D0C14601264FF084
:1021E000000A94F8F232DA070AD494F8F7223AB9DE
:1021F000012F12D0022F03D113F0020F08BF0126C6
:10220000284685F800A085F801B0AE70A5F80490C6
:10221000A5F806802F72BDE8F88F3E46F0E700BFB4
:10222000185C01202DE9F84F2DED028BFFF7B8FC6B
:10223000002843D0244B93F9000001283EDDDC7DCB
:102240001546DFF88C808E1E02EB44099FED1F8A35
:102250000FF26C0BDBE900AB4D4504D12046BDEC21
:10226000028BBDE8F88F38F8027B07EE907A26F8EB
:10227000027FF8EEE77A67EE887A17EE900A47F069
:10228000D3FE52465B4647F027FF41EC100B4BF064
:102290001BFC51EC100B48F047FA0E2F80B20AD904
:1022A00019303223B0FBF3F080B200EB800000EB7A
:1022B0008000400080B225F8020BCDE70024CDE776
:1022C0001655B5BBB16B024044030120CDCCCC3DCB
:1022D000345F012038B50D46FFF762FC044628B193
:1022E0000B48C378DB0703D580882880204638BD9B
:1022F000084A183010F9173C92F8202093FBF2F1AD
:1023000002FB1132013101320EF030F8EDE700BF6F
:1023100044030120185C012038B5134C94F8253093
:1023200094F824209A4219D004EBC3030F49D3E94F
:102330000A200023984212DC93780D4A5B08C4F807
:102340002C031370FDF720F994F825300621013392
:10235000B3FBF1F201FB123384F8253038BDD55CB4
:10236000013301F8015BE5E7185C012014590120F5
:1023700042590120A84B1B782DE9F04F81468BB0C4
:10238000002B40F0B180A54DD5F83063002E00F051
:10239000AB80A34AD46904F0F021B1F1E02F6CD1F5
:1023A000D361D5F83423944267D004930DF110081B
:1023B000C8F80430A8F80830B5F8EC3295F8E8E22F
:1023C000ADF8143095F8E9C295F8F03295F8EAA224
:1023D0008DF8183007AB8DF810E08DF811C08DF82E
:1023E00012A0904FC5F8344398E8070003C31A8041
:1023F000C4F34253C4F303423B440132597C8E453B
:1024000001D1944508D030468DF81C108DF81D2060
:102410000DF0ACFFADF82000304604F0070B0EF0D5
:102420002FFB032834D0042835D000239A4501A976
:10243000304618BF8DF81E300EF012F848B1019BDF
:10244000C4F3001103F001038B4202D030460EF0BA
:1024500009FA0A2207A940464BF0EEFD68B19DF843
:102460001E30BDF81C2085F8EA32BDF82030A5F8F2
:10247000E822A5F8EC323AF025FD95F838A304AF30
:1024800095F83833032B79D8DFE803F0083174A1CD
:102490005F44BB7DCAE75F44BB7FC7E73946304630
:1024A0000DF0E4FF044658B107A8FFF77FFE9DF842
:1024B0001E109DF810308B4260D030460EF048FA66
:1024C00095F83833013303F0030385F838330CB93A
:1024D0009A45D5D195F8F232DB0700D524B133689F
:1024E000494630461B6898470BB0BDE8F08F01A8FD
:1024F000FFF75CFE95F8F2829DF8044008F00108B1
:10250000ECB1B8F1000F39D13A460DF10301304674
:102510000EF016F8044688B307A8FFF747FE9DF8AB
:102520001C109DF803309DF81D208B4203D19DF8AF
:102530001030934222D030460EF014FAC0E7B8F1C2
:10254000000FBDD1394630460DF08DFF0446A8B1CD
:1025500007A8FFF72BFEBDF82010BDF810308B4206
:102560000CD085F83983304685F83A8333689B6907
:102570009847A5E795F8F232D80701D500249FE7E0
:1025800007A930460DF06CFF04460028F6D01E2047
:102590001CF0C8FF95F83B3380468342EED085F8A7
:1025A0003B0360B1B5F8EE32002BE7D1079BD907AA
:1025B000E4D40121304644460EF054F980E7079BED
:1025C000DA07DBD5014630460EF04CF978E738469D
:1025D000FFF7ECFD07AB97E8070003C31A809DF8EF
:1025E00010309BB10DF11D0207A930460DF0A8FF78
:1025F0000DF11E0130460DF039FF0A2207A93846B9
:102600004BF01AFD041E18BF012459E708A93046F3
:102610000DF029FFECE700BF54590120185C0120A0
:102620004403012024EE0508024B0146D3F83C0385
:1026300031F03EBD185C0120FD292DE9F041044632
:1026400084B000F0D980F02900F0BD80EF2900F0BF
:102650002B814AB10346861803AD002003F8010B15
:10266000B34205F8010BF9D19A4B0B2003F1090590
:1026700001E013F8010F814200F0C380AB42F8D1B2
:102680004B1E832B00F29380DFE813F01D01320113
:102690003C014701B401840051015C0168019100D3
:1026A00091006E016E016E01840184018401680154
:1026B000910091008E01960191009100910091008E
:1026C0009100910091009100910091009100910082
:1026D0009100910091009100910091009100910072
:1026E0009100910091009100910091009100910062
:1026F0009100910091009100910091009100910052
:10270000910091009100910091009100AA01910027
:102710009100910091009100910091009100910031
:102720009100910091009100910091009100910021
:102730009100910091009100910091009100910011
:102740009100910091009100910091009100910001
:1027500091009100910091009100910091009100F1
:1027600091009100910091009100910091009100E1
:1027700091009100910091009100910091009100D1
:1027800091009100910091009100910091009100C1
:1027900019011901504BB3F89013002900F05C8126
:1027A000019228F0E3F9019A80B2ADF80C003AB139
:1027B00003AB224413F8011B04F8011BA242F9D118
:1027C00004B0BDE8F08103214FF00508434FB84441
:1027D0000025013701E017F8011B0846FFF7D8FB79
:1027E000064660193246FFF727FF7019B845C5B293
:1027F000F1D104B0BDE8F0810B214FF00408384F4F
:10280000E5E7354BD3F8000180060CD4002AD7D079
:1028100003AB224413F8011B04F8011B9442F9D1C5
:1028200004B0BDE8F08193F84003870741D52D4DF2
:10283000287D052834BF02260326142916D97C39A1
:10284000C8B20628E2D80629E0D801A050F821F045
:10285000432A0108432A01082D2A01080D280108EE
:10286000192A0108132A01081F2A01080929CDD9AC
:102870000A390A29CAD801A757F821F0012A010804
:102880004D2A01080D2801080D2801080D2801080E
:102890000D2801080D2801080D2801080D28010840
:1028A000252A0108432A01080C214FF006080E4F83
:1028B0008DE70C4B0B29187DA8D10126C7E00B4BE7
:1028C0009B6B039373E70192FFF73CFB019AADF812
:1028D0000C006CE74CEE0508185C012030EE050892
:1028E0002CEE05081058012024EE0508404F012069
:1028F0006A4BD3EDE07AFDEEE77A17EE903AADF849
:102900000C3054E7654B93F85703B3F84413002891
:1029100040F0AA80ADF80C1049E76049B1F84433A3
:1029200091F87013B3FBF1F3ADF80C303FE75B4D5A
:1029300095F8F232DE0700F19C80B5F89033ADF8DF
:102940000C3034E7564B5749B3F9043081FB03018F
:10295000DB17C3EBA103ADF80C3028E74F4BB3F8FE
:10296000AC33ADF80C3022E70C394F4B9FED4F7A6A
:10297000C9B2D3ED007A03EB810367EE877A93ED5A
:10298000157A67EE877AFDEEE77A17EE903AADF8A2
:102990000C300CE70F39424B33F8113003EB830353
:1029A0005B00ADF80C3002E73C4B93F8F23203F0D9
:1029B0000103ADF80C30FAE63D4B1988CD0551D432
:1029C000CB4303F0010311F0440F18BF042311F0AF
:1029D000020F18BF072311F4806F18BF0923AEE759
:1029E0000192FFF7AFFA334B019A1B6C43EAC040E8
:1029F0000390DCE6294BD3F8A033ADF80C30D6E6D3
:102A00002B8A03EB830303EB83039B00ADF80C30AD
:102A1000FCE66B680393F9E62B680393F6E6AB6874
:102A20000393F3E6EB89ADF80C30EFE6EB8922492E
:102A300003EBC3039B00A1FB03135B09ADF80C3050
:102A4000E4E6B3F84233ADF80C30DFE6F6B28DF8C9
:102A50000C608DF80D00D9E6D3F8A80380F31000C0
:102A600080B2A2E60323AEE793F87033B1FBF3F133
:102A700050E701921FF0FCFED5EDE07A019AFCEEE2
:102A8000E77A17EE903A9BB200287FF458AF0B49D3
:102A9000096811F0100F18BF002350E7185C0120DF
:102AA0009C580120676666665411002000007A4435
:102AB000C0580120404F01201F85EB5130570120A5
:102AC000F8B5224C94F8AE13621892F8B023002A9D
:102AD0003AD000231E4D4A1C0133A5FB0261490870
:102AE00001EBC101511A621892F8B0230AB1092B07
:102AF000F1D1CBB284F8AE3302680C260025571C06
:102B0000076001EB41071670026801EB8701561C54
:102B1000066015700D2205680E4E6F1C314407606B
:102B20002B7040F0F1FE94F8AE130120084B0A1808
:102B30002144A3FB025381F8B003C34003EBC3035A
:102B4000D31A84F8AE33F8BD0B46D5E7185C0120E4
:102B5000398EE338D45F01202DE9F041694D84B00E
:102B600004460E46D5F8307338460DF089FF85F8D7
:102B7000310457B10DF1090202A938460DF0E0FC0D
:102B8000002840F08E8095F8310400231946ADF8F6
:102B900008308DF80A30431E0022FF208DF80C10FB
:102BA000DBB2ADF80E208DF80B00FD2B04D900230D
:102BB000184604B0BDE8F0819DF80830042B00F001
:102BC0009580052B00F09880032B00F09780022B56
:102BD00000F08B80012B00F093809DF809300DF1FF
:102BE0000E029DF80A10013BD5F830038DF809302C
:102BF0000DF0A8FB95F83134032B74D0042B0CD1C5
:102C0000414A9DF80A000121002301E012F8011F4A
:102C100081426ED20133082BF8D1D5F834240DF15E
:102C20000808029B394F9A4250D023680D21002298
:102C3000581C2060204619702368591C21601A70A6
:102C400023689DF80820591C21601A7023689DF89C
:102C50000920591C21601A7023689DF80C20591C0A
:102C600021601A7023689DF80A20591C21601A708F
:102C7000BDF80E1040F08CFE23689DF80B20204616
:102C8000591C216007211A70FAF7ACFB0123C5F823
:102C90003C6498E8030087E80300184604B0BDE8E8
:102CA000F08101A938460DF0DBFB00283FF46BAF43
:102CB00038460DF10A010DF0D9FB00283FF463AF4F
:102CC000019995F8310401F0010164E77A68D8F8B8
:102CD00004309A42A9D1D5F83C340D4AF31A9342F4
:102CE0007FF665AFA1E70B4A8BE703228DF808203A
:102CF00073E78DF80A3090E70122F7E70222F5E743
:102D00000422F3E7185C012042EE05084C60012024
:102D100080841E003AEE0508F0B52B4D0E462B4A76
:102D200083B0D5F8A033B5F840C482FB0312DC179A
:102D3000B5F8A873C4EBA204A4B2A4450CD1D5F88D
:102D400044342349F31AB5F848248B4298BFBA4259
:102D500014BF0123002334D00368342100220190E2
:102D600003F1010CC0F800C019702146036803F19B
:102D7000010CC0F800C01A7040F00AFE39460198F4
:102D800040F006FE47F6FF71019840F001FE47F65D
:102D9000FF71019840F0FCFD47F6FF71019840F08B
:102DA000F7FD47F6FF71019840F0F2FD019802210E
:102DB000FAF718FB0123A5F84044A5F84874C5F8B4
:102DC0004464184603B0F0BD185C0120676666666F
:102DD00080841E0002680E2170B5561C7F250024D9
:102DE000066015700268551C05601470FAF7FAFA4F
:102DF000012070BDC74B1B682DE9F04F814613F0D1
:102E0000800083B000F07981C34B93F8400310F049
:102E1000020000F07281DFF820A39AF81430052B2D
:102E200040F27281DAF80030BC4C002B0093BC48B1
:102E3000B8BF5B42BB49A4FB0352920D00FB0233B7
:102E400002EB8202C3EB031302EB82029B0084FBC2
:102E50000354DD17C5EBA45500FB053305EB8205D4
:102E600081FB0321ADB2DB17C3EBA111C5B100207B
:102E7000AD4F0446A7FB053CC3B22E4601304FEAD6
:102E8000DC0C9A00092E0CEB8C03A5EB43031FFA14
:102E90008CF59BB203FA02F344EA0304EAD8250452
:102EA00089B2C1B10020A04F0446A7FB013CC3B2C8
:102EB0000E4601304FEADC0C9A00092E0CEB8C0315
:102EC000A1EB43031FFA8CF19BB203FA02F344EA2D
:102ED0000304EAD82543DAF804B0904C8BEAEB738C
:102EE0008F48904AA3EBEB73A4FB0361890D00FBB1
:102EF000013301EB8101C3EB031301EB81019B0063
:102F000084FB0364DE17C6EBA45600FB063306EB16
:102F1000810682FB0312B6B2DB17C3EBA212CEB15D
:102F20000021814F0846A7FB063ECBB23446013153
:102F30004FEADE0E4FEA830C092C0EEB8E03A6EB54
:102F400043031FFA8EF69BB203FA0CF340EA030028
:102F5000E9D8060492B2CAB10021734F0846A7FB14
:102F6000023ECBB2144601314FEADE0E4FEA830C2B
:102F7000092C0EEB8E03A2EB43031FFA8EF29BB2D9
:102F800003FA0CF340EA0300E9D80643DAF8083004
:102F9000654A002B18460193B8BF5842634C6449F8
:102FA000A2FB0030030AA4FB0343DB0901FB03F18E
:102FB000C1EBD00189B2C1B1002496462746AEFBD1
:102FC000013CE3B20A4601344FEADC0C9800092ABE
:102FD0000CEB8C03A1EB43031FFA8CF19BB203FAB9
:102FE00000F347EA0307EAD8B9B2BAF81080B8F19B
:102FF000000F1AD00024DFF830E12746AEFB083C72
:10300000E3B2424601344FEADC0C9800092A0CEB8B
:103010008C03A8EB43031FFA8CF89BB203FA00F36E
:1030200047EA0307EAD81FFA87F8BAF812303E4A8F
:10303000A2FB0307FF08632F28BF6327092B67D96B
:103040004FF0000C92466046AAFB073E5FFA8CF3F5
:103050003A460CF1010C4FEADE0E9C00092A0EEBF9
:103060008E03A7EB43031FFA8EF79BB203FA04F318
:1030700040EA0300E8D8C4B2009B019A002BCCBF01
:1030800039233823BBF1000F4FEA226738DD27F0E0
:103090007F07284A3B43934543F00207C8BF43F0EC
:1030A0000607D9F800301620002203F1010CC9F8F8
:1030B00000C018704846D9F8003003F1010CC9F877
:1030C00000C01A7040F064FC2946484640F04AFCB3
:1030D0003146484640F046FC4846414640F058FCE0
:1030E000D9F8003001201A18C9F800201C70D9F84E
:1030F00000301A18C9F800201F7003B0BDE8F08F27
:1031000027F07F071F43CCE7002003B0BDE8F08F16
:103110000024B1E730570120185C01206BCA5F6BB7
:10312000806967FFD34D6210CDCCCCCCC55A7C0AE8
:10313000A0860100FFC99A3B10580120AE4B1B68C6
:103140002DE9F047064613F0800084B000F0A2801D
:10315000AA4B93F8400310F0020000F09B80DFF8C8
:10316000B4E29EF81410052940F29980632900F218
:103170009480002089B2A24F0446A7FB013CC3B251
:103180000D4601304FEADC0C9A00092D0CEB8C0344
:10319000A1EB43031FFA8CF19BB203FA02F344EA5A
:1031A0000304EAD8E4B2DEF80830964AD91782FB65
:1031B0000323C1EB633399B2002900F01981002584
:1031C000DFF83CC22846ACFB0138EBB20F460135B4
:1031D0004FEAD8089A00092F08EB8803A1EB4303B4
:1031E0001FFA88F19BB203FA02F340EA0300EAD81F
:1031F000C7B2BEF80E304FF4F365834942F20F7048
:1032000005FB03F5A1FB0535C5F38F1585424AD8AB
:10321000D5B10021DFF8E8E10846AEFB0538CBB2B6
:10322000AC4601314FEAD8089A00BCF1090F08EB0F
:103230008803A5EB43031FFA88F59BB203FA02F358
:1032400040EA0300E9D885B2704BD3E90023134369
:103250003ED14FF0FF3833682946172000225D1C0D
:1032600035601870304633685D1C35601A7040F068
:103270008FFB4146304640F075FB336830460621EF
:103280005A1C32601C7033685A1C32601F70FAF787
:10329000A9F8012004B0BDE8F087992483E7002055
:1032A00004B0BDE8F0870021DFF854C10D46ACFB47
:1032B0000032D20802EB8203A0EB430390B29BB230
:1032C0008B400431102945EA0305F0D1ADB2BBE7CC
:1032D00001A839F0CDFE9DF80810002900F08A8081
:1032E0000020DFF81CE18046AEFB0139C3B28C46FA
:1032F00001304FEAD9099A00BCF1090F09EB8903A3
:10330000A1EB43031FFA89F19BB203FA02F348EAE7
:103310000308E9D84FEA08289DF80920E2B1002106
:10332000DFF8DCE00846AEFB023ACBB2944601314E
:103330004FEADA0A4FEA8309BCF1090F0AEB8A0364
:10334000A2EB43031FFA8AF29BB203FA09F340EAA5
:103350000300E8D848EA00089DF80A204FEA082848
:10336000E2B10021DFF898E00846AEFB023ACBB2AA
:10337000944601314FEADA0A4FEA8309BCF1090F9A
:103380000AEB8A03A2EB43031FFA8AF29BB203FA09
:1033900009F340EA0300E8D848EA0008BDF80C3019
:1033A0004FEA08181A4A632BA2FB03124FEA521283
:1033B0007FF651AF0021DFF848E00846AEFB023A45
:1033C000CBB2944601314FEADA0A4FEA8309BCF1E5
:1033D000090F0AEB8A03A2EB43031FFA8AF29BB29E
:1033E00003FA09F340EA0300E8D848EA000832E7A4
:1033F0000F46FEE688468FE730570120185C012013
:10340000CDCCCCCC89B5F814D34D621068600120C6
:103410001F85EB511058012008B5A0F101030228C7
:10342000B3FA83F34FEA531301D0184608BD0F20B7
:103430001FF03AF930B9064B93F8F23203F001036A
:10344000184608BD0F20BDE808401CF06BB800BF4F
:10345000185C0120B1F5805FF0B400F0D4802AD868
:10346000102900F0F580B1F5807F4ED1046A16690D
:1034700024F4807457689A4B0462016A446821F40A
:103480000071C56941EA0621964E2B40156821F46A
:103490008071B04245EA030541EA072173D0924B9F
:1034A000984270D0D26800234460C561C263016253
:1034B0001846F0BC7047B1F5803F00F08180B1F54F
:1034C000801F48D1046A156924F480145668874B1C
:1034D0000462016A446D21F400112340146841EA3A
:1034E0000551804D43EA042421F48011A84241EAA9
:1034F00006515DD07C4B98425AD0D2680023446577
:10350000C26501621846F0BC7047012923D1046AE4
:10351000166924F001045768714B0462016A44681B
:1035200021F00201856931436E4E2B40156821F070
:103530000101B04245EA030541EA07010FD06A4B99
:1035400098420CD0D26800234460856142630162D6
:103550001846F0BC70470123F0BC18467047D2E90A
:10356000056321F0080124F4807441EA86011C43BC
:103570009668D36921F0040124F4007441EA8601BD
:1035800044EA4304DEE7D2E9056321F4006124F450
:10359000805441EA8621966844EA0314D36921F4F1
:1035A000806124F4005441EA862144EA431479E717
:1035B0004368956923F4802343EA852343609CE7AD
:1035C000046A156924F480345668494B0462016A20
:1035D000446D21F400312340146841EA0541414D16
:1035E0001C4321F48031A84241EA064155D03E4BAC
:1035F000984252D0D26800234465846D826501628E
:103600001846F0BC7047046A166924F48054576861
:10361000384B0462016A456821F40051C46941EAEB
:103620000631304E2340146821F48051B04243EA01
:10363000042441EA073138D02B4B984235D0D26868
:1036400000234560C461026401621846F0BC704703
:10365000046A166924F010045768264B0462016A54
:10366000446821F02001856941EA06111D4E2B4076
:10367000156821F01001B04243EA052541EA07111F
:1036800019D0194B984216D0D26800234460856146
:10369000826301621846F0BC70474368956923F461
:1036A000803343EA05234360A4E725F4804593690A
:1036B00045EA8315C3E7D2E9056321F0800124F4CC
:1036C000806441EA8611966844EA8304D36921F054
:1036D000400124F4006441EA861144EAC304D3E7BC
:1036E0008CFFFEFF0000014000040140FF8FFFFE41
:1036F0008FFFFEFFFF8CFFFE70B4344CB0F1804FA3
:103700000368A0EB0404B4FA84F44FEA541406D01E
:103710002CB92F4D2F4A904218BFA8421DD12E4AD6
:1037200023F070034D68821A2B43B2FA82F25209D9
:1037300023F44073D1E902652B430D880360C66210
:1037400085623CB932B9436943F0010370BC4361FF
:10375000002070470B7C0363F5E702F5806290421E
:1037600020D002F5784290421CD01C4A1C4DA84241
:1037700018BF90420CBF0122002224D0194EA5F59B
:103780009635A84218BFB042D2D0174A90421AD0FC
:1037900002F58062904216D08C680A880360C46289
:1037A0008262D0E70C4A23F07003104D821A4E68F3
:1037B000A842B2FA82F243EA06034FEA5212B7D0A5
:1037C000002AB5D1D1E70022B2E700BF00000140D6
:1037D0000004004000080040000401400040014097
:1037E0000044014000480140001C0040000C004023
:1037F0001F4BF0B4595C0446D2E9023645181069F3
:10380000334356696758034390693343D66903438A
:10381000906A3343174E03433E40D06A33436350AC
:1038200090B16E69176B26F00706536B3843976BA0
:1038300030436861605820F0C0701843605063588E
:1038400023F4C0033B436350566800201368EE60C6
:10385000AB60094E6B681E40D2E908321E436E60B1
:10386000635823F0F05313436350F0BC704700BF1C
:103870005CEF05081F80FCFF0000FFFF30B4614CC7
:103880000346614A655C0C1E18BF0124821A405928
:1038900018BF012220F00100585192B98CB95B4A3F
:1038A00000212120116051609160D160116150614F
:1038B0005A5922F0F0525A513F2200209A6030BCEF
:1038C00070475348181A18BF012014B908B9514A53
:1038D000E6E74C1E18BF01241ABB14BB4E4A002059
:1038E0002124106050609060D060106154615A597A
:1038F00022F0F0525A5101290DD0022915D0032986
:1039000024D0042927D0052914D006292BD0072933
:1039100035D00120D3E74FF47462002030BC9A60A8
:10392000704760B95CB93D4AD9E74FF47C1200207A
:103930009A60C4E74FF474620020DA60BFE78C1E1F
:1039400018BF01245AB954B9354AC8E74FF0746218
:1039500000209A60B3E73F220020DA60AFE738B971
:1039600034B9304ABBE74FF47C120020DA60A6E796
:10397000CC1E18BF01243AB934B92B4AAFE74FF037
:1039800074620020DA609AE710B90CB9274AA6E7FA
:103990000C1F18BF012412B90CB9254A9FE710B9B2
:1039A0000CB9244A9BE74C1F18BF012412B90CB96B
:1039B000214A94E710B90CB9204A90E78C1F18BF30
:1039C000012412B90CB91E4A89E710B90CB91D4A75
:1039D00085E70D4A934203D1072901D11A4A7EE7B0
:1039E0001A4A00202124106050609060D06010615D
:1039F00054615A5922F0F0525A5100297FF47BAF9A
:103A00005AE700BF5CEF050800600240106002400A
:103A100000640240106402402860024028640240B2
:103A200040600240406402405860024058640240D6
:103A30007060024070640240886002408864024006
:103A4000A0600240A0640240B8600240B864024036
:103A500030B40023154C0168C36725680B681B0749
:103A600009D4002220231446436780F8702083671E
:103A7000204630BC7047CB6913F40013F1D12268A3
:103A8000521BB2F1007FF6D30A682025032422F4EA
:103A9000D0720A608A6822F001028A60456780F865
:103AA00070308567204630BC704700BFE834012085
:103AB000436ADA0710B406D50168846A4A6822F4BA
:103AC000003222434A609C0706D50168C46A4A68EE
:103AD00022F4803222434A60590706D50168046BFC
:103AE0004A6822F4802222434A601A0706D50168F8
:103AF000446B4A6822F4004222434A60DC0606D541
:103B00000168846B8A6822F4805222438A60990695
:103B100006D50168C46B8A6822F4005222438A6089
:103B20005A060AD50168046C4A68B4F5801F22F46D
:103B3000801242EA04024A600BD01B0606D50268D6
:103B4000816C536823F400230B4353605DF8044BEE
:103B500070474A68446C22F4C00222434A60ECE792
:103B60000368042201F01F01186A02FA01F120EA39
:103B7000010010B418621A6A0A4C114319625A6C97
:103B800042F400425A649A681440062C06D0B4F5F8
:103B9000803F03D01A6842F001021A6000205DF8ED
:103BA000044B70470700010001F01F01036A10B4C5
:103BB00001248A408C4023EA04035DF8044B03622D
:103BC000016A0A4302627047034690F83C000128EC
:103BD00000F0C6800220F0B4012483F83D0083F891
:103BE0003C40002A31D0042A73D0082A1A6800F019
:103BF0009580166AC86826F480560D684F688C68F0
:103C0000010316622D03D06989B2166A05F42045B6
:103C100020F4407026F4204640EA0720354320F483
:103C200070400143D1611562D06920F44060D061D9
:103C3000D16941EA0421D16100220121104683F8B3
:103C40003D1083F83C20F0BC70471A68DFF814C1BF
:103C5000166A62450C6826F001064D68C86816624F
:103C60009769166A1DD0B2F1804F1AD0ACF57C4C22
:103C7000624516D00CF5806C624512D00CF5806C54
:103C800062450ED00CF5784C62450AD00CF5705C9C
:103C9000624506D0ACF5943C624502D047F0010580
:103CA00002E027F003073D43000125F0F00526F070
:103CB0000A0604F00A04C0B28F68344328439061B6
:103CC0001462906920F00C00906191693943916110
:103CD000B2E71A68C868166A0D6826F010064F68C1
:103CE0008C68010316622D01906989B2166A05F08D
:103CF000A00520F4407026F0A00640EA07203543D6
:103D000020F47040014391611562906920F4406095
:103D10009061916941EA042191618DE7176AC86851
:103D200027F480770E684C688D68010117623602AF
:103D3000D069C9B2176A06F4206620F0030027F4A0
:103D4000206720433E4320F0F0000143D16116621A
:103D5000D06920F00C00D061D1692943D1616BE7B3
:103D600002207047000001400368012201F01F019A
:103D7000186A02FA01F120EA010010B418620F4C2F
:103D80001A6AA34241EA0201196212D00C4A934214
:103D90000FD099680B4A0A40062A06D0B2F5803F38
:103DA00003D01A6842F001021A6000205DF8044B4B
:103DB00070475A6C42F400425A64EAE7000001403E
:103DC0000004014007000100F0B490F83D30002BE2
:103DD00066D0026802233B49B2F1804F80F83D3043
:103DE000A2EB01011368B1FA81F14FEA51113BD006
:103DF000002939D1344D354CA24218BFAA4233D0E4
:103E0000334F05F50065D71BAA42B7FA87F74FEA8B
:103E100057174AD0002F48D12E4F2F4CA24218BF1F
:103E2000BA420CBF012700274AD02C4DA4F5963486
:103E3000A24218BFAA4220D004F58064A2423FD01B
:103E400004F58064A2423BD0816923F08003C468FA
:103E50000B4341681360D46291620123536180F87F
:103E60003D300020F0BC7047194F23F07003856887
:103E7000D71B2B43B7FA87F77F09046923F44073F4
:103E800085692343C668446823F080032B4313608D
:103E9000D662946209B9002FDFD043691363DCE76F
:103EA00003F0FF0280F83C2093E70D4C23F07003F1
:103EB0008568A24243EA0503DFD0002FDDD1ABE7DE
:103EC0000027DAE70000014000040040000800403D
:103ED000000401400040014000440140004801400E
:103EE000000C004003682DE9F04F13F0010785B086
:103EF00000F0F080C44A13F40025916821F4000119
:103F00009160C46A9168B4FA84FE41EA04014FEA00
:103F10005E1E916000F0E380BB49446BD1F88C20B9
:103F2000B4F5801F22F4401242EA0402C1F88C204A
:103F300000F0B681B4FA84F413F480124FEA5414FA
:103F4000019240F0D280990600F1E480DE060CD5A3
:103F5000AD49D1F88C2022F08072C1F88C20D1F8C4
:103F60008C20066B3243C1F88C20590408D5A64931
:103F7000C66DD1F8902022F440323243C1F890202F
:103F80001A0408D5A049066ED1F8902022F44022E8
:103F90003243C1F89020DE0308D59B49466ED1F824
:103FA000902022F440123243C1F89020590608D5DF
:103FB0009549C66BD1F8902022F003023243C1F834
:103FC00090201A0608D59049066CD1F8902022F06E
:103FD0000C023243C1F89020DE0508D58A49466CB0
:103FE000D1F8902022F030023243C1F89020990598
:103FF00008D58549866CD1F8902022F0C002324362
:10400000C1F890205A0508D57F49C66CD1F8902098
:1040100022F440723243C1F890201E0508D57A4937
:10402000066DD1F8902022F440623243C1F890200E
:10403000D90408D57449466DD1F8902022F4405235
:104040003243C1F890209A0408D56F49866DD1F8A3
:10405000902022F440423243C1F8902013F4001C17
:104060000ED06949D0F87480D1F89020B8F1006F73
:1040700022F0006208BF012442EA0802C1F8902041
:104080005E0309D5DFF88081C26ED8F8901021F068
:1040900040710A43C8F89020190209D5DFF86881F9
:1040A000826FD8F8901021F080510A43C8F8902010
:1040B0005A0100F18E80B3F1007F00F09980BEF1CB
:1040C000000F40F09580012C00F0F180002005B039
:1040D000BDE8F08F13F40025BE467FF41DAF2C46DB
:1040E00013F4801201923FF42EAFDFF81CC1816BF4
:1040F000DCF88C20B1F5800F22F4400242EA010284
:10410000CCF88C2000F0D080002908BF012499064B
:104110007FF51CAFDFF8F0803C4AD8F840903C496E
:10412000944649F08059C8F84090D8F8408008F08B
:104130008058CDF80C80DDF80C80D2F8008048F46F
:104140008078C2F80080D1F8008005E00A68A2EB10
:104150000802642A00F2A080DCF80020D205F5D520
:10416000DFF8A480D8F8702012F4407C826A02F450
:10417000407919D0E14517D0D8F870C0D8F870A0B0
:104180002CF4407C4AF4803AC8F870A0D8F870A0AB
:104190002AF4803AC8F870A0C8F870C0D8F870C087
:1041A0001CF0010F40F00581B9F5407F00F0EE8072
:1041B000DFF854C0DCF8081021F4F811CCF808102E
:1041C0001149C2F30B02D1F870C042EA0C020A672F
:1041D000BCE6DFF83480B3F1007FC26FD8F89010EE
:1041E00021F0005142EA0102C8F890207FF467AF45
:1041F000054A0749D2F80080964628F08068C2F840
:104200000080D1F800800AE00038024000700040D1
:10421000E83401200A68A2EB0802642A3CD8DEF8E0
:1042200000201601F6D46FB1C26A5AB98268DEF86E
:1042300084704668120707F0706742EA86123A43B4
:10424000CEF88420002D40F08380019A22B1826B49
:10425000B2F5800F00F081809A010AD5C3684268E8
:104260001B06876843EA82135B4A43EA0773C2F876
:104270008430594B1F681A4647F080671F600F68EB
:1042800003E00B68DB1B642B06D813681B01F8D511
:10429000012C7FF41BAF0AE0032005B0BDE8F08FCE
:1042A00000244FF0010E1BE74FF0010E4BE64A4B86
:1042B0004A491C681A4624F080541C600C6803E0CC
:1042C0000B681B1B642BE7D813689E00F8D4002DE5
:1042D0006BD1019BC3B1836BB3B93F4A4369D2F839
:1042E000884005691B0604F4403443EA85132343E0
:1042F000C2F88830D2F88C30046A23F4F853013CB9
:1043000043EA0423C2F88C30BCF1000F10D0436F95
:10431000B3F1006F0CD183692F4C00691B04D4F8F2
:10432000882043EA801302F070621343C4F8883097
:10433000294B18681A4640F080501860086803E05E
:104340000B681B1A642BA7D813689B00F8D5BDE631
:10435000426BB2F5801F7FF478AFDFF87CE0C26873
:10436000DEF884704668120607F0E04842EA8612DA
:1043700042EA0802CEF88420DEF88C70C26927F089
:104380001F07013A3A43CEF88C2065E7DFF84880F2
:10439000DFF84CC0D8F8081002EA0C0C21F4F81130
:1043A00041EA0C01C8F808100AE7436B002B94D0CF
:1043B0008FE7D1F800B041F2883A06E0D1F800C0AA
:1043C000ACEB0B0CD4453FF667AFD8F870C01CF0CF
:1043D000020FF3D0E8E600BF00380240E8340120C5
:1043E000FFFCFF0F054A064B92680649C2F3822282
:1043F0000868134493F83430D840704700380240BE
:1044000024EE0508542C0120164908B58B6803F0EA
:104410000C03042B1BD0082B17D14A684B6802F001
:104420003F02496813F4800313D10F48C1F3881188
:10443000A1FB000146F0E8F90A4B5B68C3F30143B6
:1044400001335B00B0FBF3F008BD074808BD074827
:1044500008BD0648C1F388110023A1FB000146F006
:10446000D3F9E9E7003802400024F40000127A0092
:10447000F8B504468368B849E669E768B74DD0E9FE
:1044800004201A43236802431868AB4201EA000182
:1044900042EA060242EA0102A1691A605868226AE9
:1044A00020F4405042EA010240EA0700586099684F
:1044B00021F4306142EA01029A605FD0A84A934237
:1044C0001CD0A84A934200F00881A74A934200F00A
:1044D0001281A64A934200F08B80A54A934200F0D5
:1044E000A380A44A934200F05381A34A934200F070
:1044F000208100230120C4E91833F8BD9F4BA04A56
:10450000D3F8903003F00C03134493F84030B6F521
:10451000004F17D0082BECD801A151F823F000BFB1
:1045200059460108994501083F460108F34401082E
:1045300013460108F3440108F3440108F344010859
:10454000C9450108082B06D8DFE803F0BBA79E0584
:1045500092050505890001200023A3F110014FF603
:10456000EF729142C5D823F00F02C3F342032168D2
:104570001343CB600023C4E91833F8BD7F4B804A56
:10458000D3F8903003F00303013B022B40F29C80F0
:10459000B6F5004F00F0818078497A4B89681B6836
:1045A000C1F3423160680A4492F83420D34003EBEF
:1045B0005003B3FBF0F39BB2A3F110020DE0302BDC
:1045C00097D1B6F5004F4AD06268530803F500430F
:1045D000B3FBF2F39BB2A3F110024FF6EF718A42E4
:1045E00087D822680020D3600023C4E91833F8BDBF
:1045F000624BD3F8903003F44073B3F5007F1BD0C7
:1046000066D833B3B3F5807F7FF473AFB6F5004F50
:104610002ED0FFF7F9FE636800EB5300B0FBF3F315
:104620009BB2A3F11002D8E7544BD3F8903003F4B7
:104630004063B3F5006F70D1B6F5004F24D06268C7
:10464000514B03EB5203B3FBF2F39BB2A3F1100205
:10465000C3E7B6F5004F34D0FFF7C4FEDBE762686E
:104660000020530803F58033B3FBF2F39BB274E7E9
:10467000FFF7CAFE6168034600204A0802EB4303C5
:10468000B3FBF1F39BB268E7626800203F4B03EB9A
:104690005203B3FBF2F39BB25FE738490020394B7A
:1046A00089681D68C1F3423166680A44730892F84C
:1046B000342025FA02F203EB4203B3FBF6F39BB27C
:1046C0004BE7FFF78FFED5E7134493F83C301EE726
:1046D000B3F5407F3FF475AF0BE7284BD3F890302C
:1046E00003F03003202BA7D03FF669AF002BB0D0EA
:1046F000102B8BD0FDE6214BD3F8903003F0C00394
:10470000802B99D005D8002BA3D0402B3FF47EAF4F
:10471000EFE6C02B3FF455AFEBE605D8D3B1B3F5C8
:10472000806F3FF473AFE4E6B3F5406F3FF449AFF9
:10473000DFE6124BD3F8903003F44043B3F5004F5B
:104740003FF47AAF3BD8002B83D0B3F5804F3FF4D2
:104750005DAFCEE60A4A1BE7F369FFEF00100140A8
:104760000044004000480040004C00400050004021
:104770000014014000780040007C004000380240F6
:1047800024EE0508542C01200024F4000048E80120
:104790000D4BD3F8903003F44053B3F5005F3FF472
:1047A0004BAF07D8002B3FF454AFB3F5805F3FF415
:1047B0002DAF9EE6B3F5405F3FF403AF99E6B3F546
:1047C000404F3FF4FEAE94E60038024090F8BC3310
:1047D000012B29D0012380F8BC330B060ED40268CC
:1047E0001021124B116101E0013B02D01169C90691
:1047F000FAD4002380F8BC331846704701F00F014B
:104800000A4B890110B441F020010468216101E0E4
:10481000013B02D022699206FAD4002380F8BC330F
:1048200018465DF8044B704702207047400D0300A6
:10483000F8B501F00F05012600271C21C5EBC504C2
:1048400001FB050100EB84043C31A264236584F87C
:104850003C50676584F83D600369B34208BFE26479
:10486000DAB200681DB9FAF7C7FF0020F8BDFBF700
:104870004FF80020F8BD00BF11F0800F4FF01C036F
:1048800001F00F0170B432D103FB0103C1EBC1028F
:10489000002400EB820203F5FE7382F8FD411970DB
:1048A00090F8BC23012A31D00121026880F8BC13A2
:1048B0005C781D7802F500638C422AD005F00F0465
:1048C000DE6B02F53062A1401C4C02EB451226EA79
:1048D0000146DE63DD6925EA0141D96113681C40A8
:1048E0001460002380F8BC33184670BC704703FB8B
:1048F0000103C1EBC102012400EB82023C3382F8C8
:104900003D40197090F8BC23012ACDD1022070BC23
:10491000704705F00F01DE6B02F510628C4008490C
:1049200002EB451226EA0406DE63DD6925EA04048B
:10493000DC61136819401160D3E700BF0078F3EF22
:10494000007833EC70B41D4E056803E03468A41A97
:10495000A14226D3AB6913F02003F7D01022202305
:10496000EA61EB61AB699A0701D50023AB62AB69E1
:10497000DB0703D4AB6943F00103AB616B68002232
:104980000F4C202123406B60436C80F8402043F0A3
:104990000403436480F8411080F84220012070BC79
:1049A0007047426C202180F840300A43426480F80E
:1049B000411080F84230012070BC7047E83401207B
:1049C00000E800FE2DE9F041DFF8548004460E4671
:1049D00015460AE09B69DB0602D5FFF7B3FFE0B995
:1049E000D8F800305B1BB34209D823682A46314609
:1049F00020469F69BF07EDD50020BDE8F081636CBC
:104A00002021002201200B4384F84020636484F8B5
:104A1000411084F84220BDE8F0810120BDE8F0811A
:104A2000E8340120F0B484460568049F104E03E08A
:104A30003468E41B9C420AD8AC6931EA04000CBF1C
:104A4000012400249442F3D00020F0BC7047DCF82D
:104A500044302021002201200B438CF84020CCF868
:104A600044308CF841108CF84220F0BC704700BFF5
:104A7000E8340120F0B490F841200346002A40D0E9
:104A80002420DC68D3E9002183F84100012C106860
:104A900021F0706120F0010010601161916821F433
:104AA00000419160996828D041F40441022C916042
:104AB00002D14FF40061516051680020134C202650
:104AC0009F690C43D3E9041554602943DC69D56818
:104AD00041EA07211F6A25F400453C43D560D160B7
:104AE0001460116841F001011160586483F841605D
:104AF000186383F84200F0BC704741F400419160B4
:104B0000DAE702F0FF0180F84010B9E70080000208
:104B10002DE9F04F002383B0DFF810820D68DFF835
:104B200010E203E00133102B00F0B88001229A401C
:104B300032EA050405EA020CF4D14C6824F01007AF
:104B4000022F40F0AE80DF0803F0070A4FF00F0B92
:104B50000E6900EB87074FEA8A0AD7F820900BFA14
:104B60000AFB06FA0AF64FEA430A29EA0B094FF054
:104B7000030B46EA09090BFA0AF604EA0B0BC7F81D
:104B800020906FEA060907680BFA0AFB27EA060677
:104B90004BEA060606608768C4F3001607EA090BAD
:104BA000CF689E4007FA0AF747EA0B078760476815
:104BB00027EA020216434660C668E7008A6806EAEA
:104BC000090902FA0AF242EA0902C260AAD5D8F833
:104BD000447023F0030903F003020F2647F48047D3
:104BE00009F180499200C8F8447009F59C39D8F859
:104BF000447006FA02FA07F480470197444F019E79
:104C0000B842D9F8086026EA0A061AD007F5806784
:104C1000B8425ED03F4FB84260D03F4FB84262D0FA
:104C20003E4FB84264D03E4FB84266D03D4FB84286
:104C300068D03D4FB8420CBF0727082707FA02F299
:104C40001643C9F808606FEA0C07DEF80020E60397
:104C500003F1010354BF3A404CEA0202CEF80020AF
:104C6000A203DEF8046054BF3E404CEA0606E202AE
:104C7000CEF80460DEF8086054BF3E404CEA0606F9
:104C8000A402CEF80860DEF80C2054BF3A404CEA8B
:104C90000202102BCEF80C207FF448AF03B0BDE821
:104CA000F08F4FEA430A4FF00309D0F800B0013FFC
:104CB00004EA090609FA0AF9012F2BEA090B06FA98
:104CC0000AF66FEA090946EA0B0606603FF674AF7A
:104CD00061E7012707FA02F21643B2E7022707FA53
:104CE00002F21643ADE7032707FA02F21643A8E7DC
:104CF000042707FA02F21643A3E7052707FA02F290
:104D000016439EE7062707FA02F2164399E700BF0B
:104D10000000024000080240000C02400010024067
:104D20000014024000180240001C024000380240FB
:104D3000003C01402DE9F8433C4E337D012B6DD002
:104D4000012380460F463375F7F7A0FB0546002880
:104D50005FD14FF0FF333B60D8F80030012B3DD0DE
:104D6000D8E901934B444B4553D9314C2DE0022BEC
:104D70000CBF4FF400734FF44073226922F4407269
:104D80002261226913432361236923F0F80323611D
:104D9000236943EAC90343F002032361236943F40F
:104DA00080332361BFF34F8FF7F770FB236923F044
:104DB0007A032361002835D1D8F8083009F10109B8
:104DC000D8F8042013444B4523D998F80C30002B15
:104DD000D3D0012BCBD14FF48073CEE7144CD8F84D
:104DE0000C3022691B0222F440729BB222612269BC
:104DF00042F0040222612269134343F480332361A9
:104E0000BFF34F8FF7F742FB2369054623F00403F6
:104E10002361002328463375BDE8F8830225284620
:104E2000BDE8F8830546C7F80090F2E7AC530120CF
:104E3000003C0240754B002108222DE9F0411D681D
:104E400082B080460191D0E9166334689A402242CC
:104E500004D001680F68780700F18A8001229A4027
:104E6000224204D0D8F800104969090678D40422F7
:104E70009A40224204D0D8F8001009688F0767D4FE
:104E800010229A40224204D0D8F800100F68380748
:104E900049D420229A40224217D0D8F800100C683A
:104EA000E00612D5B26098F83520052A73D00B6859
:104EB00013F4802F0B6800F09080190340F19B8061
:104EC000D8F83C300BB140469847D8F854303BB343
:104ED000D8F85430DA071BD5D8F8002005214C4B00
:104EE00088F83510A3FB0535136823F00103AD0ADC
:104EF000136002E01368DB0704D5019B0133AB426A
:104F00000193F7D90022012388F8342088F835303E
:104F1000D8F84C3023B1404602B0BDE8F041184704
:104F200002B0BDE8F081B2600A6812F4802F0A680E
:104F30002AD1D70503D40A6822F008020A60D8F8FB
:104F40004020002AA5D040469047D8F85C30A0E722
:104F5000B260D8F8542042F00402C8F854208FE719
:104F6000B260D8F8542042F00202C8F854207EE71C
:104F70000F6827F004070F60B260D8F8542042F0A1
:104F80000102C8F8542069E71203D8D5D8F84820A0
:104F9000002AD8D17DE70A68D8F8404022F01602EE
:104FA0000A604A6922F080024A6154B30A6822F01A
:104FB00008020A603F220024012102FA03F3D8F814
:104FC0005020B36088F8344088F83510002AA7D004
:104FD000404602B0BDE8F041104713F480737FF4FF
:104FE0006FAF0A68012422F010020A6088F834309A
:104FF00088F8354064E7D8F84430002B7FF463AF7D
:1050000063E7D8F84820002AD0D1D3E7542C0120F8
:10501000B5814E1B90F835200346022A03D080222A
:1050200001205A65704702680521002083F8351079
:10503000136823F001031360704700BF70B5324A54
:10504000002590F84130044680F84250283BC26267
:105050004585426C022B41EA020141642BD80321B1
:10506000FCF756FC2822294B80F841204363056356
:105070002268136813F4804312D01368A06B23F4E2
:1050800080431360B0B1224A0023026584F84030A7
:10509000FFF7C0FF70B1A06BBDE87040036D18470B
:1050A000116811F4004114D194F84130602B24D0E0
:1050B00084F8401070BD0721FCF72AFC90F84130BD
:1050C000602B02D0202380F84130002323636363E8
:1050D000CEE71168E06B21F4004111600028E9D0AF
:1050E0000B4A026584F84030FFF794FF0028E1D0B6
:1050F000E06BBDE87040036D1847202384F8401032
:1051000084F8413070BD00BF0000FFFF015201086C
:105110009D1901080368202270B51E680D46DA61EA
:1051200007210446FCF7F4FB03683348596841F44F
:10513000004159605A6802405A609A69910701D546
:1051400000229A629A69D20703D49A6942F0010256
:105150009A6170042BD5A26B1AB11268526892B290
:1051600062856A0709D55A6A25F00405636A1A70D0
:10517000636A228D013363624ABB638D9BB21BB1AC
:10518000636C43F0040363640023236384F84230B8
:10519000666C636316BBE36A184DAB420DD194F89D
:1051A0004130202384F8406084F8413070BD3104E0
:1051B000D7D5E26B002AD0D1D3E72046FCF728FCF4
:1051C0002023E56284F8406084F8413070BD638D2F
:1051D000013A013B22859BB26385CEE7616C204694
:1051E000FFF72CFF94F84130282BDFD129462046C9
:1051F000BDE87040FCF7E0BB00E800FE0000FFFFE8
:10520000F8B590F84030C66A012B00F0848017464C
:105210000123CA0604460D4680F8403020D5FB061F
:105220001ED5438D9BB2002B62D190F84130B6F170
:10523000007FDBB202D1282B00F0848094F841304B
:105240001021292B2368D96102D116F5803F68D13E
:10525000AA0601D5BB0659D4002084F84000F8BD49
:10526000680710D42A072ED53B072CD594F8413077
:1052700003F02803282B61D0216808200023C8618F
:1052800084F84030E4E77907ECD5638D9BB27BB1BD
:10529000216825F00405636A496A1970638D606AA4
:1052A000218D013B01309BB201396062638521850C
:1052B000638D9BB2002BCBD116F5803FC8D0204622
:1052C000FCF7A6FBC4E7A807C2D5B907C0D5638D14
:1052D0009BB213B3606A236810F8016B218D9E6244
:1052E000638D01396062013B21859BB26385AFE725
:1052F00003681021D961436C43F00403436436F022
:105300008073A5D1416CFFF799FEA1E7294620469D
:10531000FFF700FFA0E70220F8BD36F0807397D1B9
:10532000CDE799698A0701D5002199629969CE076D
:10533000C5D4996941F001019961C0E72046FCF7A5
:1053400009FB85E7FCF738FB82E700BF38B5202270
:105350000368204D0024DA615A682A401E4D5A60C5
:1053600004634463CC06C56205D51022DA61426C41
:1053700042F0040242649A69910701D500229A62C0
:105380009A69D20703D49A6942F001029A61032113
:10539000FCF7BEFA436C90F84120602A0CD01A1E2C
:1053A00018BF012243B990F84130212B08D090F862
:1053B0004130222B04D038BD416CBDE838403DE679
:1053C000202380F8402080F8413090F8423080F867
:1053D000422038BD00E800FE0000FFFF38B590F81D
:1053E00040300446C06A012B72D0012384F840305B
:1053F000CB0616D5D50614D5D50B930B45EA9232BC
:10540000D2072BD5E26B03F001035AB3ED0729D580
:105410001268526832BBA26B52B34BB313685B681D
:1054200026E00B0707D4880601D5930612D4002086
:1054300084F8400038BD1507F5D594F8413003F0E5
:105440002803282B46D0236808220020DA6184F83C
:105450004000EFE72046FFF75DFEE8E723681022F3
:10546000DA61E4E7A26B22B31BB313685B6803BB8A
:1054700094F84130282B02D1B0F1007F2ED094F85F
:1054800041301022292B2368DA61D0D110F5803FFA
:10549000CDD09A69910701D500229A629A69D20704
:1054A00003D49A6942F001029A612046FCF7B0FAEF
:1054B000BDE723681022DA61636C43F00403636480
:1054C00030F08073B3D1616C2046FFF7B7FDAEE7D3
:1054D000022038BD2046FCF73DFAA8E72046FCF73D
:1054E0006BFAA4E7F8B590F84030012B7BD001238C
:1054F000CD06044680F8403023D5D00621D51022B1
:105500002368616B4548DA61626C814242F00402B3
:10551000626466D0424A914263D0F4211A680A4319
:105520001A609A69910701D500229A629A69D20796
:1055300003D49A6942F001029A61002084F8400085
:10554000F8BD0B0631D5570643D523681A6822F0FB
:1055500040021A60628D92B2002A46D05868618D6E
:10556000C0F309008AB2FF2A4BD8628DE56A91B276
:1055700015F5803F2185CDB24BD0E76A2D045A68DE
:10558000284E324002433A432A435A60628D521AEF
:1055900092B2628594F84120222A1A680CBF42F424
:1055A000004242F480421A60C7E74D0611D550060A
:1055B0000FD5638D9BB2FBB923685A689101BCD4A7
:1055C000E26A12F5803F13D15A6842F480425A6071
:1055D000B3E78B06B1D59206AFD52046FFF7B6FEEE
:1055E000ABE760219AE70220F8BD5B689E0103D417
:1055F0002046FCF731FAA0E740212046FFF71EFDC8
:105600009BE7FF224FF47F054FF0807711462285FC
:10561000B5E74FF000772D04B1E700BFDD53010877
:10562000E5540108009C00FC90F84030012B00F08C
:105630009C8001232DE9F041044680F84030C806E3
:105640000D4690461BD512F0100F18D0236810217C
:10565000D961616C41F0040161649969890701D5E0
:10566000002199629969CA0764D5AB0602D518F082
:10567000200F71D1002084F84000BDE8F0816B0755
:1056800012D4AF0724D518F0020F21D0606A236826
:1056900010F8016B218D9E62638D01396062013BC0
:1056A00021859BB26385E0E718F0040FE9D02168FB
:1056B00025F00405636A496A1970638D606A218D5B
:1056C000013B01309BB20139606263852185CCE7E3
:1056D0002E0615D46906C8D518F0400FC5D0638DC5
:1056E0009BB2002B33D1236859688A01BDD4E16A8B
:1056F00011F5803F27D1596841F480415960B4E7E2
:1057000018F0400FB1D0638D9BB2C3B1238DB3B9F4
:1057100020684168638DC1F309019BB2FF2B26D934
:105720004368FF27204E27853340204E19430E4300
:1057300046609AE7996941F00101996195E723680C
:105740005B68980103D42046FCF786F98DE7402179
:105750002046FFF773FC88E720462946FFF7F6FD51
:10576000002084F84000BDE8F08102207047638D7E
:10577000E66A9BB216F5803F23850AD0E76ADBB262
:105780004668094A16403E4346EA034319434160CE
:105790006BE74668DBB2044F3E40314341EA0343C6
:1057A00043F00073436060E7009C00FC0000FF01D1
:1057B000F0B4044690F834000128A66D38D00125D5
:1057C00094F83500A84284F8345005D00023022014
:1057D00084F83430F0BC704725680227002084F834
:1057E0003570A76860652868402F20F48020286005
:1057F0006B601AD0A960EA60E16D3F23226C8B4098
:10580000B3602B6843F016032B606B6943F0800391
:105810006B611AB12B6843F008032B602B680020E2
:1058200043F001032B60F0BC7047AA60E960E3E736
:105830000220F0BC704700BFF0B490F83530022B66
:1058400034D0036800221B4D2127D9B21E681039BD
:1058500026F00106A5FB0145174C5F291E6004EBED
:1058600015141A605A6094F850409A60DA601A6110
:105870005F61C46515D8114A1A4000233F21826533
:10588000A1401C469160436580F8343080F8353083
:10589000C0E90F33C0E91133C0E913332046F0BC2F
:1058A0007047A2F580621A400432E6E7DCB2204677
:1058B000F0BC7047ABAAAAAA24EE050800FCFFFFC3
:1058C0000246F0B44A4C2068002A57D002231168DF
:1058D000002582F8353082F834500B6823F001033C
:1058E0000B6003E023681B1A052B3FD80B68DD070C
:1058F000F8D4D2E90130D56803430F68D2E90440F7
:105900002B432343146AD2E90665034339483343E2
:1059100038402B43556A2343042D40EA030030D01E
:1059200008604B6923F007031D43CBB2324C4D6135
:10593000103B3248A4FB03545F2B314B4FF0010561
:1059400000EB14104FF0000403EA01034FF03F0195
:1059500090F8500088BF04338140D065204693659D
:105960009960546582F83550F0BC704703232021BC
:105970001846516582F83530F0BC70470120F0BC04
:105980007047D2E90B74936A3C43204308604D6929
:1059900025F007051D4345F00405002FC5D07EB155
:1059A000B6F5005F12D0022B03D9032BBDD1FB014A
:1059B000BBD5012340211846516582F83530D3E725
:1059C000012B11D033F00203AFD1F0E7032BACD899
:1059D00001A050F823F000BFB3590108AF590108E6
:1059E000B3590108E9590108B7F1C07F9DD1E0E73B
:1059F000E83401203F8010E0ABAAAAAA24EE0508F3
:105A000000FCFFFF002807DB00F01F010123400915
:105A1000024A8B4042F82030704700BF00E100E0AE
:105A2000034A0130116813685B1A8342FBD3704745
:105A3000E834012090F8BC33012B18D00368012210
:105A400010B50446032084F8BC23D3F8042822F0C0
:105A50000202C3F80428FFF7E3FF216800228B68E5
:105A6000104643F001038B6084F8BC2310BD022074
:105A700070470D4B93F8F222D20703D5012283F829
:105A80005824704793F8582462B9D3F830234AB1A8
:105A900093F8E822104493F8E922114483F8E802CD
:105AA00083F8E912704700BF185C0120044B93F99A
:105AB0000000012802D102221A70704700207047AE
:105AC000185C0120114AD2F85C04A0B1D2F860340D
:105AD0008BB188420DD88B4234BF002301239BB188
:105AE0005368C2F86414994202D0142382F86834CF
:105AF000DCE70023F3E7A1F59C53083BB3F57A7F7D
:105B00002CBF00230123EAE7704700BF185C012087
:105B1000002307B50DF10602ADF806300AF012FCBD
:105B200060B1084BBDF806201989A3F86A24914298
:105B300002D0142283F86C24FFF7B8FF03B05DF89D
:105B400004FB00BF185C012013B504462620019118
:105B500019F0E8FC019948B9054BD3F8DC322BB1B8
:105B6000204602B0BDE81040FCF7BEBA02B010BD3E
:105B7000185C0120B1FA81F149204909E4E72DE9D7
:105B8000F341BE4C0D4694F90030013300F06681BC
:105B9000D4F8DC32002B00F0B380022700264FF04F
:105BA0000108D4F8DC022EF07FFA002800F0A8806B
:105BB000D4F8DC022EF070FAD4F8E4325A1C2344F4
:105BC00083F86D0494F8E032C4F8E422012B09D084
:105BD000022B15D063B90F280CBF84F8E082C4F8FB
:105BE000E432DEE7A0F17203012B06D9762804D057
:105BF00084F8E062C4F8E462D3E784F8E072D0E7A6
:105C0000102ACED19E490023012211F8010F013242
:105C100003440E2ADBB2F8D194F87B2484F8E062C6
:105C20009A42C4F8E462BCD194F87C34002BB8D119
:105C300094F86E34732B59D0762B1BD0722B5FD116
:105C400094F8702494F86F3494F9001053EA022306
:105C500056D0C4F85C340029B4F87134C4F8603408
:105C60004EDC012394F88A242370002A48D184F85A
:105C70008A3445E094F8702494F86F3453EA022390
:105C80003ED0D4F880246360934202D0142284F87A
:105C9000682494F8721494F87124C4F8803442EAA9
:105CA0000122B4F884149142228102D0142184F894
:105CB0006C1494F8731494F87604617094F8741466
:105CC000A4F88424A17094F8751441EA0021A4F882
:105CD0008614D4F8641409B9C4F86434B4F86A3486
:105CE0000BB9A4F86A240223237009E094F8742401
:105CF00094F8733443EA02231AB20BB1A4F888244F
:105D000094F90030022B35D00FDCDAB2012A15D914
:105D1000A36D13B1E368002B6CD11F2259495A4877
:105D200002B0BDE8F04148F0A7BA032BF0D1D4F897
:105D30008C34564AEB1A9342EADD13E0D4F88C24F3
:105D40005349AA1A8A42E3DD2BB97220FCF7F8F90D
:105D5000C4F88C54DCE7D4F890345A1CD907C4F842
:105D6000902403D47620FCF7EBF9F1E77320FCF7DD
:105D7000E7F9EDE7D4F86414D1B194F86834BBB115
:105D80006368994214D06378DA0703D489B2462055
:105D9000FFF7DAFE94F86834013B84F8683405F5BF
:105DA0009225032305F578752370C4F88C54AFE76A
:105DB000B4F86A14238981B194F86C246AB18B42D7
:105DC0000BD06378DB0702D45020FFF7BDFE94F8B8
:105DD0006C34013B84F86C34E1E70122A4F86A34A6
:105DE00000232270626884F86C34C4F8642484F858
:105DF00068348DE7274D2A23D4F830730DF107025C
:105E000085F8203020230DF10601384685F8213031
:105E10000AF096FB30B19DF806109DF8076051EA34
:105E200006031ED1552385F82230462385F82330FA
:105E300020236268184885F82430002A34D0174996
:105E40003DF082FFB4F8863415488BB3228915499A
:105E50009A420CBF20222A223DF076FF02B0BDE814
:105E6000F08138460AF0EAFA314685F822003846D1
:105E70000AF0D0FA037885F82330D9E7185C0120BE
:105E8000856001206C71060864030120400D030049
:105E900040420F004403012069030120B7A906080E
:105EA0006D0301208671060803493DF04DFFC9E7E7
:105EB00002493DF049FFD1E78E7106088D71060851
:105EC00040F0080210B50C4C84F8432094F90020EF
:105ED000022A05DD420703D5830701D0012323727F
:105EE00005210648FBF7C0FE062184F8440003485C
:105EF000BDE81040FBF7A0BE44030120830301204E
:105F000010B5FBF74DFE98B31A4C94F90030012BF5
:105F10002EDD49B3022B2BD0237A9BB971B180239C
:105F20000521154884F84930FBF79EFE062184F8C8
:105F30004A001148BDE81040FBF77EBE0420BDE8D2
:105F40001040BDE7002914BF00200420E3781A07A1
:105F500048BF40F002005B0701D411B108B940F01E
:105F60000100BDE81040ABE7022BD5D10420EDE7DE
:105F700010BD00BF4403012089030120F8B5214C66
:105F8000030A0546062104F14B0784F8500084F803
:105F90004F303846FBF768FEE37884F85100DB07A2
:105FA00029D4A288AA4226D1174D41F26F71D4F8A4
:105FB0004B3005F29446C5F89434C3B2304685F8A8
:105FC0009A344FF6FF738A4218BF01230621134407
:105FD000C3F3072285F8993485F89824FBF744FE2B
:105FE000072185F89A043046FBF726FE052104F1C7
:105FF0005200FBF721FE07210448BDE8F840FBF7FB
:106000001BBE00BF44030120185C01208F03012048
:1060100008B5FBF7C5FD48B1A1F59C53083BB3F5A6
:106020007A7F03D20846BDE80840A7E708BD2DE9FE
:10603000F8436A4E3368002B38D0694C694D30689C
:106040002EF032F8002833D1674B19881D460929F4
:1060500009D95F8864227A43B2FBF1F2452A40F302
:106060009A811880588094F8D534012B00F0BA81B9
:10607000022B00F0D38133B905215C48FBF7DCFD2E
:10608000012384F8D5345A4B1D685A4B1B78002BDA
:1060900000F0CD81584B1B68EB1A782B40F2C7817A
:1060A000D4F82C03F9F770FAC4F8D854BDE8F88393
:1060B00030682DF0F1FF94F89B340746052BBED8CD
:1060C000DFE803F00309171D3745AA28B7D10123DC
:1060D00084F89B34B3E7552803D1022384F89B341A
:1060E000ADE7414A938801339380002384F89B34C1
:1060F000A5E7032384F89C0484F89B349FE71328C6
:1061000084F89D04C4F8B80407DD374AD388013306
:10611000D380002384F89B3491E718B9052384F8D1
:106120009B348CE70023C4F8BC34042384F89B34EC
:1061300085E7D4F8BC34E218013382F89E04D4F821
:10614000B824C4F8BC3493427FF479AFE6E7D4F8BE
:10615000B8342A4803F102094FFA89F1FBF784FDAC
:10616000874294F89C8440F00D81262019F0DAF9DA
:10617000204B48B100221A701B4A538801335380C8
:10618000002384F89B345AE71A78424519D100223B
:106190001A7008F1FF33102B00F2EF80DFE813F0E4
:1061A000300088008800D9008800ED00ED00ED0087
:1061B0003000ED00ED00ED00ED00ED00ED00ED0034
:1061C0003000B8F1090F02D0B8F1110F01D1012A46
:1061D000DDD0054A538901335381DAE71059012094
:1061E000185C01204403012034590120960301204A
:1061F000C42901204259012044590120B4600120E2
:10620000B9F1060F54DDB8F1010F06D0B8F1090F4E
:106210000CBF4FF002084FF0030894F8A10494F863
:10622000A21494F8A02441EA002194F99EC494F9A0
:10623000A074900709B294F89F3485F8008085F81F
:1062400001C0EF70A98005D512F00C0F14BF012218
:1062500000222A72B8F1030F11D1B9F1090F27DD1D
:1062600094F9A4240023082AA8BF082222EAE27293
:10627000EA7558B20133824259DC94F8A334002005
:10628000D4F80C909BB202464A45964657DB784BB1
:10629000A8701B78232B0BD108EB8803754A03EBFE
:1062A0008303A2F802C0918007EB8303D0801380A0
:1062B0000A227149284647F0BFFE10B1002384F836
:1062C000CA346D4B2A681A606A685A602A891A8132
:1062D00094F8CA3433BB2B7A94F8E822002B14BF0D
:1062E0000223012384F8CA34EB7813F0010302D0AF
:1062F000B2FA82F35B0984F8CC24D9B294F8E9228B
:1063000094F8EA0284F8CD24B4F8EC2284F8CB1493
:10631000A4F8CE2484F8D00413B10AB1A4F8D2248E
:1063200084F8D4140AF072FD0AF070FD24E704EB3F
:10633000400E204490F8A604AEF81C0399E7013201
:1063400004EB4E0E52B2BEF810E09E4508BF104658
:106350009AE7B9F1040FABDD94F89E2494F89F34CA
:1063600043EA022359041AB203D5C3F30D03EB80A9
:106370009EE7002AF9DBAB809AE7404A9389013314
:106380009381F9E618F0010F7FF4FAAE3B4A1389C6
:1063900001331381F4E63A4B9A6DB3F85C10012A8D
:1063A00018D141F25632914202D14FF0FF329A6534
:1063B0009A6D306802EB820202EB820201EB42012D
:1063C00089B2A3F85C1003681B69984700232B80EF
:1063D0006B8048E60132EBD1B1F5965FE8D101223E
:1063E0009A65E5E7264D95F90060002E3FF44BAE27
:1063F000022E0FD14FF48040FFF7C0FD84F8D56422
:1064000095F90030012B7FF73EAEEB78C3F34003E4
:106410002B7238E6032384F8D534F1E7184BDB8878
:10642000002B3FF430AE032384F8D5342BE694F8E8
:10643000242094F825309A4204D0FBF76DFFC4F86D
:10644000D85433E6D4F8D834EB1AB3F57A7FBFF4D6
:106450002DAE0C4B1B68ED1A952D7FF627AE05214E
:106460000948FBF7E9FBBDE8F843FBF755BF00BF60
:106470008549012088490120D86001203459012034
:1064800044030120445901209603012010B5134C08
:10649000D4F8300308B394F8E81251B194F8E92223
:1064A00009F064FFB4F8EC32834212D00121A4F861
:1064B000EC02B4F8EE2272B141F288339342B8BFD5
:1064C00013469A4207D0A4F8EE32BDE8104036F0E9
:1064D000F9BC0021EDE70029F7D110BD185C0120BF
:1064E0000023014410B410F8014B0822634002E07D
:1064F000013AE3B209D013F0800F4FEA4304F7D01A
:1065000084F00703013ADBB2F5D18842EBD118469B
:106510005DF8044B704700BF30B54FF4806085B024
:1065200026F078FB48B3164C002301214FF4E132EA
:1065300094F8DC5490F904009D42019100924FF4CC
:10654000806118BF08250F4A029526F0C2FB20661D
:1065500000384FF0FF0318BF012084F87C3084F826
:106560008C3084F89C3084F8AC3084F8BC3084F8EB
:10657000CC3084F8DC3084F8EC3005B030BD00BF9E
:10658000185C0120151F0108384B1B6813F00063CD
:106590005DD0374B2DE9F0471F78B84252D3FF2822
:1065A00057D1DFF8E0A09AF81030002B47D0DFF881
:1065B000D8800022C8F8E024C8F8E424C8F8E82409
:1065C000A8F8EC24002F4DD008F17C0310461446A7
:1065D00011461546164603EB0719B3F802E01033CF
:1065E00033F804CC714413F810EC624413F90FCC67
:1065F000764509B212B238BF7646654553F80CECC1
:10660000B8BF654653F808CC994574446044E4D15A
:1066100088F8E06488F8E154C8F8E444C8F8E8046D
:1066200091FBF7F192FBF7F2124B0020A8F8E2146D
:106630001B78A8F8EC24092B8AF810000CD00E481F
:10664000BDE8F0870D4A02EB0010BDE8F087184660
:1066500070470020BDE8F08798F8E024084B064812
:10666000DA80F2E73A463946DEE700BF30570120CC
:10667000800A002085490120F8600120945C0120F7
:106680008849012044030120185C0120F8B53B4EE5
:10669000054601687E20B6F9F034394A4F1C03EBF9
:1066A000C3032F6082FB0342DC170870FF202B68B6
:1066B000C4EB62040022591C20342960A4B21A7071
:1066C000FFF762FF2F4B00284CD01B78B0F90C105D
:1066D00023BBA1F57A722C4B9A4245D82B48B0FBCC
:1066E000F1F189B228463DF02FF996F85733B6F804
:1066F000441328467BB196F87033B1FBF3F13DF0BB
:1067000023F9214628463DF01FF928460821F6F7CF
:1067100069FE0120F8BD3DF017F9F2E71C4B1F7828
:10672000002FD6D000231B4800EB8302013392894F
:10673000BB421144F8DB184B07EE901A9FED176A25
:106740009B7EF8EE676A07EE103AB8EEC77AC6EE9F
:10675000077A67EEA67AFCEEE77A17EE901AB1FB9D
:10676000F7F1B6E71B7813B94EF69C21BAE7084B50
:106770001F78002FF8D00146D4E700BF185C012035
:10678000676666667009002017839303008793038A
:10679000800A0020B8110020CC29012000004843C5
:1067A0002DE9F8434378434C190703F00F0594F89B
:1067B000F22400D072B10021AA4284F8F41404D962
:1067C0004FF000084046BDE8F883AA1AD1B20E295E
:1067D000F6D803E084F8F25484F8F424224492F8C2
:1067E00058130029ECD003F0F003802B40D0902BFD
:1067F00049D0A02BE4D1084665F05F05FBF7C8FB44
:1068000002462D48131D84F8F55484F8F434FBF740
:1068100013FF94F8F484B8F1000FD1D0A8F102036B
:1068200013F0FF0641D0254A4FF6FF71901912F878
:10683000015B491B904289B2F9D15FFA81F90D0AD7
:106840004BB11E4FFE1817F8011BD4F818052DF098
:106850002FFCBE42F7D14946D4F818052DF028FC8C
:10686000D4F8180529462DF023FC4046BDE8F883EE
:10687000042365F07F050226984684F8F43484F8F2
:10688000F5543346CFE7084665F06F05FBF780FB0C
:106890000426062284F8F704334684F8F55490461B
:1068A00084F8F61484F8F424BDE7FF254FF00208BD
:1068B000A946C5E7185C01200E6101200C6101208A
:1068C000C21D2DE9F04702F4FC7282B0DFF830817E
:1068D0000C4600AFD8F81861ADEB020DD8F81031B6
:1068E000C7F800D0684432686D4678609A4298F8DC
:1068F0001C3559D0591C0DF1010203F00F033A6009
:1069000088F81C158DF80030A0EB0209D6E90012BA
:106910005FFA89F9521A09F107035FFA82FA03F460
:10692000FC73CA45ADEB030D57D25246684647F09B
:1069300039FB3368524669465344384633603CF06D
:10694000E3FFD8F810313068D8F81811C21A834222
:10695000097A706082EA01023360D2B288F81D259C
:1069600009D001333360984213F8011C82EA010216
:10697000F7D188F81D253B68591C39601A70D7E992
:106980000032D21A012A08DD00215A1C3A6019701F
:10699000D7E90032D21A012AF7DC2846A0470020A6
:1069A0000837BD46BDE8F087B6F90C20591C03F046
:1069B0000F03002A88F81C1543F0100305F10101AC
:1069C0002A46B8BF43F02003396002F8023BD6E9FB
:1069D00000133A605B1A6B7096E74A46684647F0C8
:1069E000E1FA33684A4669464B44384633603CF026
:1069F0008BFF2846A04701200837BD46BDE8F08739
:106A0000185C01202DE9F04F784C83B09046834606
:106A1000D4F8186100AF0D46D6E900239B1A002B6D
:106A200028DD002384F81E35FBF706FB00200BEB66
:106A300005030BF1010AD4F81451C4E941A39BF8F2
:106A400000607109012940F09D8006F00F0916F0E1
:106A5000100614D150B194F82025013202F00F0233
:106A60004A4500F09880304684F81E650C37BD46D4
:106A7000BDE8F08F94F81E050028D8D1D4E70BF1BB
:106A800002030BF10302D4F80C014FF0000CC4F820
:106A900004319BF80130C4F804219BF80260C2184D
:106AA000286073406A6084F81E1584F81F352E81B3
:106AB000A5F80CC0D4E941A3A3EB0A03121ADEB275
:106AC0005FFA82FBF31DB34503F4FC73ADEB030DDA
:106AD0006ED25A465146684647F064FA0AEB0B03F9
:106AE0005A4628466946C4F804313CF00DFFD4F8F4
:106AF0000C31286894F81F258342C5E9003009D07D
:106B000001332B60984213F8011C82EA0102F7D18D
:106B100084F81F25D4F804311B7893423ED1B5F98F
:106B20000830FA2B05D1B8F1000F02D0052388F800
:106B300000302A680026D4F80C113B1DD4F8C0029E
:106B400084F81E65C5E90012D4F81821D4F8101194
:106B5000168151609681D4F814117E6026F0D2FC23
:106B600001303AD07B680BB100209847D4F8183137
:106B70000120D4F810110C371A68C3E90012BD4681
:106B8000BDE8F08F00210846FBF73AFA01200C37E8
:106B9000BD46BDE8F08FD5E900028DE70023012056
:106BA000B5F9081084F81E35FBF72AFA01205DE7D5
:106BB00032465146684647F0F5F90AEB0603284687
:106BC00032466946C4F804313CF09EFE00200C3782
:106BD00084F82095BD46BDE8F08FD4F81821022135
:106BE0001368581C10601970BCE700BF185C0120C6
:106BF0000B4B93F88E2312B1B3F8682352B9094BAB
:106C0000094AB3F9043082FB0312D817C0EBA20083
:106C100000B27047D3F8A80390FBF2F000B27047BF
:106C2000185C01209C58012067666666F8B5054629
:106C3000174CEEB2D4F82405C5F3072731462DF0E2
:106C400037FA94F828353946D4F824055E4084F89C
:106C500028652DF02DFA94F82835C5F30746D4F8A9
:106C600024052D0E5F40314684F828752DF020FA5A
:106C700094F828352946D4F824055E4084F8286520
:106C80002DF016FA94F82805454084F82855F8BDEB
:106C9000185C012070B504460B4DE6B2D5F824050A
:106CA000240A31462DF004FA95F828352146D5F806
:106CB00024055E4085F828652DF0FAF995F8280539
:106CC000444085F8284570BD185C012038B50B4C50
:106CD000002305462421D4F8240584F828352DF016
:106CE000E7F9D4F8240554212DF0E2F92946D4F827
:106CF0002405BDE838402DF0DBB900BF185C012049
:106D00002DE9F043DFF870930E46154699F82945B2
:106D10002DED028B83B0002C00F0E581013C89F859
:106D20002945CD4F9FEDCD8ADFF850833378002B76
:106D300000F08E8099F82945002C40F0898035B10B
:106D40002BF082FF2B68C01A002880F2B48399F8D8
:106D50002A25002A40F0528399F82B05062840F294
:106D60008F81BF4B93F8651093F864408C4200F01C
:106D7000AA8153F8604F013099F82CC54A1C34F8A9
:106D80001140C0B2D2B2644489F82B055A71A4B242
:106D9000B4F5C06F00F08A817CD8B4F5806F00F044
:106DA000248224D8B4F5067F4FD8B4F5007F54D39D
:106DB000A4F50073182B48D8DFE813F0EB01E201CB
:106DC000E201E201E201E201E201E201E201470047
:106DD000470047004700470047004700C701AC0194
:106DE000AC01AC01AC01AC01AC01AC01AC01B4F53F
:106DF000846F00F0EA8140F2EB80B4F5A06F00F000
:106E000059826FF4A06C04EB0C03072B1DD8601E95
:106E1000C0B2FFF7B9FBC0B1B0F90C301021914AF4
:106E2000684603EB83038DF80010917E03EB830328
:106E3000D9F8C4224908ADF801409B0093FBF1F357
:106E4000CDF80330904700233370002D7FF46EAFF0
:106E500003B0BDEC028BBDE8F083B4F5807F00F099
:106E60004F82B4F5887FF0D1B9F9AC131023012219
:106E70000024CDF803108DF8003068468DF80130FD
:106E80008DF80220D9F8C43298473470002D7FF471
:106E90004DAFDDE7B4F5046F00F0748277D8B4F538
:106EA000006F00F0518228D9B4F5026F00F0F28132
:106EB000B4F5036FC9D199F840339C07C5D56A4A28
:106EC00010214FF4F3630024D28968468DF8001036
:106ED000302103FB02F308228DF80110A7FB0313F6
:106EE0008DF802205B09D9F8C422CDF80330904711
:106EF0003470002D7FF41AAFAAE7B4F5E26F00F00A
:106F00001282B4F5E46F1FD1584B002493ED170A99
:106F1000D3ED007A20EE270A20EE080A44F03CFD6B
:106F2000102120220723CDF803008DF800108DF8E2
:106F300002306846D9F8C4328DF801209847347081
:106F4000002D7FF4F3AE83E7B4F5E06F7FF47DAFFF
:106F5000464B002493ED150AD3ED007A20EE270A64
:106F600020EE080A44F018FD10220723CDF8030094
:106F70008DF802306846D9F8C4328DF800208DF8BB
:106F8000014098473470002D7FF4D0AE60E740F6A2
:106F900078339C4249D8B4F5376F00F2B981B4F523
:106FA000116F00F06F81B4F5376F7FF44EAFFF20A3
:106FB000FFF7EAFA00283FF448AF90F901001021EA
:106FC00070220B230024CDF803008DF80010AEE7EB
:106FD00040F201439C4200F0F081B4F5826F7FF4EF
:106FE00034AFD9F80031980600F11782204B1B68A6
:106FF0001B0640F16682002410220421D9F8C43215
:1070000068468DF800208DF801208DF803408DF83A
:1070100004408DF805408DF806408DF80210984721
:107020003470002D7FF482AE12E745F230239C428B
:1070300000F01C8145F240239C427FF406AF0D49CD
:10704000102040225223B1F9001000248DF80000D6
:10705000CDF803106BE700BF1F85EB510000C8425D
:1070600044030120CC290120105801205411002094
:10707000305701209C580120185C0120C5B3A29113
:107080000130D34BC0B293F86D1093F86C208A4254
:1070900014D04A1C4900D2B29C6ECE4B645A89F877
:1070A0002B05B4F5C06F5A717FF476AED9F8A813EA
:1070B000102200240623CDF8031059E700210122F5
:1070C00083F86D10E8E799F82C15C348013183F86F
:1070D00065200078C9B2013089F82C15814200F092
:1070E00089810120CFE700283FF41BAE0378303BB5
:1070F000012B3FF616AE013009F229520621FFF7A7
:1071000081FC99F8293589F82A05002B3FF409AE4E
:10711000347006E6A4F11100C0B2FFF735FA00287A
:107120003FF493AEB0F9022010236846ADF8014059
:107130008DF80030CDF80320D9F8C43298470023E9
:107140003370002D7FF4F2AD82E699F85723B9F839
:107150004433002A40F0A981102202210024CDF8F6
:1071600003306846D9F8C4328DF800208DF801202C
:107170008DF8021098473470002D7FF4D7AD67E684
:10718000601EC0B2FFF700FA00283FF45EAE42680E
:10719000CAE7D9F8A0331022904900248DF80020C6
:1071A000DA1781FB0313022168468DF80140C2EB18
:1071B000A3038DF80210D9F8C422CDF8033090470C
:1071C0003470002D7FF4B2AD42E699F840339A074F
:1071D0007FF53BAEB9F8420310212022042300249E
:1071E000CDF803008DF80010A1E699F8343501338D
:1071F000DAB2042A00F04E8142F2107389F8342585
:1072000003FB02F3D9F83825002A00F00481023389
:1072100099F8F222D007724A128848BF0433D10786
:1072200048BF0A33940748BF1433D00548BF2833FA
:1072300051074FF0100148BF643354064FF000046B
:107240004FF0040248BF03F57A63CDF80330684677
:10725000D9F8C4328DF800108DF801408DF8022065
:1072600098473470002D7FF461ADF1E55D49102041
:1072700030225223B1F9021000248DF80000CDF81D
:10728000031054E699F87033002B40F00981102266
:10729000092163E799F840339B077FF5D6AD524942
:1072A000102020220823896800248DF80000CDF8E2
:1072B00003103CE6FF20FFF767F900283FF4C5AD57
:1072C000B0F90C301021494A002403EB83038DF8F8
:1072D0000010917E052203EB8303684649088DF870
:1072E00002209B00D9F8C4228DF8014093FBF1F3F2
:1072F000CDF8033090473470002D7FF417ADA7E52B
:10730000D9F83015102200240123CDF803102FE600
:10731000A4F17100C0B2FFF737F900283FF495AD32
:1073200090F9012000E7324B002493ED160AD3EDCB
:10733000007A20EE270A20EE080A44F02DFB1023E5
:107340000722CDF8030096E599F8403398077FF5BA
:107350007CADD107244B40F1C1805A6882EAE273C8
:10736000002AA3EBE27303EB5303A7FB03134FEADB
:10737000D303ACBF43F0004343F04043102100244B
:10738000082262E7174B102240210024B3F9043091
:1073900068468DF80020082203EB83038DF8011066
:1073A0008DF802205B00CDF80330D9F8C43298473D
:1073B0003470002D7FF4BAAC4AE5B9F9F00410211D
:1073C000012204230024CDF803008DF80010AEE55F
:1073D00044030120AC030120800A00206766666632
:1073E000C05801209C58012010580120CC290120B0
:1073F00054110020012089F82C2544E65D4906201F
:10740000FFF75EFA002389F82A05337003B0BDEC5C
:10741000028BBDE8F0830133FAE6574A99F840132E
:10742000508A6438C0EB4073C0EBC30088FB003463
:10743000C31720440024C3EB20230933092BA8BF22
:10744000092311F0020F23EAE37314BF4FF47A709B
:107450000020C90703EB83034FF0040148BF00F588
:10746000FA6003EB83039B009BB20344107D102260
:107470008DF80210034468468DF80020CDF80330E3
:107480008DF80120D9F8C43298473470002D7FF46C
:107490004DACDDE4012242F2107389F83425B1E6E7
:1074A000B9F84423B2FBF3F3F1E699F87023002A0C
:1074B00058D1134650E6347003B0BDEC028BBDE8E2
:1074C000F08399F85633002B3FF4BFAC99F83C3564
:1074D000032B4AD8DFE803F03C3223121A6882EA11
:1074E000E273002AA3EBE27303EB5303A7FB03133E
:1074F0004FEAD303B8BF43F080433FE7D9F84025B4
:107500000020537A917A03F14073D27A89F83C05CE
:1075100003EB012303EB0243102204211EE6174A6A
:1075200011688A7D087C1204897A02EB00220A44E1
:10753000591C02EB036389F83C15EDE70F4A11680B
:107540004A7DC87B1204497A02EB00220A44EFE725
:107550000A4A11680A7D887B1204097A02EB00222C
:107560000A44E5E7B3FBF2F3F6E55A1C1B0689F87B
:107570003C25D1E7792001081058012098580120B6
:1075800030B5044683B00D461046A4F17D03012BAF
:1075900008D921462CF08CFD15B1288804442C8094
:1075A00003B030BD7D2101922CF082FD019884F062
:1075B00020012CF07DFDEFE70F4A002330B5D2F813
:1075C000442585B00446C51DADF80E3014F8010BF6
:1075D0000DF10E010192FFF7D3FFA542019AF5D1FB
:1075E0000DF10E0011F034FE019A00219DF80E00FD
:1075F000FFF7C6FF05B030BD185C0120034A044BFD
:10760000D2F848150B43C2F848357047185C012082
:1076100000FC0600013070B5094EC4B202E03CF037
:107620002BFE50B9E5B2214630460134152DF6D96E
:10763000162D02D1034B93F84C55284670BD00BF60
:1076400060610120185C012000B1D7E7034A044BB8
:10765000D2F848150B40C2F848357047185C012035
:10766000FF03F9FFF0B5114C85B005460E46D4F87E
:10767000500525F08FFA94F8502394F85133003ACE
:1076800018BF01220BB142F0080200234FF49647C5
:10769000029208211A46019695F90000009725F0FC
:1076A00018FBC4F8500505B0F0BD00BF185C012000
